:100000000C9425210C9450210C9450210C945021D7
:100010000C9450210C9450210C9450210C9450219C
:100020000C9450210C940BD30C9450210C9450211F
:100030000C9450210C9406920C9450210C94502155
:100040000C9450210C94AB9A0C9421D00C94502118
:100050000C94503D0C9450210C9450210C94502140
:100060000C9450210C9450210C9486C80C9450216F
:100070000C9450210C9450210C9450210C9450213C
:100080000C9447900C9450210C945021084AD73B73
:100090003BCE016E84BCBFFDC12F3D6C74319ABD57
:1000A00056833DDA3D00C77F11BED9E4BB4C3E917B
:1000B0006BAAAABE000000803F05A84CCDB2D44E6A
:1000C000B93836A9020C50B9918688083CA6AAAA6C
:1000D0002ABE000000803F4D383420582059205A55
:1000E0002045006563686F3A0043616E6E6F74204F
:1000F000656E746572207375626469723A20004D92
:100100003234004D3233202573006175746F2569D8
:100110002E67004572726F723A006572726F7220BC
:1001200077726974696E6720746F2066696C650008
:100130004E6F74205344207072696E74696E67004C
:100140002F005344207072696E74696E6720627963
:10015000746520002E0044656C6574696F6E2066BE
:1001600061696C65642C2046696C653A20004669BB
:100170006C652064656C657465643A002E006F7070
:10018000656E206661696C65642C2046696C653A11
:10019000200057726974696E6720746F2066696CFD
:1001A000653A20002E006F70656E206661696C658F
:1001B000642C2046696C653A20002E006F70656ED5
:1001C000206661696C65642C2046696C653A200084
:1001D00046696C652073656C6563746564002053C3
:1001E000697A653A200046696C65206F70656E65B6
:1001F000643A20002E006F70656E206661696C6540
:10020000642C2046696C653A20004E6F7720667238
:100210006573682066696C653A20004E6F772064CC
:100220006F696E672066696C653A20002220706FE6
:1002300073002220706172656E743A220053554239
:10024000524F5554494E452043414C4C20746172E5
:100250006765743A2200747279696E6720746F2042
:1002600063616C6C207375622D67636F64652066D3
:10027000696C6573207769746820746F6F206D6195
:100280006E79206C6576656C732E204D4158206C1C
:100290006576656C2069733A002E0A0044656C65CA
:1002A00074696F6E2862696E29206661696C656485
:1002B0000046696C652862696E292064656C657406
:1002C00065640057726974696E6720746F2066698F
:1002D0006C653A20002E0A006F70656E20666169B9
:1002E0006C65642C2046696C653A20005344206399
:1002F000617264206F6B006F70656E526F6F742057
:100300006661696C656400766F6C756D652E696EEB
:100310006974206661696C656400534420696E6984
:1003200074206661696C006563686F3A00486172A9
:1003300064636F6465642044656661756C74205302
:10034000657474696E6773204C6F61646564002026
:1003500044002049002020204D33303120500050EF
:1003600049442073657474696E67733A00205A00BB
:1003700020590020204D323036205800486F6D65DE
:10038000206F666673657420286D6D293A002045DC
:1003900000205A0020580020420020540020204D08
:1003A000323035205300416476616E636564207697
:1003B00061726961626C65733A20533D4D696E20CC
:1003C000666565647261746520286D6D2F73292CD4
:1003D00020543D4D696E2074726176656C206665AF
:1003E00065647261746520286D6D2F73292C20421D
:1003F0003D6D696E696D756D207365676D656E74B1
:100400002074696D6520286D73292C20583D6D611D
:1004100078696D756D205859206A65726B20286D5A
:100420006D2F73292C20205A3D6D6178696D756D93
:10043000205A206A65726B20286D6D2F73292C203D
:1004400020453D6D6178696D756D2045206A657246
:100450006B20286D6D2F73290020540020204D3211
:100460003034205300416363656C65726174696F59
:100470006E3A20533D616363656C65726174696FA8
:100480006E2C20543D7265747261637420616363E5
:10049000656C65726174696F6E00204500205A00BA
:1004A00020590020204D3230312058004D617869AC
:1004B0006D756D20416363656C65726174696F6E03
:1004C00020286D6D2F7332293A00204500205A00F4
:1004D00020590020204D3230332058004D6178697A
:1004E0006D756D2066656564726174657320286D35
:1004F0006D2F73293A00204500205A002059002012
:10050000204D393220580053746570732070657225
:1005100020756E69743A006563686F3A00457272BF
:100520006F723A0053544F505045442E2000507281
:10053000696E7465722073746F7070656420647581
:100540006520746F206572726F72732E2046697811
:1005500020746865206572726F7220616E64207508
:100560007365204D39393920746F20726573746159
:1005700072742E202854656D706572617475726591
:100580002069732072657365742E20536574206929
:100590007420616674657220726573746172746927
:1005A0006E6729004B494C4C45442E20005072691F
:1005B0006E7465722068616C7465642E206B696C62
:1005C0006C28292063616C6C656421006F6B00529C
:1005D0006573656E643A20002200556E6B6E6F770E
:1005E0006E20636F6D6D616E643A20220043686116
:1005F0006E67652066696C616D656E74006C63641E
:1006000020636F6E74726173742076616C75653AE5
:1006100020007A5F6D696E3A2000795F6D696E3AED
:100620002000785F6D696E3A20005A3A00593A000E
:1006300020436F756E7420583A2000453A005A3AAC
:1006400000593A00583A004649524D574152455FC9
:100650004E414D453A4D61726C696E2056313B20DA
:10066000537072696E7465722F6772626C206D616F
:100670007368757020666F722067656E3620464914
:10068000524D574152455F55524C3A687474703A16
:100690002F2F7777772E6D656E64656C2D70617284
:1006A00074732E636F6D2050524F544F434F4C5F05
:1006B00056455253494F4E3A312E30204D41434812
:1006C000494E455F545950453A7777772E63787392
:1006D0007733642E636F6D2045585452554445520C
:1006E0005F434F554E543A3120555549443A3030C6
:1006F0003030303030302D303030302D3030303000
:100700002D303030302D30303030303030303030EF
:1007100030300A007777772E6378737733642E63EF
:100720006F6D209BFF2E0042656420646F6E652E06
:100730000020423A0020453A00543A0042656420C5
:1007400048656174696E672E0048656174696E67FB
:1007500020646F6E652E0020453A00543A004865CB
:100760006174696E672E2E2E002042403A002040B0
:100770003A00202F003A00205400202F0020423A57
:1007800000202F006F6B20543A002569206D696EA0
:100790002C2025692073656300456E642066696CB2
:1007A00065206C69737400426567696E2066696CC8
:1007B00065206C697374004E6F206D6F76652E0036
:1007C0008A8BC7C884FFFFFFFF00576169742066EA
:1007D0006F7220757365722E2E2E00D4D584202E54
:1007E0002EFFFFFF00FFFFFF00006B4300006B4385
:1007F000000082430000A0400000A0400000803FB5
:1008000000000000000000000000000000000000E8
:10081000000000000000000000006B4300006B437C
:1008200000008243256920686F7572732025692056
:100830006D696E7574657300446F6E6520707269C2
:100840006E74696E672066696C650053544F505032
:1008500045442E20005072696E7465722073746F67
:10086000707065642064756520746F206572726FA6
:1008700072732E2046697820746865206572726FE5
:100880007220616E6420757365204D39393920748A
:100890006F20726573746172742E202854656D70B8
:1008A0006572617475726520697320726573657411
:1008B0002E205365742069742061667465722072FD
:1008C000657374617274696E6729006F6B004E6F97
:1008D000204C696E65204E756D6265722077697473
:1008E0006820636865636B73756D2C204C6173744D
:1008F000204C696E653A20004E6F20436865636B3B
:1009000073756D2077697468206C696E65206E75EB
:100910006D6265722C204C617374204C696E653A6F
:100920002000636865636B73756D206D69736D611D
:100930007463682C204C617374204C696E653A2096
:10094000004C696E65204E756D626572206973207A
:100950006E6F74204C617374204C696E65204E7507
:100960006D6265722B312C204C617374204C696E62
:10097000653A20004D31313000446F6E652073615F
:1009800076696E672066696C652E006F6B004D326C
:1009900039002020506C616E6E6572427566666526
:1009A0007242797465733A20002046726565204D65
:1009B000656D6F72793A20004D61722032382032B5
:1009C00030313800436F6D70696C65643A200028DF
:1009D000456E646572332900207C20417574686F10
:1009E000723A20004D617220323820323031382086
:1009F00030393A31363A353000204C617374205525
:100A00007064617465643A2000312E302E30004DE0
:100A100061726C696E200020536F66747761726535
:100A200020526573657400205761746368646F6752
:100A3000205265736574002042726F776E206F7567
:100A400074205265736574002045787465726E6118
:100A50006C20526573657400506F77657255700035
:100A600073746172740062696E004D3131372049D0
:100A70004E56414C494420444154412E004D3131A1
:100A800037205072696E74696E672E2E2E004730C3
:100A9000205A2573004732382058302059300047FB
:100AA00030205A257300473932205A2573204525B6
:100AB000730062696E002200656E717565696E670C
:100AC0002022007C3C3E5E2B3D3F2F5B5D3B2C2A71
:100AD000225C0045313A200045303A20005A3A2045
:100AE00000593A2000583A20004D53312C4D5332D2
:100AF0002050696E730A0024F404D9201BC40C5CD6
:100B00000E9804C4095F0265077101F405F900FB42
:100B100004B30048048700C103690058035500036B
:100B2000034500BE023A008402310053022A002924
:100B300002250004022000E4011C00C8011900AFD6
:100B40000117009801140084011300710110006165
:100B500001100051010E0043010D0036010B002B66
:100B6000010B0020010B00150109000C0109000315
:100B7000010800FB000800F3000800EB000700E498
:100B8000000600DE000600D8000600D2000600CCF9
:100B9000000500C7000500C2000500BD000400B943
:100BA000000400B5000400B1000400AD000400A979
:100BB000000400A5000300A20003009F0004009BA6
:100BC00000030098000300950002009300030090CA
:100BD0000003008D0002008B0003008800020086E5
:100BE00000020084000300810002007F0002007DFB
:100BF0000002007B0002007900020077000100760D
:100C00000002007400020072000100710002006F17
:100C10000002006D0001006C0002006A0001006922
:100C20000002006700010066000100650001006429
:100C30000002006200010061000100600001005F2D
:100C40000002005D0001005C0001005B0001005A31
:100C50000001005900010058000100570001005632
:100C60000001005500010054000100530000005332
:100C70000001005200010051000100500001004F2E
:100C80000001004E0000004E0001004D0001004C2C
:100C90000001004B0000004B0001004A0001004928
:100CA0000001004800000048000100470001004624
:100CB000000000460001004500000045000100441E
:100CC0000001004300000043000100420000004218
:100CD0000001004100000041000100400001003F10
:100CE0000000003F0001003E0000003E0001003D0A
:100CF0000000003D0001003C0000003C0000003C02
:100D00000001003B0000003B0001003A0000003AF7
:100D100000010039000000390001003800000038EF
:100D200000000038000100370000003700010036E5
:100D300000000036000000360001003500000035DC
:100D400000000035000100340000003400000034D1
:100D500000010033000000330000003300010032C6
:100D600000000032000000320001003100000031BC
:100D700000000031000100300000003000000030B1
:100D80000001002F0000002F0000002F0000002FA6
:100D90000001002E0000002E0000002E0001002D9A
:100DA0000000002D0000002D0000002D0001002C8F
:100DB0000000002C0000002C0000002C0001002B83
:100DC0000000002B0000002B0000002B0001002A77
:100DD0000000002A0000002A0000002A000100296B
:100DE000000000290000002900000029000000295F
:100DF0000001002800000028000000280000002852
:100E00000000002800010027000000270000002744
:100E10000000002700000027000100260000002637
:100E2000000000260000002600000026000100252A
:100E3000000000250000002500000025000000251E
:100E40000000002500010024000000240000002410
:100E50000000002400000024000100230000002303
:100E600000000023000000230000002300000023F6
:100E700000000023000100220000002200000022E8
:100E800000000022000000220000002200010021DA
:100E900000000021000000210000002100000021CE
:100EA00000000021000000210001002000000020BF
:100EB00000000020000000200000002000000020B2
:100EC00000000020000000200001001F0000001FA3
:100ED0000000001F0000001F0000001F0000001F96
:100EE0000000001F0001001E0000001E0000001E88
:100EF0000000001E00000024F4D43050C38E20C235
:100F0000A24017828B7011127A910D816CD90AA8B8
:100F100061E108C7586607615143061E4B5D05C174
:100F200045A7041A411104093D9803713931034062
:100F300036DB0265339102D4305402802E1D0263E9
:100F40002CEE01752AC501B028A001102781018F60
:100F50002564012B244B01E0223401AC211F018DBB
:100F6000200D01801FFC00841EED00971DDF00B8DE
:100F70001CD200E61BC600201BBC00641AB200B2E3
:100F800019A8000A19A0006A189900D11791004009
:100F9000178B00B516840031167E00B31579003A20
:100FA000157300C7146F0058146A00EE13660088AA
:100FB00013630025135E00C7125B006C1257001507
:100FC000125400C111510070114F0021114B00D675
:100FD0001049008D1047004610440002104200C026
:100FE0000F4000800F3E00420F3C00060F3B00CB3D
:100FF0000E3800930E37005C0E3500270E3400F3D8
:101000000D3200C10D3100900D3000600D2E003208
:101010000D2D00050D2C00D90C2B00AE0C290085E0
:101020000C29005C0C2700350C27000E0C2600E86C
:101030000B2400C40B2400A00B23007D0B23005ABB
:101040000B2100390B2100180B2000F80A1F00D9D2
:101050000A1E00BB0A1E009D0A1D00800A1D0063B7
:101060000A1C00470A1B002C0A1B00110A1A00F771
:10107000091A00DD091900C4091900AB0919009209
:101080000917007B091800630917004C0916003680
:10109000091600200916000A091500F5081500E0D8
:1010A000081400CC081400B8081400A40814009018
:1010B0000813007D0812006B081300580812004640
:1010C0000812003408110023081100120811000151
:1010D000081100F0071000E0071000D0071000C052
:1010E000071000B0070F00A107100091070E008342
:1010F000070F0074070F0065070E0057070E004921
:10110000070E003B070D002E070E0020070D0013F1
:10111000070D0006070D00F9060C00ED060D00E0B6
:10112000060C00D4060C00C8060C00BC060C00B06F
:10113000060C00A4060B0099060C008D060B00821D
:10114000060B0077060B006C060B0061060A0057C1
:10115000060B004C060A0042060A0038060A002E5A
:10116000060A0024060A001A060A001006090007EB
:10117000060A00FD050900F4050900EB050900E277
:10118000050900D9050900D0050900C7050900BEF9
:10119000050900B5050800AD050800A50509009C76
:1011A000050800940508008C050800840508007CEB
:1011B000050800740508006C050700650508005D5A
:1011C000050700560508004E0507004705070040C3
:1011D00005080038050700310507002A0507002328
:1011E0000507001C050600160507000F0507000887
:1011F00005060002050700FB040600F5040700EEE3
:10120000040600E8040600E2040700DB040600D53B
:10121000040600CF040600C9040600C3040600BD8E
:10122000040600B7040600B1040500AC040600A6DD
:10123000040600A00405009B040600950405009028
:101240000406008A04050085040500800406007A6F
:1012500004050075040500700405006B04050066B4
:10126000040500610405005C0405005704050052F4
:101270000405004D04050048040500430405003E34
:101280000404003A04050035040500300404002C71
:1012900004050027040400230405001E0404001AAA
:1012A00004040016040500110404000D04040009E0
:1012B0000405000404040000040400FC030400F816
:1012C000030400F4030400F0030400EC030400E84A
:1012D000030400E4030400E0030400DC030400D87A
:1012E000030400D4030400D0030400CC030400C8AA
:1012F000030300C50303006563686F3A00656E640D
:1013000073746F7073206869743A205A00205A3AD7
:1013100000656E6473746F7073206869743A205945
:101320000020593A00656E6473746F7073206869A9
:10133000743A20580020583A00656E6473746F70D8
:1013400073206869743A20004572726F723A0045E2
:1013500072723A204D415854454D50204245440048
:1013600054656D706572617475726520686561742D
:1013700065642062656420737769746368656420BE
:101380006F66662E204D415854454D502074726949
:10139000676765726564202121004572723A204DAD
:1013A000494E54454D50003A204578747275646535
:1013B00072207377697463686564206F66662E2097
:1013C0004D494E54454D502074726967676572658A
:1013D000642021004572723A204D415854454D50C9
:1013E000003A204578747275646572207377697469
:1013F00063686564206F66662E204D415854454DE4
:101400005020747269676765726564202100202D21
:1014100020496E76616C69642065787472756465C4
:1014200072206E756D62657220210070012C019032
:10143000012701B0012201C0011D01F001180110B6
:1014400002130130020E016002090190020401C082
:1014500002FF000003FA004003F5008003F000D013
:1014600003EB002004E6007004E100E004DC00402F
:1014700005D700C005D2004006CD00D006C80080C8
:1014800007C3003008BE00F008B900C009B400B0BE
:101490000AAF00B00BAA00D00CA500000EA00050AF
:1014A0000F9B00C01096005012910000148C00C0D9
:1014B000158700B0178200B0197D00D01B7800009E
:1014C0001E730040206E0090226900F024640040EA
:1014D000275F0090295A00E02B5500102E50002065
:1014E000304B0010324600E033410090353C001094
:1014F00037370070383200A0392D00B03A2800A0EC
:101500003B2300603C1E00103D1900903D1400106C
:101510003E0F00703E0A00C03E0500003F00005034
:101520004944204175746F74756E652066696E69F3
:1015300073686564212050757420746865204B7051
:101540002C204B6920616E64204B6420636F6E73A6
:1015500074616E747320696E746F20436F6E666978
:101560006775726174696F6E2E680050494420413E
:1015700075746F74756E65206661696C6564212091
:1015800074696D656F75740020403A006F6B20546C
:101590003A006F6B20423A00504944204175746F05
:1015A00074756E65206661696C6564212054656D93
:1015B000706572617475726520746F6F20686967F9
:1015C0006800204B643A2000204B693A2000204BF1
:1015D000703A200020436C617369632050494420B5
:1015E000002054753A2000204B753A2000206D6190
:1015F000783A2000206D696E3A200020643A20007D
:1016000020626961733A20000000000000000000C1
:1016100000000000003FFFF000000000000000009C
:101620000000000000380070000000000000000012
:1016300000000000003387300000000000000000C0
:10164000000000000027879000000000000000005C
:1016500000000000002F87D0000000000000000004
:1016600000000000002F87D00000000000000000F4
:1016700000000000002F03D0F80180000C1FE000E4
:10168000000820800020301048008000123FF00049
:10169000000410400020781043C38CD0023FF000BB
:1016A000000410400020781071249267CC3FF000B5
:1016B000000820800020301041249E40021FE000DE
:1016C00000104100002F03D049249040121FE00079
:1016D00000208200002F87D0FBB3CEE00C3FF0004B
:1016E00000208200002F87D000000000003FF000A3
:1016F000001041000027879000000000003FF0002C
:10170000000820800033873000000000000FC00078
:10171000000000000038007000000000000780009A
:1017200000FFFFC0003FFFF00000000000030000CA
:1017300000FFFFC0000000000000000000000000EB
:1017400000000000003FFFF000000000000000006B
:1017500000000000003800700000000000000000E1
:10176000000000000030FC3000000000000000001D
:10177000000000000020FC1000000000000000003D
:1017800000000000002078100000000000000000B1
:1017900000000000002030100000000000000000E9
:1017A00000000000002C00D0F80180000C1FE000B9
:1017B00000104100002E31D048008000123FF000A0
:1017C00000082080002F7BD043C38CD0023FF00064
:1017D00000082080002F7BD071249267CC3FF0005E
:1017E00000104100002E31D041249E40021FE00035
:1017F00000208200002C00D049249040121FE000FD
:101800000041040000203010FBB3CEE00C3FF0009C
:10181000004104000020781000000000003FF000AC
:10182000002082000020FC1000000000003FF000BB
:10183000001041000030FC3000000000000FC0002C
:101840000000000000380070000000000007800069
:1018500000FFFFC0003FFFF0000000000003000099
:1018600000FFFFC0000000005900B02000B02000C1
:10187000B02000B020002D2D3A2D2D004D3231002A
:10188000496E69742E2053442D4361726400C08CEC
:101890008D8EFFFFFFFF004D3231004368616E67A0
:1018A000652053442D4361726400D38C8D8EFFFFFD
:1018B000FFFF00CFD28A8B00D0D18A8BFFFFFFFFC2
:1018C00000CECF8A8BFFFFFFFF00B5B6FFFF008879
:1018D00089FFFF00CCCDFFFF00BCBDBEBFFFFFFFF7
:1018E000FF00F92E2E00F8CACBFFFF00949596005A
:1018F0004D3234004D3233202573004D383420589A
:101900002059205A2045004732382058302059307D
:10191000004D3130362053323535004D31303920CD
:10192000532569004D31393020532569004732383D
:1019300020583020593000C7C893C9A3A4FFFFFF27
:10194000FF00A8B0FFFF0094959600B3B4AFB0FFBE
:10195000FFFFFF00B3B4AFB0FFFFFFFF00A6B2FF71
:10196000FF00A6B2FFFF00AB93B1FFFFFF00AB93F8
:10197000B1FFFFFF00B5B6FFFF00AD98AEFFFFFF60
:1019800000A7A8FFFF00A5A62041425300A5A6205E
:10199000504C4100473238009798A0A1A2004D3822
:1019A00034009B9C9D9E9F9800949596004D6F7669
:1019B0006520302E316D6D004D6F766520316D6D77
:1019C000004D6F76652031306D6D008889FFFF0016
:1019D0004578747275646572004D6F7665205A00A3
:1019E0004D6F76652059004D6F7665205800AD9893
:1019F000AEFFFFFF004578747275646572005A008F
:101A0000590058004D363030004368616E676520DC
:101A100066696C616D656E7400466C6F7700466C2C
:101A20006F7700B3B4AFB0FFFFFFFF00B3B4AFB048
:101A3000FFFFFFFF00A6B2FFFF00A6B2FFFF00AB53
:101A400093B1FFFFFF00AB93B1FFFFFF00AFB0FF0B
:101A5000FF00AFB0FFFF00949596004E6F005965F0
:101A60007300D0D18A8BFFFFFFFF3F00FFFFFFFF16
:101A7000FFFFFFFFFFFFFFFFFFFFFFFFFFFFFFFF76
:101A8000FFFFFFFFFFFFFFFFFFFFFFFFFFFFFFFF66
:101A9000FFFFFFFFFFFFFFFFFFFFFFFFFFFFFFFF56
:101AA000FFFFFFEFFFFFFFFFFFFFFFFFFFFFFFFF56
:101AB000FFFFFFEFEFFFFFFFFFFFFFFFFFFFFFFF56
:101AC000FFFFFFE7DFFFFFFFFFFFFFFFFFFFFFFF5E
:101AD000FFFFFFE7DFFFFFFFFFFFFFFFFFFFFFFF4E
:101AE000FFFFFFE3DFFFFFFFFFFFFFFFFFFFFFFF42
:101AF000FFFFFFF3CFFFFFFFFFFFFFFFFFFFFFFF32
:101B0000FFFFE1E1CFFFFFFFFFFFFFFFFFFFFFFF51
:101B1000FE78000003DDFFFFFFFFFFFFFFFFFFFE7A
:101B2000FF807E0001EEFFFFFFFFFFFFFFFFFFFED4
:101B30007DCFFC0000F77FFFFFFFFFFFFFFFFFFFF0
:101B40008E060000007BBFFFFFFFFFFFFFFFFFFFD0
:101B5000C0000000007DDFFFFFFFFFFFFFFFFFFF72
:101B6000FC01FE00003EE7FFFFFFFFFFFFFFFFFF5E
:101B7000FFFFFC00031F73FFFFFFFFFFFFFFFFFFDF
:101B8000FFFFF800018F81FFFFFFFFFFFFFFFFFF57
:101B9000FFFFE0000083F9FFFFFFFFFFFFFFFFFFF4
:101BA000FFFF00FC0000F0FFFFFFFFFFFFFFFFFF54
:101BB000FFE00FFFC00000FFFFFFFFFFFFFFFFFF81
:101BC000FE03FFFFC00000FFFFFFFFFFFFFFFFFF5F
:101BD000FFFFFFF9000000FFFFFFFFFFFFFFFFFF18
:101BE000FFFFFFFC0007C0FFFFFFFFFFFFFFFFFF3E
:101BF000FFFFFFFF0007E0FFFFFFFFFFFFFFFFFF0B
:101C0000FFFFFFFFE007F1FFFFFFFFFFFFFFFFFF09
:101C1000FFFFFFFFFC07F9FFFFFFFFFFFFFFFFFFD5
:101C2000FFFFFFFFFF03F9FFFFFFFFFFFFFFFFFFC6
:101C3000FFFFFFFFFF83F9FFFFFFFFFFFFFFFFFF36
:101C4000FFFFFFFFFFC3FFFFFFFFFFFFFFFFFFFFE0
:101C5000FFFFFFFFFFE1FFFFFFFFFFFFFFFFFFFFB2
:101C6000FFFFFFFFFFF0BFFFFFFFFFFFFFFFFFFFD3
:101C7000FFFFFFFFFBF83FFFFFFFFFFFFFFFFFFF3F
:101C8000FFFFFFFFF9F83FFFFFFFFFFFFFFFFFFF31
:101C9000FFFFFFFF7EF0FFFFFFFFFFFFFFFFFFFFE4
:101CA000FFFFFFFF8E03FFFFFFFFFFFFFFFFFFFFB1
:101CB000FFFFFFFFE01FFFFFFFFFFFFFFFFFFFFF33
:101CC000FFFFFFFFFFFFFFFFFFFFFFFFFFFFFFFF24
:101CD000FFFFFFFFFFFFFFFFFFFFFFFFFFFFFFFF14
:101CE000FFFFFFFFFFFF7FFFFFFFFFFFFFFFFFFF84
:101CF00000007FFFFFF87FFFFFFFFFFFFFFFFFFFF9
:101D000080007FFFFFE07FFFFFFFFFFFFFFFFFFF80
:101D1000C3FCFFFFFFF8FFFFFFFFFFFFFFFFFFFF19
:101D2000C3FCFFFFFFF8FFFFFFFFFFFFFFFFFFFF09
:101D300087FDFFFFFFF1FFFFFFFFFFFFFFFFFFFF3B
:101D400087FFFFFFFFF1FFFFFFFFFFFFFFFFFFFF29
:101D50000FE7F30FFC23FC3FFFFFFFFFFFFFFFFF39
:101D60000FEF8007F003F01E007FFFFFFFFFFFFE75
:101D70001FCF8187C787C70C007FFFFFFFFFFFFED4
:101D8000001FC7C78FC79F0F0CFFFFFFFFFFFFFE9E
:101D9000001F878F1F8F1F0F1FFFFFFFFFFFFFFC1D
:101DA0003F9F8F8F1F8E001E3FFFFFFFFFFFFFFC37
:101DB0007F3F0F1E3F1E3FFE3FFFFFFFFFFFFFF86D
:101DC0007FFF1F1C3F1C7FFC7FFFFFFFFFFFFFF813
:101DD000FFFF1E1C7E1C7FFC7FFFFFFFFFFFFFF04D
:101DE000FFCE3E3C7E3C7FB8FFFFFFFFFFFFFFF0D2
:101DF000FF9E3C387C387E78FFFFFFFFFFFFFFE14E
:101E0000FF3C7C787C783CF1FFFFFFFFFFFFFFE1A8
:101E1000F8387878101801F1FFFFFFFFFFFFFF008F
:101E20000060203C007C07807FFFFFFFFFFFFFFF7B
:101E3000FFFFFFFE1FFE1FFFFFFFFFFFFFFFFFFF74
:101E4000FFFFFFFFFFFFFFFFFFFFFFFFFFFFFFFFA2
:101E5000FFFFFFFFFFFFFFFFFFFFFFFFFFFFFFFF92
:101E6000FFFFFFFFFFFFFFFFFFFFFFFF000609006F
:101E7000FE06018902FE20FFFE07FE06FE000000AE
:101E800006000701060606020080808080008003AD
:101E90000303060103A0A0A00507070600FF50509A
:101EA000F850F850500509090600FE2070A8A070EF
:101EB00028A870200608080600FF40A848102048FF
:101EC00054080507070600FF60909060989068012D
:101ED00003030602038080800207070602FF40809A
:101EE00080808080400207070602FF80404040401B
:101EF00040800505050600008850F8508805050556
:101F00000600002020F820200204040602FEC04043
:101F10004080050101060002F8020202060200C02C
:101F2000C00406060601001010204080800406064A
:101F30000601006090909090600306060601004044
:101F4000C0404040E00406060601006090102040BA
:101F5000F0040606060100F020601010E0050606F9
:101F600006000010305090F810040606060100F03C
:101F700080E01010E00406060601006080E090900A
:101F800060040606060100F010102040400406061A
:101F900006010060906090906004060606010060F3
:101FA0009090701060020505060200C0C000C0C01D
:101FB0000207070602FEC0C000C0404080050505BC
:101FC0000600001860806018050303060001F80091
:101FD000F8050505060000C0300830C004070706F4
:101FE0000100609010604000400506060600007089
:101FF00090A8B08070050606060000205088F8887A
:1020000088050606060000F088F08888F0040606B9
:10201000060100609080809060040606060100E0E2
:1020200090909090E0040606060100F080E0808029
:10203000F0040606060100F080E0808080040606B9
:10204000060100609080B0906004060606010090D2
:1020500090F0909090030606060100E0404040405A
:10206000E005060606000038101010906004060611
:1020700006010090A0C0A090900406060601008012
:1020800080808080F005060606000088D8A8A88811
:102090008804060606010090D0B0909090050606D0
:1020A000060000708888888870040606060100E033
:1020B0009090E080800407070601FF609090D0B008
:1020C0006010040606060100E09090E0909004067F
:1020D000060601006090402090600506060600009C
:1020E000F820202020200406060601009090909001
:1020F0009060040606060100909090F0606005066E
:10210000060600008888A8A8D888050606060000EC
:102110008850202050880506060600008888502038
:102120002020040606060100F010204080F003067F
:1021300006060100E080808080E0040606060100BB
:10214000808040201010030606060100E0202020B9
:1021500020E0050303060003205088050101060066
:10216000FEF8020202060204804004040406010094
:10217000709090700406060601008080E09090E068
:102180000404040601007080807004060606010045
:1021900010107090907004040406010060B0C070CC
:1021A000040606060100205040E0404004060606F2
:1021B00001FE6090907010600406060601008080A9
:1021C000E09090900306060601004000C04040E009
:1021D0000308080601FE200060202020A04004061D
:1021E000060601008080A0C0A0900306060601003C
:1021F000C040404040E0050404060000D0A8A88884
:10220000040404060100E090909004040406010018
:10221000609090600406060601FEE09090E08080E9
:102220000406060601FE7090907010100404040667
:102230000100A0D0808004040406010070C030E0DA
:102240000406060601004040E04050200404040655
:10225000010090909070040404060100909060606A
:1022600005040406000088A8A85004040406010020
:10227000906060900406060601FE90909070906059
:10228000040404060100F02040F0030707060100E3
:10229000204040804040200107070602FF808080E8
:1022A0008080808003070706010080404020404076
:1022B0008004020206010350A0FFFFFFFFFFFFFFA3
:1022C000FFFFFFFFFFFFFFFFFFFFFFFFFFFFFFFF1E
:1022D000FFFFFFFFFFFFFFFFFFFF000000060007FB
:1022E0000106060602008000808080800406060643
:1022F00001FF2070A0A070200507070600FF3048EE
:1023000040F04040F8050505060000A8508850A898
:102310000506060600008850F820F8200107070689
:1023200002FF808080008080800407070601FF7024
:102330008060906010E0030101060105A006070718
:10234000060000788494A4948478030505060101AE
:1023500060A06000E00505050600002850A0502898
:10236000040303060100F01010040101060102F04D
:102370000607070600007884B4A4A4847804010149
:10238000060105F0040303060102609060050707DB
:102390000600FF2020F8202000F8030505060101B3
:1023A00040A02040E0030505060101C0204020C0F8
:1023B00002020206020440800405050601FF909017
:1023C000B0D08005060606000078E8E868282801F5
:1023D0000101060202800202020602FE408003059D
:1023E0000506010140C04040E0030505060101402B
:1023F000A04000E0050505060000A0502850A005FB
:1024000008080600FF40C0405070307810050808EA
:102410000600FF40C0405068081038050808060054
:10242000FFC0204030F0307810040707060100207C
:1024300000206080906005070706000040202050C3
:1024400070888805070706000010202050708888D3
:1024500005070706000020502050708888050707F0
:1024600006000028502050708888050707060000E5
:102470005000205070888805070706000020502073
:102480005070888805060606000078A0F0A0A0B865
:102490000408080601FE60908080906020400407D8
:1024A000070601004020F080E080F00407070601E5
:1024B000002040F080E080F0040707060100205073
:1024C000F080E080F00407070601005000F080E093
:1024D00080F00307070601008040E0404040E00331
:1024E00007070601002040E0404040E003070706E0
:1024F000010040A0E0404040E0030707060100A0C3
:1025000000E0404040E00506060600007048E8484C
:10251000487004070706010050A090D0B0909004C6
:1025200007070601004020609090906004070706AE
:102530000100204060909090600407070601002091
:1025400050609090906004070706010050A06090D2
:102550009090600407070601005000609090906022
:10256000050505060000885020508804080806016B
:10257000FF1070B0B0D0D0E0800407070601004023
:1025800020909090906004070706010020409090F2
:102590009090600407070601002050909090906092
:1025A000040707060100500090909090600507070F
:1025B0000600001020885020202004060606010096
:1025C00080E09090E0800406060601006090A0A0E4
:1025D00090A004070706010040200070909070044E
:1025E000070706010020400070909070040707065E
:1025F0000100205000709090700407070601005001
:10260000A0007090907004060606010050007090C3
:10261000907004070706010020502070909070050C
:10262000040406000070A8B0780406060601FE70D7
:10263000808070204004070706010040200060B041
:10264000C07004070706010020400060B0C070049D
:10265000070706010020500060B0C070040606069F
:102660000100500060B0C070030707060100804001
:1026700000C04040E0030707060100204000C040C2
:1026800040E003070706010040A000C04040E0030F
:102690000606060100A000C04040E004070706014E
:1026A000003060107090906004070706010050A091
:1026B00000E0909090040707060100402000609021
:1026C00090600407070601002040006090906004BD
:1026D000070706010020500060909060040707067D
:1026E000010050A0006090906004060606010050B2
:1026F00000609090600505050600002000F80020AD
:1027000004040406010070B0D0E0040707060100CD
:1027100040200090909070040707060100204000C0
:102720009090907004070706010020500090909050
:10273000700406060601005000909090700409098C
:102740000601FE20400090909070906004080806FA
:1027500001FE8080E09090E080800408080601FE81
:10276000500090909070906000060900FE0701995B
:10277000032B20FFFE08FE07FE00000006000001FC
:102780000707060200808080808000800303030624
:102790000104A0A0A00507070600005050F850F85B
:1027A00050500507070600002070A0702870200513
:1027B000070706000048A8502050A8900507070604
:1027C000000040A0A040A890680103030602048016
:1027D000808003070706010020408080804020039E
:1027E00007070601008040202020408005050506DF
:1027F00000018850F850880505050600012020F8E2
:1028000020200303030601FF60408005010106004C
:1028100003F80303030601FF40E040050707060035
:10282000000808102040808005070706000020509F
:1028300088888850200507070600002060A0202017
:1028400020F8050707060000708808304080F8056A
:102850000707060000F8081030088870050707060B
:10286000000010305090F81010050707060000F81F
:1028700080B0C8088870050707060000304080B0A7
:10288000C88870050707060000F8081010204040AF
:10289000050707060000708888708888700507079C
:1028A000060000708898680810600307070601FF9B
:1028B00040E0400040E0400307070601FF40E040E1
:1028C000006040800407070601001020408040207F
:1028D00010050303060002F800F8040707060100CC
:1028E00080402010204080050707060000708810F7
:1028F00020200020050707060000708898A8B080F7
:102900007005070706000020508888F888880507AA
:1029100007060000F04848704848F0050707060021
:102920000070888080808870050707060000F048E6
:1029300048484848F0050707060000F88080F08006
:1029400080F8050707060000F88080F08080800589
:1029500007070600007088808098887005070706C2
:102960000000888888F8888888030707060100E047
:102970004040404040E005070706000038101010B6
:102980001090600507070600008890A0C0A09088FE
:10299000050707060000808080808080F805070713
:1029A0000600008888D8A8888888050707060000E0
:1029B0008888C8A898888805070706000070888856
:1029C00088888870050707060000F08888F08080F6
:1029D000800508080600FF7088888888A8700805A8
:1029E0000707060000F08888F0A090880507070612
:1029F000000070888070088870050707060000F8DE
:102A000020202020202005070706000088888888CD
:102A10008888700507070600008888885050502075
:102A2000050707060000888888A8A8D88805070732
:102A30000600008888502050888805070706000097
:102A400088885020202020050707060000F808107D
:102A5000204080F8030707060100E0808080808026
:102A6000E0050707060000808040201008080307E3
:102A700007060100E02020202020E00503030600D7
:102A8000042050880501010600FFF8020202060238
:102A9000068040050505060000700878887805075F
:102AA000070600008080B0C888C8B005050506008C
:102AB000007088808870050707060000080868987D
:102AC0008898680505050600007088F8807005077D
:102AD00007060000304840F0404040050707060068
:102AE000FE788888780888700507070600008080CF
:102AF000B0C88888880307070601004000C040402E
:102B000040E00409090601FE1000301010109090FA
:102B10006005070706000080808890E09088030722
:102B200007060100C04040404040E00505050600A2
:102B300000D0A8A8A888050505060000B0C88888A8
:102B40008805050506000070888888700507070657
:102B500000FEB0C888C8B080800507070600FE6880
:102B6000988898680808050505060000B0C88080A8
:102B70008005050506000070807008F0050707064F
:102B800000004040F0404048300505050600008840
:102B9000888898680505050600008888505020053B
:102BA00005050600008888A8A85005050506000050
:102BB00088502050880507070600FE888898680816
:102BC0008870050505060000F8102040F804070786
:102BD000060100304020C0204030010707060200F7
:102BE00080808080808080040707060100C020402C
:102BF000304020C005030306000448A890000000F0
:102C000001000000000001000000000001000000C1
:102C100000000100000000000100000000000100B1
:102C200000000000010000000000010000000000A2
:102C30000100000000000100000000000100000091
:102C40000000010000000000010000000000010081
:102C50000000000001000000000001000000000072
:102C60000100000000000100000000000100000061
:102C70000000010000000000010000000000010051
:102C80000000000001000000000001000000000042
:102C90000100000000000100000000000100000031
:102CA0000000010000000000010000000000010021
:102CB0000000000001000000000001000000000012
:102CC0000100000000000600000107070602008066
:102CD0000080808080800507070600FF2078A0A084
:102CE000A07820050707060000304840E04048B0C3
:102CF0000505050600008870507088050808060064
:102D0000FF88885020F82020200107070602008055
:102D10008080008080800508080600FF7080E090B9
:102D200048380870030101060107A00507070600DF
:102D3000007088A8C8A88870040606060101709073
:102D4000B05000F006050506000024489048240411
:102D50000202060102F010040101060103F005075A
:102D6000070600007088E8C8C888700501010600E1
:102D700007F803030306010440A040050606060009
:102D8000002020F82020F8040505060103609020AB
:102D900040F0040505060103E0106010E0020202A5
:102DA00006020640800506060600FF888888C8B02F
:102DB0008005070706000078E8E868282828010150
:102DC00001060203800202020602FE40800305059E
:102DD00006010340C04040E0040606060101609081
:102DE000906000F006050506000090482448900613
:102DF00009090600FF40C04040E40C143C040609E9
:102E0000090600FF40C04040E81404081C050909F9
:102E10000600FFC0204020C81828780805070706CC
:102E200000002000202040887005080806000040AF
:102E300020708888F888880508080600001020702F
:102E40008888F8888805080806000020507088885F
:102E5000F8888805080806000048B0708888F88857
:102E6000880508080600005000708888F8888805E2
:102E700008080600002050708888F8888806070730
:102E80000600003C50909CF0909C0509090600FE4D
:102E90007088808080887020400508080600004007
:102EA000F88080F08080F805080806000010F8809F
:102EB00080F08080F805080806000020F88080F087
:102EC0008080F805080806000050F88080F08080B7
:102ED000F80308080601008040E040404040E0035D
:102EE00008080601002040E040404040E003080898
:102EF00006010040A0E040404040E0030808060111
:102F000000A000E040404040E0050707060000F058
:102F10004848E84848F0050808060000285088C8D6
:102F2000A8988888050808060000402070888888CE
:102F3000887005080806000010207088888888704E
:102F400005080806000020507088888888700508E9
:102F500008060000285070888888887005080806D0
:102F600000005000708888888870050505060000FC
:102F70008850205088050707060000709898A8C858
:102F8000C870050808060000402088888888887076
:102F900005080806000010208888888888700508C1
:102FA00008060000205000888888887005080806F8
:102FB000000050008888888888700508080600008E
:102FC000102088885020202005070706000080F088
:102FD00088F0808080050707060000708890A09028
:102FE00088B005080806000040200070087888783E
:102FF0000508080600001020007008788878050889
:103000000806000020500070087888780508080637
:10301000000028500070087888780507070600002F
:1030200050007008788878050808060000205020B5
:10303000700878887806050506000078147C907C76
:103040000507070600FE7088808870204005080884
:103050000600004020007088F8807005080806000F
:10306000001020007088F880700508080600002015
:1030700050007088F8807005070706000050007047
:1030800088F88070030808060100804000C04040B6
:1030900040E0030808060100408000C0404040E0D6
:1030A00003080806010040A000C0404040E0060AB6
:1030B0000A0600FEA4A800FC8480808084FC060A26
:1030C0000A0600FE549400FC8404040484FC0508F1
:1030D00008060000285000B0C8888888050808063F
:1030E00000004020007088888870040A0A0602FEEA
:1030F00030408090909090909090040A0A0600FED4
:10310000C0201090909090909090060707060001C4
:10311000448C8C8480403C06070706000188C4C4A8
:10312000840408F00505050600012000F8002005CC
:10313000080806000040F0C888889878100508083C
:10314000060000E0F88888888888F80505050600EC
:10315000012030F830200508080600002070F82013
:10316000202020E00509090600FF2070A8A8B888E3
:103170008850200509090600FFE080C0B0A8A830EB
:1031800028280509090600FFF8A88888888888A8E3
:10319000F8050A0A0600FE205050505088A8A8885A
:1031A00070000B0B00FF0901CF039E20FFFF0AFFF9
:1031B00009FF0000000600010109090602008080E5
:1031C00080808080000080050303060006D84890B8
:1031D0000609090600002828287C28FC50505005C4
:1031E00009090600002070A8A07028A87020060A0F
:1031F0000A0600FF48A8A8B050285454948805092E
:10320000090600002050505060A890906802030307
:10321000060206C04080030A0A0601FF20404080E3
:10322000808080404020030A0A0601FF8040402041
:1032300020202040408005070706000120A87020BC
:1032400070A820050707060001202020F820202074
:10325000020303060200C04080050101060004F8D5
:103260000102020602008080050A0A0600FF080823
:1032700010102020404080800509090600002050E1
:103280008888888888502003090906010040C040CA
:103290004040404040E00509090600007088880869
:1032A00010204088F80509090600007088080830D9
:1032B0000808887005090906000010303050509049
:1032C000F8103805090906000078404040700808E9
:1032D000887005090906000070888080F088888859
:1032E00070050909060000F8880810102020202029
:1032F000050909060000708888887088888870052C
:103300000909060000708888887808088870010715
:103310000706020180800000008080020707060285
:1033200000C0C00000C04080050A0A0600FF081067
:103330002040808040201008050303060002F800AA
:10334000F8050A0A0600FF804020100808102040F7
:1033500080050909060000708888102020200020C0
:10336000060A0A0600FF3048B4D4D4D4D4A8807822
:103370000509090600002020205050708888880523
:103380000909060000F0888888F0888888F0050917
:10339000090600003048888080808048300509098F
:1033A000060000E090888888888890E00509090672
:1033B0000000F8808080F0808080F8050909060010
:1033C00000F8808080F08080808005090906000078
:1033D00030488080809888483005090906000088B8
:1033E000888888F888888888030909060100E040F1
:1033F000404040404040E0050909060000381010F8
:10340000101010109060050909060000888890A02F
:10341000E090908888050909060000E0404040409F
:10342000404048F80509090600008888D8D8A8A8AF
:10343000A8888805090906000088C8C8A8A8A8980F
:103440009888050909060000708888888888888817
:1034500070050909060000F048484870404040E007
:103460000509090600007088888888E898700805B2
:103470000909060000F0888888F0A090888805096E
:10348000090600007088888070088888700509091E
:10349000060000F8A8202020202020700509090639
:1034A000000088888888888888887005090906004F
:1034B0000088888850505020202005090906000007
:1034C000A8A8A8A8F850505050050909060000887F
:1034D00088505020505088880509090600008888C7
:1034E00050502020202020050909060000F88810EF
:1034F0001020204088F8030A0A0602FFE08080803E
:103500008080808080E0050A0A0600FF80804040BD
:10351000202010100808030A0A0601FFE0202020DE
:103520002020202020E00503030600062050880507
:1035300001010600FFF8030303060106C040200551
:103540000606060000E01070909068050909060064
:1035500000808080F0888888C8B0050606060000D4
:1035600070888080887005090906000008080878BE
:1035700088888898680506060600007088F88088A4
:1035800070050909060000304840F040404040E026
:103590000507070600FF689090609088700509098C
:1035A000060000808080B0C88888888803090906E2
:1035B0000100400000C040404040E0040A0A06000C
:1035C000FF1000003010101010906005090906006F
:1035D0000080808890A0C0A090880309090601009F
:1035E000C040404040404040E0050606060000D094
:1035F000A8A8A8A8A8050606060000B0484848489C
:103600004805060606000070888888887005070748
:103610000600FFF08888F08080800507070600FF1D
:1036200078888888780808050606060000D0684073
:103630004040E005060606000070886010887005AE
:1036400008080600004040F04040404830050606AB
:1036500006000088888888986805060606000088A5
:103660008850502020050606060000A8A8A8505043
:1036700050050606060000885020205088040707E1
:103680000601FF909050502020C00506060600005D
:10369000F888102048F8030A0A0601FF204040403D
:1036A000408040404020010B0B0602FF808080805C
:1036B00080808080808080030A0A0601FF8040406D
:1036C0004040204040408004020206010450A00A0D
:1036D0000A140B00FF30404840854079404940497A
:1036E000405940404044403DC00A0A140B00FF04CA
:1036F00000FFC090401F0031004E001100FFC021AC
:10370000003F00090A140B01FF0800FF80A0801889
:103710000048002800FF8008003600C1800B0A1412
:103720000B00FF71006300A4C0AF80F0001240598D
:1037300080948011002FE0090A140B01FF0800FF9C
:103740008080807F0022007D0008007F000800FF4D
:1037500080090A140B01FF08000800FF8088808898
:1037600080FF8088800800080008000A0A140B0007
:10377000FF08000400FFC0110011000A0004000A45
:103780000031C0C080090A140B01FF0800FF800847
:103790000008007F002200140008003600C1800AE3
:1037A0000A140B00FF210027C0F1002FC030806FEA
:1037B000C0A8802480208063800A0A140B00FF4583
:1037C000002FC0090019002FC02900CFC0490049AF
:1037D000004FC0090A140B01FF3F0052008C003259
:1037E00000C1807F0049007F0049007F000A0A1461
:1037F0000B00FF27C02100F90021003900E1002162
:10380000002900E70042000A0A140B00FF7BC042B7
:103810004042407A4042404A405240E2C0420002A8
:1038200000090A140B01FF1000FF8010002F8061B7
:1038300000A2003F80220022002E000A0A140B0082
:10384000FF610057C04140F7C0510053C056405B74
:10385000C0524043C0090A140B01FF080008000FC2
:10386000000800FF8008000C000A00090008000999
:103870000A140B01FFFF000100010041007F00401E
:10388000004000408040803F800A0A140B00FF2166
:10389000C026007FC022002EC0EA402EC02A402F42
:1038A000C06840090A140B01FF3000080008000836
:1038B000000800080014002200410080800A0A1459
:1038C0000B01FF45004400FF8048006900CD005611
:1038D0000052004500C8C0090A140B01FF08004946
:1038E00000490049007F000800888088808880FFA8
:1038F00080090A140B01FF10000900FF800800086E
:10390000007F00080008000900FF800A0A140B006D
:10391000FFFFC0120003807C00250024407FC016FA
:103920000025804440090A140B01FF220014007F87
:103930000049007F0049007F000800FF8008000761
:103940000A0A0B02FF3020FE82FE82FE82FE820AFD
:103950000A140B00FF7200020007C0FA4022402246
:103960004042404A40FC400980090A140B01FFFF15
:1039700080220022002200FF80220022002200423A
:103980000082000A0A140B00FF21002200FC4057AD
:10399000C0500057C05440244057C09440090A14F6
:1039A0000B01FF220014007F0008000800FF8008C0
:1039B0000014002200C1800909120B01004F80A0F1
:1039C000808480BE808C809480A480C48081800AA2
:1039D0000A140B00FF040027802400FFC004001419
:1039E0000024804100060078000A0A140B00FF44FE
:1039F0008024800FC00480E4802FC0248028805061
:103A0000008FC00B0A140B00FF77C054005600A5AE
:103A100080748015803540D440140017E0090A14E2
:103A20000B01FFFF808080BE80A280A280BE80A2AA
:103A3000808080FF8080800A0A140B00FF7FC044D2
:103A4000005F8050805F8050805F805500A480CCF4
:103A500040090A140B01FF08000F8008007F004294
:103A60000042007E000000908012000A0A140B0140
:103A7000FF8F0049000900C1C05F004900460042B5
:103A8000004D0010C00A0A140B00FF04007FC04064
:103A9000403F80040024002780240054008FC00A87
:103AA0000A140B00FF77C0120027C09D4075402507
:103AB000402540260022402C000A0A140B00FF2259
:103AC00000FA0027803280E68023C06440128049DB
:103AD0004089400A0A140B00FFE7C0A480AB00C471
:103AE000C0A900AFC0A500EFC0810081000A0A1480
:103AF0000B00FF4F8028808F8058802F80C0005F90
:103B0000C0554055407FC00A0A140B00FF0800FF53
:103B1000808880FF808880FF8088800800084007B8
:103B2000C00A0A140B00FF5FC0310097C054403731
:103B3000C03440D7C0510055806B400A0A140B01B5
:103B4000FF42005F80EA0046004DC0D900490049AD
:103B500000490011000A0A140B00FF14005400571A
:103B6000C054805C8052807280D100128014400A60
:103B70000A140B00FF1A00E3C02440FA802700312A
:103B8000C06E40A28021002E000A0A140B00FF0123
:103B900000F10047C0A540FD4027C03540E5402763
:103BA000C024400A0A140B00FF82005FC002000F0D
:103BB00080EA802F8026002A8052408FC00A0A1493
:103BC0000B00FF04007FC049007FC049005F8049AF
:103BD0000046008900B0C0090A140B01FF2400143C
:103BE00000440024000400FF80080014002200C1EB
:103BF000800A0A140B00FF04007FC042007FC0420D
:103C0000004B0052805280A240A2400A0A140B00CE
:103C1000FF7F80408052804A80448044804A8052A6
:103C200080408080400909120B01FF7F807F804027
:103C3000007B806A8048808A80EC8019800A0A14A0
:103C40000B00FF22002FC0F840250028807040AFF5
:103C5000802200A2005FC00A0A140B00FF50407DC2
:103C60004091407F4011407D40554054405C4011A0
:103C7000C00A0A140B00FF3F8020803F802080FF95
:103C8000C048007BC04A40FD800A40090A140B016D
:103C9000FF08000800FF8008000800080014002248
:103CA00000410080800A0A140B00FF040004000495
:103CB00000150024804440844024001C00080009B2
:103CC0000A140B01FFFF8088808880FF808880882D
:103CD000809480A280FF8080800A0A140B01FFA2DA
:103CE000003400FBC0B4800480F300530071002254
:103CF00080CC000A0A140B00FF22003FC020006F96
:103D000080A0002F8020002F8028802F800A0A1496
:103D10000B00FF08003F8020803F8020803F8020F4
:103D2000803F8054809F40090A140B01FF7F0049A7
:103D3000007F0049007F0022005300928022004251
:103D4000000A0A140B00FFFFC008007F8052805E4B
:103D50008052805E8052807F804080090A140B016F
:103D6000FF7F0008000800FF8014001400140024E6
:103D700080448083800A0A140B00FF200023C0FACD
:103D8000402A402A402A402A402A404BC092400AFA
:103D90000B160B00FF20003FC020005F80948012B4
:103DA00080FFC024803FC0008003000A0A140B007B
:103DB000FF4F80200000001FC0E200248029C03E89
:103DC0004050008FC00A0A140B00FF2F8028802863
:103DD000806F80A2003FC0220027002A8032400965
:103DE0000A140B01FF22007F001100FF802A00D17E
:103DF000802400190002007C00090A140B01FF2333
:103E000000FA80FF804200FA80AB00F9002900F33D
:103E10008024000A0A140B00FF22002FC0B200A564
:103E200000A94035802500230024802840090A1479
:103E30000B01FF3F806100BF0021003F0010003FE9
:103E40000052008C0073800A0A140B00FF7FC040F0
:103E500000400040004000400040004000800080E2
:103E6000000A0A140B00FF7C4045407D4051407D14
:103E7000405540554054409C4090C00A0A140B00E5
:103E8000FF23C0FA005200FBC02280FA8022807219
:103E900080AC806080090A140B01FF5F8012801FD4
:103EA00080D2805780578075805780208001800A9B
:103EB0000A140B00FFFF0055C07D40588095407FDD
:103EC000C0040027802400FFC00B0A140B00FFFB76
:103ED000C052007BE02480F4803F0020803F80209F
:103EE000803F800A0A140B00FF22002FC0200067C9
:103EF00080A4802FC030402F8021002300090A14A5
:103F00000B01FF5200BA80B600DF809200D3001E82
:103F1000805A0092001F800A0B160B01FF42008F8F
:103F200080A200BFC0C8808600AA00DFC01400E7DE
:103F30008018000A0A140B00FF0400040004002487
:103F40000027802400240024002480FFC0090A14D4
:103F50000B01FF08000800FF8088808880FF8088B0
:103F6000808880FF8080800A0A140B00FF120012F4
:103F7000002FC06200A20027002A803240220022C7
:103F8000000A0A140B01FFEF80A880AF80EA80AA24
:103F900000EFC0AA00E900A8C00040FFFFFFFFFF3C
:103FA000FFFFFFFFFF060A0A0B0300201000007846
:103FB000888888887C0609090B0201200000708827
:103FC0008888887CFFFFFFFFFFFF050A0A0B0300BC
:103FD000403000007088F8808870050A0A0B0300E2
:103FE000102000007088F88088700509090B030113
:103FF0007008007088F8808870FF030A0A0B0400BC
:1040000080400000C040404040E0030A0A0B04002A
:1040100040800000C040404040E0FFFFFFFF050936
:10402000090B0300402000708888888870050A0A00
:104030000B030010200000708888888870FFFFFF45
:104040000807070B0101181800FF001818FF0609E0
:10405000090B0200201000CC4444444C340B0306EE
:104060000B00030080FFE000C0030B0B0B04FF40BC
:1040700040E040404040404040400609090B0200FB
:10408000440000CC4444444C34FFFFFF00002100B6
:10409000240027002A0000002200250028002B0011
:1040A0000000200023002600290002020202020272
:1040B00002020404040404040404030303030303CA
:1040C00003030101010101010101010204081020A3
:1040D00040800102040810204080010204081020E2
:1040E000408080402010080402010000000102000E
:1040F00000000000000004030706000000000000AC
:104100000000000000000000000002494E46494E39
:104110004954594E414ECDCCCC3D0AD7233C17B71C
:10412000D13877CC2B329595E6241FB14F0A000089
:1041300020410000C84200401C4620BCBE4CCA1BA7
:104140000E5AAEC59D7400407A10F35A00A0724E0C
:1041500018090010A5D4E80000E87648170000E42C
:104160000B54020000CA9A3B000000E1F505000074
:1041700080969800000040420F000000A0860100D9
:104180000000102700000000E803000000006400A9
:10419000000000000A000000000001000000000014
:1041A0002C76D888DC674F0823DFC1DFAE59E1B138
:1041B000B796E5E3E453C63AE651997696E8E6C247
:1041C0008426EB898C9B62ED407C6FFCEFBC9C9F4E
:1041D00040F2BAA56FA5F490055A2AF75C936B6C70
:1041E000F9676DC11BFCE0E40D47FEF520E6B50064
:1041F000D0ED902E0300943577050080841E0800D2
:1042000000204E0A000000C80C333333330F986E81
:1042100012831141EF8D2114893BE65516CFFEE63E
:10422000DB18D1844B381BF77C1D901DA4BBE42404
:10423000203284725E228100C9F124ECA1E53D2781
:10424000E43DC740E0C0F3C7C04011241FBECFEF1C
:10425000D0E4DEBFCDBF14E0A0E0B1E0EEE8F7EBC4
:1042600001E00BBF02C007900D92A838B107D9F743
:104270001BBE1BE1A8E8B4E001C01D92A531B10747
:10428000E1F712E4C8E4D2E404C02297FE010E94E0
:104290006CDBC034D107C9F70E9476D20C94BADB2C
:1042A0000C940000EF92FF920F931F93F22FF02EC9
:1042B00047FD02C0E4E001C0E4E1242F332727FDDD
:1042C000309537FF03C0309521953F4F4F2D512F2B
:1042D0000F2FEE2E0E94F5268F2D912F1F910F91FB
:1042E000FF90EF900895A0E0B0E0E9E7F1E20C94D0
:1042F0008BDBEC01A880B980CA80DB80A114B104FB
:10430000C104D10441F484E2A82E89EDB82E8BE5D6
:10431000C82E87E0D82EC601B5012DE133EF41E06C
:1043200050E00E944FDB27EA31E440E050E00E9479
:10433000E7DA7B018C01C601B5012DE133EF41E0E5
:1043400050E00E944FDBCA01B9012CEE34EF4FEF71
:104350005FEF0E94E7DA6E0D7F1D801F911F97FFB0
:1043600004C06150704080409048688379838A839C
:104370009B839B01AC015F77B901CA01CDB7DEB762
:10438000EAE00C94A7DB0E94732108958EE593E088
:104390000E947321089560935E0370935F0380937E
:1043A0006003909361030895A0E0B0E0EAEDF1E2CC
:1043B0000C9489DBEC015B016115710519F0FB01BF
:1043C00091838083F9908F2D90E00E9470DB892B80
:1043D000C9F7FDE2FF1621F4F990EE24E39405C03D
:1043E0002BE2F21609F4F990EE248E0101501040F0
:1043F000C8016BE071E443E050E00E946324892B24
:1044000001F58E010E5F1F4FC8016EE071E445E0BB
:1044100050E00E946324892B19F48E01095F1F4F1D
:10442000A114B10419F0F50111830083E0FC04C06C
:1044300070E090E080E814C070E090E080E86FEFFA
:1044400008C1C80163E171E443E050E00E946324C5
:10445000892B69F4A114B10429F470E090E080EC98
:104460006FE7F7C02296F501D183C083F6CF882489
:10447000992440E050E060E070E0EF2DE053EA3036
:10448000A0F5F2E0EF2A8E2D90E09C0128703070AC
:10449000E2FE06C0232B79F50894811C911C2BC0E9
:1044A000232B19F0089481089108DB01CA0112E05E
:1044B000880F991FAA1FBB1F1A95D1F7480F591FC4
:1044C0006A1F7B1F440F551F661F771F4E0F511D1C
:1044D000611D711D483929E9520729E9620729E15F
:1044E000720748F084E0E82A06C0EE3F31F4E3FCAE
:1044F00039C098E0E92AF990C0CFE53311F0E531F1
:1045000089F529912D3219F4E0E1EE2A05C02B320C
:1045100019F081E090E003C0299182E090E0E22F61
:10452000E053EA3018F0C81BD90B1CC020E030E083
:10453000FCE020383F075CF4C901880F991F880F01
:10454000991F280F391F220F331F2E0F311DE9919C
:10455000E053EA3068F3E4FE03C0309521953F4F05
:10456000820E931ECE2CDD24E1FE07C0A114B104FF
:1045700021F02197F501D183C083CB01BA010E94BC
:10458000D5D77B018C01F3E0CF22DD2423E0C216D6
:10459000D10421F417FB109517F910955701680104
:1045A000C801B70120E030E040E050E00E9435D77C
:1045B000882309F44AC097FE0DC02AE2E22E21E4C6
:1045C000F22E9094819491089394C0E2D0E000E0A0
:1045D00010E012C092E4E92E91E4F92EF6CFF70133
:1045E0002591359145915491C601B5010E9415DA86
:1045F0005B016C018C1A9D0A8C169D0684F7D5957B
:10460000C7950F5F1F4F0630110529F08CEF9FEF04
:10461000E80EF91EF1CFC501D6017C018D018C2D6C
:10462000880F8D2D881F8F3F51F0C601B50120E006
:1046300030E040E050E00E9435D7882331F482E238
:1046400090E09093141B8093131B7E2D9F2D802F41
:10465000612F272F392F482F562FB901CA01CDB707
:10466000DEB7ECE00C94A5DB2F923F925F926F9245
:104670007F928F929F92AF92BF92CF92DF92EF92F2
:10468000FF920F931F93CF93DF938C011B01EA01DD
:104690006115710519F0FB0191838083209749F022
:1046A000CE010297839728F020E030E040E050E010
:1046B000F6C0F801A1908F018A2D90E00E9470DB76
:1046C000892BB9F7FDE2AF1631F4F801A1908F0103
:1046D0005524539407C0FBE2AF1619F4F801A190DA
:1046E0008F015524209719F0C031D105C1F4F0E3B2
:1046F000AF1679F4F8018081883711F0883549F4D4
:10470000F801A1800E5F1F4FF2E05F2AC0E1D0E008
:1047100006C0209721F480E3A816E9F427C0C8302A
:10472000D10531F1C930D10524F4C230D10531F5BC
:104730000CC0CA30D10589F0C031D105F9F4C12CC3
:10474000D12CE12CB8E0FB2E28C0C12CD12CE12CBF
:10475000A0E4FA2E22C0CAE0D0E0FCECCF2EFCECA4
:10476000DF2EFCECEF2EFCE0FF2E17C0C8E0D0E0FF
:10477000C12CD12CE12CE0E1FE2E0FC09E0144277C
:1047800037FD4095542F60E070E080E090E80E9493
:104790002DDBC901DA016C017D0120E030E040E051
:1047A00050E060E03E01882477FC8094982C70ED06
:1047B000B72EBA0CE9E0EB1570F48A2D81548A31DA
:1047C00018F499ECB92E06C08A2D81568A3150F51D
:1047D00089EAB82EBA0C8B2D90E08C179D0714F542
:1047E0006F3FE1F0C216D306E406F506B0F0CA0149
:1047F000B901A40193010E94E7DA9B01AC012B0DE2
:10480000311D411D511D2130F0E03F07F0E04F0701
:10481000F0E85F0710F461E001C06FEFF801A190CC
:104820008F01C5CF2114310481F0662331F001508E
:104830001040F1011183008308C051FE1AC00250DC
:104840001040F1011183008314C067FF12C050FCB7
:1048500005C02FEF3FEF4FEF5FE704C020E030E0EF
:1048600040E050E882E290E09093141B8093131B89
:1048700016C050FE08C050954095309521953F4F89
:104880004F4F5F4F0CC057FF0AC082E290E09093F9
:10489000141B8093131B2FEF3FEF4FEF5FE7B9011E
:1048A000CA01DF91CF911F910F91FF90EF90DF90A0
:1048B000CF90BF90AF909F908F907F906F905F90C0
:1048C0003F902F900895FB01DC014150504088F04B
:1048D0008D9181341CF08B350CF4805E65916134D0
:1048E0001CF06B350CF4605E861B611171F3990B43
:1048F0000895881BFCCFFB01DC014150504048F07B
:1049000005900D920020C9F701C01D924150504002
:10491000E0F70895FB0155915523A9F0BF01DC0193
:104920004D9145174111E1F759F4CD010590002053
:1049300049F04D9140154111C9F3FB014111EFCFF1
:1049400081E090E001970895FB01DC0104C08D91A6
:104950000190801921F441505040C8F7881B990BF1
:104960000895FB01DC0102C001900D9241505040BE
:10497000D8F70895FB01DC010D900020E9F71197AD
:1049800001900D920020E1F70895FC0181918617B6
:1049900021F08823D9F7992708953197CF010895F9
:1049A000FB01DC0101900D920020E1F70895FB016D
:1049B000DC014150504030F08D910190801919F484
:1049C0000020B9F7881B990B0895FB01DC014150C9
:1049D000504048F001900D920020C9F701C01D928F
:1049E00041505040E0F70895AEE0B0E0EAEFF4E265
:1049F0000C9491DB0D891E898EE08C831A830983C8
:104A00008FEF9FE79E838D839E01275E3F4FCE01F0
:104A100001966F89788DA9010E9418252F8138850C
:104A2000020F131FF80110822E96E4E00C94ADDB08
:104A3000ABE0B0E0EEE1F5E20C9483DB3C012B014E
:104A40005A01FC0117821682838181FD03C06FEF3A
:104A50007FEFC6C19AE0892E1E010894211C311CEB
:104A6000F3012381F20123FD859123FF81912F0121
:104A7000882309F4B2C1853239F423FD859123FFDF
:104A800081912F01853229F490E0B3010E944529DC
:104A9000E7CF982FFF24EE249924FFE1FF15D0F0F3
:104AA0009B3269F09C3228F4903259F0933291F4A1
:104AB0000EC09D3249F0903369F441E024C052E0C9
:104AC000F52A84E0F82A28C098E0F92A25C0E0E118
:104AD000FE2A22C0F7FC29C0892F80538A3070F447
:104AE000F6FE05C0989C902C1124980E15C0E89CE9
:104AF000E02C1124E80EF0E2FF2A0EC09E3229F4C9
:104B0000F6FC6BC140E4F42A07C09C3619F450E867
:104B1000F52A02C0983649F4F20123FD959123FF4E
:104B200091912F01992309F0B8CF892F85548330B3
:104B300018F08052833038F444E050E0A40EB51EE3
:104B40005FE359830FC0933631F0933779F0933593
:104B500009F056C020C0F5018081898342E050E011
:104B6000A40EB51E610101E010E012C0F501C08085
:104B7000D180F6FC03C06FEF7FEF02C0692D70E0BB
:104B800042E050E0A40EB51EC6010E943A298C01F5
:104B90005FE7F52214C0F501C080D180F6FC03C0A8
:104BA0006FEF7FEF02C0692D70E042E050E0A40E8D
:104BB000B51EC6010E942F298C0150E8F52AF3FE8C
:104BC00007C01AC080E290E0B3010E944529EA9430
:104BD0008E2D90E008171907A8F30EC0F601F7FC18
:104BE0008591F7FE81916F0190E0B3010E94452904
:104BF000E110EA94015010400115110579F7EAC05F
:104C0000943611F0993669F5F7FE08C0F501208158
:104C100031814281538184E090E00AC0F5018081B6
:104C200091819C01442737FD4095542F82E090E00C
:104C3000A80EB91E9FE6F92257FF09C0509540956E
:104C4000309521953F4F4F4F5F4FE0E8FE2ACA0154
:104C5000B901A1012AE030E00E947129D82ED218B2
:104C600040C0953729F41F2D1F7E2AE030E01DC07B
:104C70001F2D197F9F3661F0903720F4983509F089
:104C8000ACC00FC0903739F0983709F0A6C004C007
:104C900028E030E00AC0106114FD146020E130E02B
:104CA00004C014FD166020E132E017FF08C0F501D2
:104CB000608171818281938144E050E008C0F501F8
:104CC00080819181BC0180E090E042E050E0A40E40
:104CD000B51EA1010E947129D82ED2188FE7F82E97
:104CE000F122F6FE0BC05EEFF522D91438F4F4FE83
:104CF00007C0F2FC05C08FEEF82202C01D2D01C0D6
:104D0000192DF4FE0DC0FE01ED0DF11D80818033E3
:104D100019F499EEF92208C01F5FF2FE05C003C026
:104D20008F2D867809F01F5F0F2DF3FC14C0F0FE65
:104D30000FC01E1510F09D2C0BC09D2C9E0C911ABF
:104D40001E2D06C080E290E0B3010E9445291F5F3E
:104D50001E15C0F304C01E1510F4E11A01C0EE24A4
:104D600004FF0FC080E390E0B3010E94452902FFD9
:104D70001DC001FD03C088E790E00EC088E590E00B
:104D80000BC0802F867891F001FF02C08BE201C03A
:104D900080E2F7FC8DE290E0B3010E94452906C055
:104DA00080E390E0B3010E9445299A94D914C0F39E
:104DB000DA94F101ED0DF11D808190E0B3010E94C4
:104DC0004529DD20A9F706C080E290E0B3010E94EA
:104DD0004529EA94EE20C1F743CEF301668177813D
:104DE000CB012B96E2E10C949FDBA9E0B0E0EBEF66
:104DF000F6E20C9487DB6A01122FA02EBE2C2BE367
:104E0000201718F42CE3922E02C0902E9394AE013A
:104E10004F5F5F4F27E0092D0E945728BC01898111
:104E2000E82EFF24C70189709070019711F4ADE25C
:104E300009C0B1FE02C0ABE205C0B0FC02C0A0E0F8
:104E400001C0A0E2E3FE3BC0AA2311F423E001C0AD
:104E500024E0211710F020E002C0121B212FEB2CC0
:104E6000B4FE02C0322F0AC0F601322F80E202C027
:104E7000819331503323E1F7C20ED11CAA2319F0DC
:104E8000F601A1936F01F6013196E2FE05C09EE4A2
:104E9000D6019C9381E404C09EE6D6019C9381E6F2
:104EA00011968C9391833296DF01832F90E202C09A
:104EB0009D9381508823E1F7E30FF11D40C0E2FE8E
:104EC00042C0AA2311F423E001C024E0211710F00E
:104ED00020E002C0121B212FEB2CB4FE02C0922F47
:104EE0000AC0F601922F80E202C08193915099236B
:104EF000E1F7C20ED11CAA2319F0F601A1936F01AC
:104F0000F6013196E2FE08C089E4D6018C938EE466
:104F100011968C9386E407C089E6D6018C938EE6C1
:104F200011968C9386E681833296DF01892F20E2E9
:104F300002C02D9381508823E1F7E90FF11D108203
:104F40002EEF3FEFAFC0161617061CF041E050E001
:104F500003C0AB014F5F5F4FAA2019F480E090E0DF
:104F600003C08A2D90E0019620E030E0AA2311F0E2
:104F700021E030E0240F351F280F391F812F90E0EA
:104F80002817390714F020E002C0121B212F4B2DE7
:104F900050E0CA0180719070B4FC0DC0B3FC0BC02E
:104FA000F601322F40E202C0419331503323E1F742
:104FB000C20ED11C01C0322FAA2319F0F601A19311
:104FC0006F01892B11F0132F0AC0F601132F80E314
:104FD00002C0819311501123E1F7C30ED11C092D9A
:104FE000060FBA8090E1892E912C8E209F20E4FE3E
:104FF00004C0F1E3BF1609F40150101614F001E0EB
:1050000003C0093008F008E09B0177FF02C020E0F0
:1050100030E0CB010196821B930BFE013196E80F25
:10502000F91F8EE2F82E3B01601A71088A2D90E07C
:1050300044275527481B590B8FEF2F3F380719F48A
:10504000D601FD926D01621773072CF0621673068C
:1050500014F4808101C080E3215030403196241740
:10506000350724F0D6018D936D01E6CF261737075B
:1050700049F4B5E3BB1528F0BB1621F48114910463
:1050800009F481E3F6018193D601812F90E202C0F9
:105090009C93815011968823D9F7E10FF11D10825E
:1050A00020E030E0C9012996EEE00C94A3DB283023
:1050B00008F027E03327DA01990F311D87FD916051
:1050C00000966105710539F432602E5F3D9330E33F
:1050D0002A95E1F708959F3F30F08038710561050A
:1050E00009F03C5F3C5F3D93913008F08068911D72
:1050F000DF93CF931F930F93FF92EF92192F987F17
:105100009695E92F96959695E90FFF27E056FE4B69
:1051100099273327EE24FF24A701E701059008947F
:10512000079428F4360FE71EF81E491F511D660F1D
:10513000771F881F991F0694A1F70590079428F4FC
:10514000E70EF81E491F561FC11D770F881F991FB4
:10515000661F0694A1F70590079428F4F80E491FDE
:10516000561FC71FD11D880F991F661F771F0694F2
:10517000A1F70590079420F4490F561FC71FD81FA9
:10518000990F661F771F881F0694A9F784911095C1
:10519000177041F0D695C79557954795F794E794C2
:1051A0001A95C1F7E6E4F1E46894159015913591EC
:1051B0006591959105907FE27395E118F10A430B93
:1051C000560BC90BD009C0F7E10CF11E431F561F47
:1051D000C91FD01D7EF4703311F48A95E6CFE89490
:1051E000015030F0080F0AF40027021708F4202FAE
:1051F0002395022F7A3328F079E37D932A95E9F7F6
:1052000010C07D932A9589F60694979567953795F2
:1052100017951794E118F10A430B560BC90BD009E7
:1052200098F023957E9173957A3308F070E37C9320
:105230002013B8F77E9170617D9330F0839571E310
:105240007D9370E32A95E1F71124EF90FF900F9181
:105250001F91CF91DF91992787FD90950895FC01CB
:105260000590615070400110D8F7809590958E0F91
:105270009F1F0895FC016150704001900110D8F704
:10528000809590958E0F9F1F08950F931F93CF9336
:10529000DF938C01EB018B8181FF1BC082FF0DC06E
:1052A0002E813F818C819D812817390764F4E88124
:1052B000F9810193F983E88306C0E885F985802F99
:1052C0000995892B31F48E819F8101969F838E836E
:1052D00002C00FEF1FEFC801DF91CF911F910F9117
:1052E0000895FA01AA27283051F1203181F1E8947C
:1052F0006F936E7F6E5F7F4F8F4F9F4FAF4FB1E0C9
:105300003ED0B4E03CD0670F781F891F9A1FA11DC3
:10531000680F791F8A1F911DA11D6A0F711D811DC4
:10532000911DA11D20D009F468943F912AE0269F89
:1053300011243019305D3193DEF6CF010895462FE8
:105340004770405D4193B3E00FD0C9F7F6CF462FC9
:105350004F70405D4A3318F0495D31FD4052419332
:1053600002D0A9F7EACFB4E0A695979587957795EF
:105370006795BA95C9F700976105710508959B0176
:10538000AC010A2E06945795479537952795BA95FF
:10539000C9F7620F731F841F951FA01D0895FC019C
:1053A000128213820895FC018381882311F081E029
:1053B00082830895FC018281811112820895CF9326
:1053C000DF93DC01FC01EB55FE4F8081918100975A
:1053D000C9F1019791838083ED01CC5ADF4FFD0124
:1053E000ED58FF4F8BE1019009928150E1F7FD01EB
:1053F000EE5AFF4FAF58BF4F8D919C911197A15717
:10540000B04091838083FD01ED58FF4F20E030E0F4
:10541000AD014B555E4F10C02F5F3F4FEF01DF01D5
:105420005F968BE10D9009928150E1F7858D968D05
:10543000329791838083B196DA018D919C912817E0
:10544000390750F3DF91CF910895FC0181E694E094
:10545000918380838781882321F0CF0104960E9465
:105460002F82089583519E4F0E942F820895CF92DC
:10547000DF92EF92FF920F931F93DF93CF93CDB7FD
:10548000DEB76F970FB6F894DEBF0FBECDBF8C01AD
:105490006B01095A1F4FD8018C9107551040882382
:1054A00021F42FE2E22EF12C03C090E5E92EF12C3D
:1054B000E00EF11E81E694E09A8389831C821B82B0
:1054C00018861D82B7016C5F7F4FCE010596A6013D
:1054D00021E00E943D89882391F5E3EEF0E094916C
:1054E00008C08091C00085FFFCCF9093C600319624
:1054F00094919923B1F7E9EEF0E0949108C080917E
:10550000C00085FFFCCF9093C600319694919923FB
:10551000B1F709C08091C00085FFFCCF0894C11C81
:10552000D11C9093C600F6019081992399F7809140
:10553000C00085FFFCCF8AE08093C6005AC0F80106
:10554000EB55FE4F208131812A30310508F040C0F3
:105550002F5F3F4F3183208321503040F90185E098
:10556000EE0FFF1F8A95E1F7E21BF30BED58FF4F9B
:10557000E00FF11F13C0AF01415E5F4FBF018BE130
:10558000DB010D90BD01DA010D92AD018150C1F733
:10559000929182913296968F858F7F9721503040DD
:1055A000BFEF2E3F3B0739F7D801AD58BF4FF7018A
:1055B00034968BE101900D928150E1F70F581F4F07
:1055C000F70182819381D8018D939C9301571040FC
:1055D000D801AC5ABF4FFE0135968BE101900D9278
:1055E0008150E1F70E5A1F4F8B819C81F801918306
:1055F0008083CE0101960E94252A6F960FB6F894FB
:10560000DEBF0FBECDBFCF91DF911F910F91FF90F5
:10561000EF90DF90CF9008959C01AB0183519E4F96
:105620002D5C3F4FB90121E00E943D8908950F9301
:105630001F93FC01162F072F242F8381882309F441
:1056400063C0E051FE4F8081E05FF140882309F0A4
:105650005BC0CF0183519E4FF396BF01412F502F66
:105660000E943D89882361F5E8EDF2E0949108C03D
:105670008091C00085FFFCCF9093C6003196949135
:105680009923B1F7812F902F9C01F90107C08091D8
:10569000C00085FFFCCF31969093C600908199237E
:1056A000B1F7E5EDF2E0949108C08091C00085FF6C
:1056B000FCCF9093C600319694919923B1F724C002
:1056C000E3ECF2E0949108C08091C00085FFFCCF2C
:1056D0009093C600319694919923B1F7812F902F22
:1056E0009C01F90107C08091C00085FFFCCF319675
:1056F0009093C60090819923B1F78091C00085FFF7
:10570000FCCF8AE08093C6001F910F910895EF921D
:10571000FF920F931F938C013EECE32E31E0F32EAA
:10572000E80EF91EC7010E94E181C7010E942F8285
:10573000F801108211821F910F91FF90EF90089550
:10574000CF92DF92EF92FF920F931F93CF93DF934D
:105750007C016B01DB010D900020E9F78D01015008
:105760001040061B170BEEECF1E0EE0EFF1ED7010A
:105770001C92E2E3FEEFEE0EFF1ECB016EE470E042
:105780000E94C524EC01009731F4F8013197EC0D2B
:10579000FD1D86010EC060E270E00E94C5248C01F0
:1057A0000F5F1F4FCE016AE270E00E94C524FC012A
:1057B00031978DE081838AE082831382C70186530B
:1057C0009E4FB8010E943F8A8EEC91E0E80EF91ED0
:1057D000D7018C91882319F1E3E1F1E0949108C09D
:1057E0008091C00085FFFCCF9093C60031969491C4
:1057F0009923B1F7EAE1F1E0949108C08091C000EB
:1058000085FFFCCF9093C600319694919923B1F710
:105810008091C00085FFFCCF8AE08093C600DF91B5
:10582000CF911F910F91FF90EF90DF90CF9008954F
:10583000CF93DF93EC018B81882309F43BC0E2E432
:10584000F1E0949108C08091C00085FFFCCF909357
:10585000C600319694919923B1F7CE55DD4F48811A
:1058600059816A817B81C25AD2408CE095E02AE05E
:1058700030E00E947F3EE0E4F1E0949108C0809126
:10588000C00085FFFCCF9093C60031969491992378
:10589000B1F7C656DD4F488159816A817B818CE022
:1058A00095E02AE030E00E947F3E8091C00085FFB5
:1058B000FCCF12C0E0E3F1E0949108C08091C000F9
:1058C00085FFFCCF9093C600319694919923B1F750
:1058D0008091C00085FFFCCF8AE08093C600DF91F5
:1058E000CF9108952F923F924F925F926F927F9245
:1058F0008F929F92AF92BF92CF92DF92EF92FF92E0
:105900000F931F93DF93CF93CDB7DEB7AC970FB64E
:10591000F894DEBF0FBECDBF5C014B01FC0183815B
:10592000882309F438C1C50182539E4F0E942F82FB
:10593000F50112821A8A1D8A198A188A81E694E072
:105940009F878E875EE4C52ED12CCA0CDB1C2FE20C
:1059500030E0A20EB31EF601B182A08221ED3FEF2E
:10596000A20EB31EF40180818F3209F090C0C401F1
:105970006FE270E00E94C5247C010894E11CF11CD8
:105980003E010894611C711C260142E1242E312C39
:105990002C0E3D1E77C0C7016FE270E00E94C52447
:1059A0006C01009709F481C0E816F90608F07DC083
:1059B0008C010E191F09C301B701A8010E94E5243B
:1059C000060D171DF8011082F30107C08091C00079
:1059D00085FFFCCF31969093C60090819923B1F753
:1059E0008091C00085FFFCCFFAE0F093C600F20181
:1059F000608171816115710519F460E070E002C089
:105A00006C5F7F4FC101A30121E00E943D89882383
:105A100071F5EEE7F1E0949108C08091C00085FF38
:105A2000FCCF9093C600319694919923B1F7FE0173
:105A3000319607C08091C00085FFFCCF31969093CE
:105A4000C60090819923B1F7ECE7F1E0949108C08A
:105A50008091C00085FFFCCF9093C6003196949151
:105A60009923B1F78091C00085FFFCCF8DC02EE057
:105A700030E02C0F3D1FF201318320837601089422
:105A8000E11CF11CE114F10409F085CF0BC080E5A5
:105A900090E0A80EB91EF601B182A08220EB3FEF84
:105AA000A20EB31ED82C092D02C0DE2C0F2D8EE4C1
:105AB00090E0A80EB91EF5018081918122EB3FEFA5
:105AC000A20EB31E009719F480E090E001C0049686
:105AD0006D2D702F0E940F8A882339F1EEE6F1E0D8
:105AE000949108C08091C00085FFFCCF9093C600C0
:105AF000319694919923B1F78D2D902F9C01F90146
:105B000007C08091C00085FFFCCF31969093C600FE
:105B100090819923B1F782EA92E0A80EB91EF501AF
:105B2000108211821282138232C0E6E5F1E0949174
:105B300008C08091C00085FFFCCF9093C6003196CD
:105B400094919923B1F78D2D902F9C01F90107C0F5
:105B50008091C00085FFFCCF31969093C600908164
:105B60009923B1F7E4E5F1E0949108C08091C00079
:105B700085FFFCCF9093C600319694919923B1F79D
:105B80008091C00085FFFCCF8AE08093C600CE01E3
:105B90000E960E94252AAC960FB6F894DEBF0FBE73
:105BA000CDBFCF91DF911F910F91FF90EF90DF90CC
:105BB000CF90BF90AF909F908F907F906F905F90AD
:105BC0004F903F902F900895C3966BE37AE00E9428
:105BD0000F8A882379F0E1EBF2E0949108C080917C
:105BE000C00085FFFCCF9093C60031969491992315
:105BF000B1F70EC0ECE9F2E0949108C08091C000CA
:105C000085FFFCCF9093C600319694919923B1F70C
:105C1000E9E9F2E0949108C08091C00085FFFCCFD3
:105C20009093C600319694919923B1F70895BF924D
:105C3000CF92DF92EF92FF920F931F93CF93DF9358
:105C40008C01EB018FE28993FF24EE24E39475EA43
:105C5000C72E71E0D72EC00ED11E6FE1B62E14C034
:105C6000FB9CC00111248D589F4F800F911FBE01D6
:105C70000E94418202C02196E3948881882319F012
:105C80008CE88E15C0F7F3942F2D30E0F60180815B
:105C900091812817390720F3E7FC07C0C801825318
:105CA0009E4FBE010E94418201C01882DF91CF91B8
:105CB0001F910F91FF90EF90DF90CF90BF900895CC
:105CC0002F923F924F925F926F927F928F929F920C
:105CD000AF92BF92CF92DF92EF92FF920F931F93FA
:105CE000DF93CF93CDB7DEB7AD970FB6F894DEBF95
:105CF0000FBECDBF6C014B014DA7DC0113968C91FB
:105D0000882309F44AC3E1EDF1E0CE0EDF1ED6018F
:105D10008C91EFE2FEEFCE0EDF1E882309F419C14D
:105D2000222309F0E1C028E032E0C20ED31ED601E2
:105D30008C91E8EFFDEFCE0EDF1E882371F1E3E1D9
:105D4000F1E0949108C08091C00085FFFCCF909352
:105D5000C600319694919923B1F7E6E5F2E094916B
:105D600008C08091C00085FFFCCF9093C60031969B
:105D700094919923B1F78CE095E061E070E04AE0FE
:105D800050E00E94E43E8091C00085FFFCCF8AE095
:105D90008093C6000E94104100C3E3EEF0E09491AE
:105DA00008C08091C00085FFFCCF9093C60031965B
:105DB00094919923B1F7EDE3F2E0949108C08091BA
:105DC000C00085FFFCCF9093C60031969491992333
:105DD000B1F7F40107C08091C00085FFFCCF319678
:105DE0009093C60090819923B1F7E2E3F2E0949199
:105DF00008C08091C00085FFFCCF9093C60031960B
:105E000094919923B1F7C6012DE032E0C20ED31E62
:105E1000B6010E94172E4BEF5FEFC40ED51ED601C0
:105E20009C91E8EFFDEFCE0EDF1E8DE8989FF0010C
:105E30001124E35FFD4FEC0DFD1D07C08091C000F4
:105E400085FFFCCF31969093C60090819923B1F7DE
:105E5000ECE2F2E0949108C08091C00085FFFCCF95
:105E60009093C600319694919923B1F722EA32E0DB
:105E7000C20ED31ED6014D915D916D917C91EEE5E0
:105E8000FDEFCE0EDF1E8CE095E02AE030E00E94B0
:105E90007F3E8091C00085FFFCCF8AE08093C600E2
:105EA000A601485F5D4FDA012C91E22FF0E0EE0F82
:105EB000FF1FEE0FFF1FEC0DFD1DE75FFD4F82EA98
:105EC00092E0C80ED91ED6014D905D906D907C90E9
:105ED0008EE59DEFC80ED91E408251826282738288
:105EE0002F5FDA012C932FC0E3EEF0E0949108C00D
:105EF0008091C00085FFFCCF9093C60031969491AD
:105F00009923B1F7EBE1F2E0949108C08091C000D1
:105F100085FFFCCF9093C600319694919923B1F7F9
:105F2000F40107C08091C00085FFFCCF31969093AB
:105F3000C60090819923B1F78091C00085FFFCCF06
:105F40008AE08093C600C60182539E4F0E942F8232
:105F500039C0E8E0F2E0CE0EDF1ED6011C92E8EF79
:105F6000FDEFCE0EDF1EE3EEF0E0949108C08091CD
:105F7000C00085FFFCCF9093C60031969491992381
:105F8000B1F7EAE0F2E0949108C08091C00085FF8B
:105F9000FCCF9093C600319694919923B1F7F40108
:105FA00007C08091C00085FFFCCF31969093C6005A
:105FB00090819923B1F78091C00085FFFCCF8AE0E2
:105FC0008093C600D60112961C921A8A1D8A198ADD
:105FD000188A81E694E09F878E87FEE4AF2EB12C6D
:105FE000AC0CBD1CEFE2F0E0CE0EDF1ED501CD9271
:105FF000DC92E1EDFFEFCE0EDF1ED4018C918F32EB
:1060000009F090C0C4016FE270E00E94C5247C01D9
:106010000894E11CF11C3E010894611C711C2501CF
:10602000E2E12E2E312C2C0E3D1E77C0C7016FE20F
:1060300070E00E94C5245C01009709F481C0E81655
:10604000F90608F07DC08C010E191F09C301B701C4
:10605000A8010E94E524060D171DF8011082F30126
:1060600007C08091C00085FFFCCF31969093C60099
:1060700090819923B1F78091C00085FFFCCFFAE0B1
:10608000F093C600D2016D917C916115710519F4F0
:1060900060E070E002C06C5F7F4FC101A30121E0AE
:1060A0000E943D89882371F5E6EFF1E0949108C0E4
:1060B0008091C00085FFFCCF9093C60031969491EB
:1060C0009923B1F7FE01319607C08091C00085FF8A
:1060D000FCCF31969093C60090819923B1F7E4EFFD
:1060E000F1E0949108C08091C00085FFFCCF9093AF
:1060F000C600319694919923B1F78091C00085FF35
:10610000FCCF1BC12EE030E02C0F3D1FF20131838C
:10611000208375010894E11CF11CE114F10409F0DD
:1061200085CF0BC040E550E0C40ED51ED501CD9201
:10613000DC92E0EBFFEFCE0EDF1E082DF92C01C044
:106140000E2DF601E25BFF4F2DA5222309F4B1C00D
:10615000608171816115710519F460E070E002C021
:106160006C5F7F4FC60182539E4F402F5F2D21E011
:106170000E943D89882309F46CC04FED51E0C40EA4
:10618000D51ED6014D915D916D917C91EBEBF0E0C8
:10619000CE0EDF1ED6014D935D936D937C931397C6
:1061A000E6E6FDEFCE0EDF1EE6EEF1E0949108C0CC
:1061B0008091C00085FFFCCF9093C60031969491EA
:1061C0009923B1F7802F9F2D9C01F90107C0809181
:1061D000C00085FFFCCF31969093C6009081992333
:1061E000B1F7EEEDF1E0949108C08091C00085FF19
:1061F000FCCF9093C600319694919923B1F78CE02F
:1062000095E02AE030E00E947F3E8091C00085FF4B
:10621000FCCF8AE08093C60022EA32E0C20ED31E91
:10622000D6011D921D921D921C921397E0EDF1E094
:10623000949108C08091C00085FFFCCF9093C60068
:10624000319694919923B1F78091C00085FFFCCFDE
:1062500099C0ECEBF1E0949108C08091C00085FFFB
:10626000FCCF9093C600319694919923B1F7802F7B
:106270009F2D9C01F90107C08091C00085FFFCCFD4
:1062800031969093C60090819923B1F7EAEBF1E043
:10629000949108C08091C00085FFFCCF9093C60008
:1062A000319694919923B1F78091C00085FFFCCF7E
:1062B00044C0608171816115710519F460E070E07E
:1062C00002C06C5F7F4FC60182539E4F402F5F2DEF
:1062D00026E50E943D89882309F033C0E6EAF1E013
:1062E000949108C08091C00085FFFCCF9093C600B8
:1062F000319694919923B1F7802F9F2D9C01F9013C
:1063000007C08091C00085FFFCCF31969093C600F6
:1063100090819923B1F7E4EAF1E0949108C080916B
:10632000C00085FFFCCF9093C600319694919923CD
:10633000B1F78091C00085FFFCCF8AE08093C60052
:1063400028C081E0F6018083E2E9F1E0949108C081
:106350008091C00085FFFCCF9093C6003196949148
:106360009923B1F7F40107C08091C00085FFFCCFED
:1063700031969093C60090819923B1F78091C00027
:1063800085FFFCCF8AE08093C600802F9F2D0E945E
:1063900048C1CE010E960E94252AAD960FB6F894FC
:1063A000DEBF0FBECDBFCF91DF911F910F91FF9048
:1063B000EF90DF90CF90BF90AF909F908F907F90A5
:1063C0006F905F904F903F902F900895FC0181E077
:1063D0008183CF0140E021E00E94602E0895835127
:1063E0009E4F0E9447830895CF92DF92EF92FF92D3
:1063F0000F931F938C017B016A0183519E4F40E0F4
:1064000050E060E070E00E941781C80187519E4F04
:10641000B701A6010E945D8A1F910F91FF90EF9036
:10642000DF90CF900895EF92FF920F931F93CF9339
:10643000DF93EC010E94EB918E01085F1D4FD801A4
:106440008C919EECE92E91E0F92EEC0EFD1E882336
:10645000A9F1C7010E942F82F80160816150608319
:106460008DE8689FB0011124635F7D4F6C0F7D1F25
:10647000CE0141E021E00E94602ED801EC91F0E0D5
:10648000EE0FFF1FEE0FFF1FEC0FFD1FE75FFD4F2D
:106490004081518162817381CE55DD4F488359839C
:1064A0006A837B83C25AD240C7010E9417818B81C5
:1064B000882309F462C081E08A835FC00E94C8918A
:1064C000C7010E942F821A82CE016BE37AE04AE56F
:1064D0000E94172B1092FD0710924B0ACE016DEF10
:1064E00077E04FE452E00E94F4318F5F9F4FA1F4B8
:1064F000E0E0F1E007C08091C00085FFFCCF31965D
:106500009093C60090819923B1F78091C00085FFD8
:10651000FCCF8AE08093C60010924D0A10924C0A7C
:10652000CE0183519E4F0E942F8287ED90E00E9402
:106530000F498091ED0F882301F11092ED0F8091AA
:10654000EB07C82FD0E0CC0FDD1FCD5AD84E6881A5
:106550007981882777FD8095982F0E94D7D7209141
:10656000A7033091A8034091A9035091AA030E9468
:1065700043D9181614F419821882DF91CF911F9114
:106580000F91FF90EF900895EF92FF920F931F935A
:10659000CF93DF938C01FC01138286A9882321F01D
:1065A000C801C3960E942F8227EAE22E21E0F22E34
:1065B000E00EF11EC70160E04FE10E94D57F882305
:1065C00009F5E3EEF0E0949108C08091C00085FFEA
:1065D000FCCF9093C600319694919923B1F7EAE1EC
:1065E000F3E0949108C08091C00085FFFCCF9093A8
:1065F000C600319694919923B1F78091C00085FF30
:10660000FCCF7DC0E801C455DE4FCE01B70141E0AB
:106610000E94D88A882341F5CE01B70140E00E944C
:10662000D88A882309F5E3E1F1E0949108C08091CC
:10663000C00085FFFCCF9093C600319694919923BA
:10664000B1F7E7E0F3E0949108C08091C00085FFC6
:10665000FCCF9093C600319694919923B1F7809125
:10666000C00085FFFCCF4BC0C801C396BE010E948D
:106670003085882309F5E3E1F1E0949108C0809129
:10668000C00085FFFCCF9093C6003196949199236A
:10669000B1F7E7EFF2E0949108C08091C00085FF68
:1066A000FCCF9093C600319694919923B1F78091D5
:1066B000C00085FFFCCF23C081E0F8018383E3EEB7
:1066C000F0E0949108C08091C00085FFFCCF9093CA
:1066D000C600319694919923B1F7ECEEF2E09491D3
:1066E00008C08091C00085FFFCCF9093C600319612
:1066F00094919923B1F78091C00085FFFCCF8AE087
:106700008093C600D801AC5ABF4FF801F3968BE1D5
:1067100001900D928150E1F7F80181A992A90E5ADA
:106720001F4FF8019183808302551040C8018F9656
:10673000025B1F4FF80191838083DF91CF911F91FE
:106740000F91FF90EF9008952F923F924F925F929A
:106750006F927F929F92AF92BF92CF92DF92EF9211
:10676000FF920F931F93DF93CF93CDB7DEB7CC5536
:10677000D0400FB6F894DEBF0FBECDBF6C016623CC
:1067800011F526EA32E0C20ED31ED6018C91EAE55D
:10679000FDEFCE0EDF1E882309F4E6C02EE932E0BD
:1067A000C20ED31ED601ED90FD900D911C91E2E634
:1067B000FDEFCE0EDF1E0E9469D0E616F706080731
:1067C000190708F4D1C026EA32E0C20ED31ED60162
:1067D0001C92EAE5FDEFCE0EDF1ED60113968C91DA
:1067E000882341F4C6010E94C432F60183818823C4
:1067F00009F4BAC000D000D000D0EDB7FEB7319692
:106800007E010894E11CF11CADB7BEB71296FC9254
:10681000EE9211978AE091E093838283D6019D9650
:106820008D919C919E97958384830E94F424870187
:10683000EDB7FEB736960FB6F894FEBF0FBEEDBFAC
:1068400057010AC0D8018C91992787FD90950E9425
:1068500078DBF80181938F01F50101900020E9F7C1
:106860003197EA19FB09802F8E198E175CF363E3C9
:10687000A62EB12CAC0CBD1CC50140E050E060E080
:1068800070E00E94178199245DE3E52EF12CEC0E57
:10689000FD1E2E010894411C511C4FE1642E712CE9
:1068A0006C0E7D1E33E0232E31E0332E43C0D80121
:1068B0008C9190E00E9478DBF80181938F01D701E1
:1068C0000D900020E9F71197AE19BF09802F8E199E
:1068D0008A176CF327968FAD27978E3759F1C7012A
:1068E000B20145E050E00E94D724009719F500D08E
:1068F00000D000D0EDB7FEB73196ADB7BEB7129657
:106900007C926E92119733822282558244820E9439
:10691000F424EDB7FEB736960FB6F894FEBF0FBE5F
:10692000EDBFC3010E943A488FEF90E00E940F49EB
:1069300099249394C501B70140E050E00E944C8433
:10694000181614F48701BBCF992041F48FEF9FEF05
:10695000D6019E969C938E939D9706C0F60185A5C1
:1069600096A5019696A785A7C45ADF4F0FB6F8944F
:10697000DEBF0FBECDBFCF91DF911F910F91FF9072
:10698000EF90DF90CF90BF90AF909F907F906F90EF
:106990005F904F903F902F9008952F923F924F928B
:1069A0005F926F927F928F929F92AF92BF92CF929F
:1069B000DF92EF92FF920F931F93DF93CF93CDB7A8
:1069C000DEB7CF58D0400FB6F894DEBF0FBECDBFB4
:1069D0008C013B016A0184E090E0C80ED91EF801E9
:1069E0007196C757DF4FF983E883C958D040C80173
:1069F0000496CA57DF4F99838883C658D040C8573A
:106A0000DF4F1882C858D040B6E6EB2EF12CEC0EC2
:106A1000FD1EF7013B96C557DF4FF983E883CB583E
:106A2000D040A7EA8A2EA2E09A2E800E911EF9EAA3
:106A3000AF2EF2E0BF2EA00EB11EEEE02E2E312CB6
:106A40002C0E3D1E77E4472E512C4C0E5D1EC201CC
:106A50000496C357DF4F99838883CD58D040E3EE27
:106A6000F0E09491C157DF4F9883CF58D0404FC189
:106A7000F7018385482F50E0BA016871707060316A
:106A8000710509F052C1F4012081318121303105B5
:106A900009F44BC12230310509F447C1F701DE0189
:106AA00011969081903239F08E2F8E19883011F422
:106AB0008EE28D939D933196C557DF4F88819981E2
:106AC000CB58D040E817F90761F71C921E86F301F6
:106AD0008081882329F4C10165E271E00E94BA2413
:106AE000C101B3010E94BA24C101BE016F5F7F4F93
:106AF0000E94BA24C10165E271E00E94BA241CA67A
:106B00001FA61BA61AA681E694E099A788A7CE0126
:106B10008C96B601AE014F5F5F4F21E00E943D8928
:106B2000882309F03FC0F40180819181892BD1F540
:106B3000C157DF4F9881CF58D040E3EEF0E008C056
:106B40008091C00085FFFCCF9093C6003196949150
:106B50009923B1F7E7E2F1E007C08091C00085FF1B
:106B6000FCCF31969093C60090819923B1F7809124
:106B7000C00085FFFCCFFAE0F093C600FE0131961D
:106B800007C08091C00085FFFCCF31969093C6006E
:106B900090819923B1F78091C00085FFFCCF8AE0F6
:106BA0008093C600C357DF4FA881B981CD58D0402C
:106BB000FE01BC968BE101900D928150E1F78AA510
:106BC0009BA5F2019383828381E694E09183808385
:106BD000C801B101A2010E94CD34C2010E94252A40
:106BE000CE0188960E94252A92C0953E09F48FC056
:106BF0009E3209F48CC09F3509F489C0F80191894F
:106C0000992331F09E3209F482C09F3509F47FC088
:106C100043FD7DC080E06031710509F481E0F80139
:106C200084A7882349F4F7018085873409F06FC071
:106C300081858E3709F46BC0CA57DF4FA881B981AF
:106C4000C658D040F7018081803241F08E2F8E19D6
:106C5000883011F48EE28D9380818D933196C557E3
:106C6000DF4F88819981CB58D040E817F90759F751
:106C70001C92F40180819181009729F5F30107C0EE
:106C80008091C00085FFFCCF31969093C600908123
:106C90009923B1F7CA57DF4FE881F981C658D04030
:106CA00007C08091C00085FFFCCF31969093C6004D
:106CB00090819923B1F78091C00085FFFCCFFAE065
:106CC000F093C60024C08130910539F4F50180812C
:106CD00091810196918380831AC00297C1F4C857AD
:106CE000DF4FF881C858D0402F2F30E0F501808168
:106CF000918128173907F1F0C857DF4FF881C8583C
:106D0000D040FF5FC857DF4FF883C858D040C60156
:106D1000B701C757DF4F48815981C958D0400E94F9
:106D20004C8418160CF4A4CE05C0F7019081992369
:106D300009F05BCFC157DF4F0FB6F894DEBF0FBE2F
:106D4000CDBFCF91DF911F910F91FF90EF90DF901A
:106D5000CF90BF90AF909F908F907F906F905F90FB
:106D60004F903F902F900895EF92FF920F931F93B3
:106D7000DF93CF93CDB7DEB76F970FB6F894DEBF32
:106D80000FBECDBF7C018C01025B1F4F805B9F4F0C
:106D9000F8019183808327EA32E0E20EF31E21E0BE
:106DA00030E0F701219331937F011182108227E5B2
:106DB0003DEFE20EF31E049640E050E060E070E02C
:106DC0000E941781F80120813181DE011596F901B9
:106DD00034968BE101900D928150E1F7F9018281A7
:106DE00093819C838B8381E694E09A838983C70196
:106DF0006AE371E08E010F5F1F4FA8010E94CD343E
:106E0000C8010E94252AF701E755FD4F8081918135
:106E10006F960FB6F894DEBF0FBECDBFCF91DF9156
:106E20001F910F91FF90EF900895EF92FF920F93B3
:106E30001F93DF93CF93CDB7DEB76F970FB6F8945C
:106E4000DEBF0FBECDBF7C018C01025B1F4F805B9C
:106E50009F4FF8019183808327EA32E0E20EF31E10
:106E600022E030E0F7013183208329E53DEFE20E97
:106E7000F31EF701E755FD4F60831182049640E051
:106E800050E060E070E00E941781F80120813181BC
:106E9000DE011596F90134968BE101900D92815037
:106EA000E1F7F901828193819C838B8381E694E0F1
:106EB0009A838983C7016AE371E08E010F5F1F4FD8
:106EC000A8010E94CD34C8010E94252A6F960FB6F2
:106ED000F894DEBF0FBECDBFCF91DF911F910F9110
:106EE000FF90EF900895EF92FF920F931F93DF931F
:106EF000CF93CDB7DEB76F970FB6F894DEBF0FBE56
:106F0000CDBF7C0187EA92E0E80EF91EF7011182FD
:106F1000108289E59DEFE80EF91E87010D5C1F4F79
:106F2000C80140E050E060E070E00E941781DE019F
:106F30001596F8018BE101900D928150E1F7F70170
:106F400081A992A99C838B8381E694E09A838983AB
:106F5000C7016AE371E08E010F5F1F4FA8010E9415
:106F6000CD34C8010E94252A6F960FB6F894DEBF73
:106F70000FBECDBFCF91DF911F910F91FF90EF908A
:106F800008950F931F93CF93DF93DC01D3961C9248
:106F9000D397D6961C92D697D2961C921E92D197D2
:106FA00081E694E0D0969C938E939F97AC5ABF4F06
:106FB0001C9213961C92A755B040FD01E05BFF4F59
:106FC000AE5ABF4F11961C921E92A255B0409183AB
:106FD0008083ED01C159DF4FFE0120E030E0482FF2
:106FE000148217821382128240839183215E3F4F65
:106FF0007F9681E02633380799F7A855BE4F89E17F
:107000008C9313961C9258961C921B961C92139666
:107010001C92A15DB140FD01E653FE4FA453BE4F4B
:1070200011961C921E924083918391961C92139606
:107030001C92A05FB140FD01E751FE4FA551BE4F2C
:1070400011961C921E9240839183A155BF4F1D92B1
:107050001D921D921C92139718961D921D921D92BF
:107060001C921397A25AB24012961C921297139632
:107070001C9213971C9211961C9211978D01025627
:107080001D4FF8011082118212821382AB55BE4F40
:1070900011961C921E92AD59BF4F1C92FE01C90160
:1070A00011920197E9F7A256BF4F81E08C93A65A3F
:1070B000B2409E961C921E929D970E9469D068577E
:1070C0007C4E8F4F9F4FF80160837183828393833F
:1070D000DF91CF911F910F910895DF93CF93CDB79B
:1070E000DEB7E0970FB6F894DEBF0FBECDBFDE016E
:1070F0001196E1E1F4E080E101900D928150E1F719
:10710000DE015196E1E0F4E080E101900D928150C2
:10711000E1F7DE019196E1EFF3E080E101900D925D
:107120008150E1F789819A81AB81BC818093910F75
:107130009093920FA093930FB093940F89899A899B
:10714000AB89BC898093810F9093820FA093830FAA
:10715000B093840F89A19AA1ABA1BCA18093A10F88
:107160009093A20FA093A30FB093A40F8D819E8143
:10717000AF81B8858093950F9093960FA093970F4A
:10718000B093980F8D899E89AF89B88D8093850FB4
:107190009093860FA093870FB093880F8DA19EA127
:1071A000AFA1B8A58093A50F9093A60FA093A70FAA
:1071B000B093A80F89859A85AB85BC858093990F7C
:1071C00090939A0FA0939B0FB0939C0F898D9A8DEB
:1071D000AB8DBC8D8093890F90938A0FA0938B0FFA
:1071E000B0938C0F89A59AA5ABA5BCA58093A90FD8
:1071F0009093AA0FA093AB0FB093AC0F8D859E8593
:10720000AF85B88980939D0F90939E0FA0939F0F99
:10721000B093A00F8D8D9E8DAF8DB8A180938D0FF3
:1072200090938E0FA0938F0FB093900F8DA59EA576
:10723000AFA5B8A98093AD0F9093AE0FA093AF0FF9
:10724000B093B00F0E94046D80E090E0AAEFB3E429
:107250008093B50F9093B60FA093B70FB093B80F6C
:107260008093B90F9093BA0FA093BB0FB093BC0F4C
:1072700020E030E040E050E02093B10F3093B20FB7
:107280004093B30F5093B40F80E29EE4A0E0B0E0CF
:1072900080937D0F90937E0FA0937F0FB093800F0C
:1072A0002093C90F3093CA0F4093CB0F5093CC0F4C
:1072B00080E090E0A0EAB1E48093BD0F9093BE0F10
:1072C000A093BF0FB093C00F8DEC9CECACECBEE371
:1072D0008093C10F9093C20FA093C30FB093C40FBC
:1072E00080E090E0A0EAB0E48093C50F9093C60FD1
:1072F000A093C70FB093C80F2093D8073093D90736
:107300004093DA075093DB072093D4073093D507D7
:107310004093D6075093D7072093D0073093D107D7
:107320004093D2075093D30789EB90E09093A61730
:107330008093A5171092A8171092A7172FEF30E08F
:107340003093AA172093A91780EF90E09093AC1781
:107350008093AB171092AE171092AD173093B01701
:107360002093AF1780E290E09093B3198093B21905
:107370008AE097EDADEAB1E48093B4039093B5034E
:10738000A093B603B093B70368EB7EE185EC9FE36F
:107390000E94DA996093B8037093B9038093BA039B
:1073A0009093BB036AE979E189E992E40E94E89944
:1073B0006093BC037093BD038093BE039093BF039F
:1073C0000E94F89880E090E0A0E8BFE38093C003BB
:1073D0009093C103A093C203B093C303E7E2F3E029
:1073E000949108C08091C00085FFFCCF9093C600A7
:1073F000319694919923B1F7EDE2F3E0949108C0AE
:107400008091C00085FFFCCF9093C6003196949187
:107410009923B1F78091C00085FFFCCF8AE080936B
:10742000C600E0960FB6F894DEBF0FBECDBFCF9179
:10743000DF910895CF93DF93C7E2D3E0FE019491EB
:1074400008C08091C00085FFFCCF9093C6003196A4
:1074500094919923B1F7E7E0F5E0949108C0809109
:10746000C00085FFFCCF9093C6003196949199237C
:10747000B1F78091C00085FFFCCF8AE08093C60001
:10748000FE019491E7E2F3E008C08091C00085FF1F
:10749000FCCF9093C600319694919923B1F7409117
:1074A000910F5091920F6091930F7091940F8FEF05
:1074B00094E00E94A1434091950F5091960F6091E6
:1074C000970F7091980F8CEF94E00E94A143409128
:1074D000990F50919A0F60919B0F70919C0F89EFBB
:1074E00094E00E94A14340919D0F50919E0F6091A6
:1074F0009F0F7091A00F86EF94E00E94A143EBE3F1
:10750000F1E007C08091C00085FFFCCF31969093D9
:10751000C60090819923B1F78091C00085FFFCCF10
:107520008AE08093C600FE019491E7E2F3E008C090
:107530008091C00085FFFCCF9093C6003196949156
:107540009923B1F7ECEDF4E0949108C08091C0006C
:1075500085FFFCCF9093C600319694919923B1F7A3
:107560008091C00085FFFCCF8AE08093C600FE01B9
:107570009491E7E2F3E008C08091C00085FFFCCF62
:107580009093C600319694919923B1F74091810F61
:107590005091820F6091830F7091840F83ED94E07E
:1075A0000E94A1434091850F5091860F6091870FF3
:1075B0007091880F80ED94E00E94A1434091890F63
:1075C00050918A0F60918B0F70918C0F8DEC94E02D
:1075D0000E94A14340918D0F50918E0F60918F0FAB
:1075E0007091900F8AEC94E00E94A143EBE3F1E0EC
:1075F00007C08091C00085FFFCCF31969093C600F4
:1076000090819923B1F78091C00085FFFCCF8AE07B
:107610008093C600FE019491E7E2F3E008C08091F8
:10762000C00085FFFCCF9093C600319694919923BA
:10763000B1F7ECEAF4E0949108C08091C00085FFB6
:10764000FCCF9093C600319694919923B1F7809125
:10765000C00085FFFCCF8AE08093C600FE019491B4
:10766000E7E2F3E008C08091C00085FFFCCF909373
:10767000C600319694919923B1F74091A10F509192
:10768000A20F6091A30F7091A40F83EA94E00E946F
:1076900026484091A50F5091A60F6091A70F7091B9
:1076A000A80F80EA94E00E9426484091A90F5091CB
:1076B000AA0F6091AB0F7091AC0F8DE994E00E941E
:1076C00026484091AD0F5091AE0F6091AF0F709171
:1076D000B00F8AE994E00E942648EBE3F1E007C08E
:1076E0008091C00085FFFCCF31969093C6009081B9
:1076F0009923B1F78091C00085FFFCCF8AE0809389
:10770000C600FE019491E7E2F3E008C08091C0005A
:1077100085FFFCCF9093C600319694919923B1F7E1
:10772000E5E6F4E0949108C08091C00085FFFCCFAD
:107730009093C600319694919923B1F78091C0003F
:1077400085FFFCCF8AE08093C600FE019491E7E2BA
:10775000F3E008C08091C00085FFFCCF9093C60085
:10776000319694919923B1F74091B50F5091B60F8E
:107770006091B70F7091B80F8CE594E00E94A1431F
:107780004091B90F5091BA0F6091BB0F7091BC0F2F
:1077900089E594E00E94A143EBE3F1E007C080910A
:1077A000C00085FFFCCF31969093C600908199234D
:1077B000B1F78091C00085FFFCCF8AE08093C600BE
:1077C000FE019491E7E2F3E008C08091C00085FFDC
:1077D000FCCF9093C600319694919923B1F7E6EAD5
:1077E000F3E0949108C08091C00085FFFCCF909396
:1077F000C600319694919923B1F78091C00085FF1E
:10780000FCCF8AE08093C600FE019491E7E2F3E0AA
:1078100008C08091C00085FFFCCF9093C6003196D0
:1078200094919923B1F74091B10F5091B20F6091AB
:10783000B30F7091B40F8DE993E00E94A143409182
:10784000C90F5091CA0F6091CB0F7091CC0F8AE98C
:1078500093E00E94A14340917D0F50917E0F609173
:107860007F0F7091800F87E993E00E942648409136
:10787000BD0F5091BE0F6091BF0F7091C00F84E992
:1078800093E00E94A1434091C10F5091C20F6091BB
:10789000C30F7091C40F81E993E00E94A14340910E
:1078A000C50F5091C60F6091C70F7091C80F8EE839
:1078B00093E00E94A143EBE3F1E007C08091C00098
:1078C00085FFFCCF31969093C60090819923B1F744
:1078D0008091C00085FFFCCF8AE08093C600FE0146
:1078E0009491E7E2F3E008C08091C00085FFFCCFEF
:1078F0009093C600319694919923B1F7ECE7F3E0A9
:10790000949108C08091C00085FFFCCF9093C60081
:10791000319694919923B1F78091C00085FFFCCFF7
:107920008AE08093C600FE019491E7E2F3E008C08C
:107930008091C00085FFFCCF9093C6003196949152
:107940009923B1F74091D0075091D1076091D207A8
:107950007091D30783E793E00E94A1434091D4073D
:107960005091D5076091D6077091D70780E793E0D3
:107970000E94A1434091D8075091D9076091DA073E
:107980007091DB078DE693E00E94A143EBE3F1E009
:1079900007C08091C00085FFFCCF31969093C60050
:1079A00090819923B1F78091C00085FFFCCF8AE0D8
:1079B0008093C600FE019491E7E2F3E008C0809155
:1079C000C00085FFFCCF9093C60031969491992317
:1079D000B1F7EFE5F3E0949108C08091C00085FF16
:1079E000FCCF9093C600319694919923B1F7809182
:1079F000C00085FFFCCF8AE08093C600FE01949111
:107A0000E7E2F3E008C08091C00085FFFCCF9093CF
:107A1000C600319694919923B1F74091B4035091E7
:107A2000B5036091B6037091B70385E593E00E94BA
:107A3000A1436091B8037091B9038091BA0390910A
:107A4000BB030E94E199AB01BC0182E593E00E9477
:107A5000A1436091BC037091BD038091BE039091DE
:107A6000BF030E94EF99AB01BC018FE493E00E9439
:107A7000A143EBE3F1E007C08091C00085FFFCCF9C
:107A800031969093C60090819923B1F78091C00000
:107A900085FFFCCF8AE08093C600DF91CF910895E7
:107AA0001F920F920FB60F920BB60F9211242F93C5
:107AB0003F934F938F939F93EF93FF934091C60013
:107AC000E0910805F091090531969F012F773070FC
:107AD000319780910A0590910B052817390739F0E5
:107AE000E857FB4F40833093090520930805FF9129
:107AF000EF919F918F914F913F912F910F900BBEDE
:107B00000F900FBE0F901F9018959A01AB01203077
:107B100081EE380780E0480780E0580749F182E0AD
:107B20008093C00060E079E08DE390E00E944FDB3D
:107B30002150304040405040CA01B90122E030E0BD
:107B400040E050E00E944FDB3093C5002093C4001A
:107B50008091C10080618093C1008091C1008860E4
:107B60008093C1008091C10080688093C100089516
:107B70001092C00020E130E0E7CF20910A0530915B
:107B80000B0580910805909109058217930719F458
:107B90002FEF3FEF0EC0F901E857FB4F80812F5FB9
:107BA0003F4F2F77307030930B0520930A05282F15
:107BB00030E0C901089580910A0590910B059093DA
:107BC000090580930805089508952F923F924F92DA
:107BD0005F926F927F928F929F92AF92BF92CF925D
:107BE000DF92EF92FF920F931F93DF93CF93CDB766
:107BF000DEB7A0970FB6F894DEBF0FBECDBF1C0155
:107C00006A017B01411551056105710549F440E3A5
:107C100050E060E070E020E030E00E94AF3E56C0EF
:107C2000882499245401422E55246624772401E0A7
:107C300010E00C0F1D1F080D191DC701B601A3018F
:107C400092010E942DDBF80160830894811C911C35
:107C5000A11CB11CC701B601A30192010E942DDB3A
:107C6000C901DA016C017D01C114D104E104F10400
:107C7000F1F681E0E82EF12CEC0EFD1EE80CF91C6B
:107C80003E010894611C711CD501C4010197A10932
:107C9000B1096C01C818D90816C0F601EE0DFF1D18
:107CA00040814A3010F4405D01C0495C552747FDD2
:107CB0005095652F752FC10120E030E00E94AF3E46
:107CC0000894E108F1086E147F0439F7A0960FB606
:107CD000F894DEBF0FBECDBFCF91DF911F910F9102
:107CE000FF90EF90DF90CF90BF90AF909F908F90DC
:107CF0007F906F905F904F903F902F900895211547
:107D0000310539F48091C00085FFFCCF4093C60057
:107D100008950E94E53D0895EF92FF920F931F93FF
:107D20009A017B0100E010E0B801A7010E947F3EAC
:107D30001F910F91FF90EF900895EF92FF920F9394
:107D40001F939A01E62EFF2400E010E0B801A7017E
:107D50000E947F3E1F910F91FF90EF900895EF9248
:107D6000FF920F931F93CF93DF93EC017A018B0166
:107D70002115310539F48091C00085FFFCCFE092D8
:107D8000C6001BC02A303105B1F477FF10C04DE2A8
:107D900050E060E070E020E030E00E94AF3E1095DF
:107DA0000095F094E094E11CF11C011D111DCE0121
:107DB000B801A7012AE00E94E53DDF91CF911F9114
:107DC0000F91FF90EF900895EF92FF920F931F9302
:107DD0007B019A010027F7FC0095102FB801A7013D
:107DE0000E94AF3E1F910F91FF90EF9008950F9367
:107DF0001F938C014DE050E060E070E020E030E047
:107E00000E94AF3EC8014AE050E060E070E020E030
:107E100030E00E94AF3E1F910F910895CF92DF9204
:107E2000EF92FF920F931F938C019A016B01EE2446
:107E3000FF24B701A6010E947F3EC8010E94F73EC1
:107E40001F910F91FF90EF90DF90CF9008959F9238
:107E5000AF92BF92CF92DF92EF92FF920F931F9358
:107E6000CF93DF93EC017A018B01922ECB01BA0103
:107E700020E030E040E050E00E9435D788236CF4E9
:107E8000CE014DE250E060E070E020E030E00E9482
:107E9000AF3E17FB109517F91095AA2420E030E0AB
:107EA00040E05FE30BC0CA01B90120E030E040E2EE
:107EB00051E40E943CD79B01AC01A394A91498F310
:107EC000C801B7010E945CD67B018C010E94A9D732
:107ED0005B016C010E94D5D79B01AC01C801B701C1
:107EE0000E945BD67B018C01CE01B601A5012AE080
:107EF00030E00E947F3E9920A1F1ECE3F1E007C061
:107F00008091C00085FFFCCF31969093C600908190
:107F10009923B1F726C0C801B70120E030E040E264
:107F200051E40E9415DA7B018C010E94A4D75B0109
:107F30006C01CC24B7FCC094DC2CCE01B601A501A9
:107F40002AE030E00E94AF3EC601B5010E94D7D7BB
:107F50009B01AC01C801B7010E945BD67B018C017B
:107F60009A949920C1F6DF91CF911F910F91FF90C4
:107F7000EF90DF90CF90BF90AF909F9008950E94B8
:107F8000273F0895EF92FF920F931F93CF93DF93B4
:107F9000EC01E090DC07F090DD070091DE07109126
:107FA000DF07688179818A819B81A80197010E94FE
:107FB00035D7882324F4E882F9820A831B83E09072
:107FC000E007F090E1070091E2071091E3076C8170
:107FD0007D818E819F81A80197010E9435D78823DA
:107FE00024F4EC82FD820E831F83E090E407F0907E
:107FF000E5070091E6071091E707688579858A858E
:108000009B85A80197010E9435D7882324F4E88630
:10801000F9860A871B87E0907A03F0907B03009132
:108020007C0310917D03688179818A819B81A801FD
:1080300097010E9443D9181624F4E882F9820A8332
:108040001B83E0907E03F0907F03009180031091EA
:1080500081036C817D818E819F81A80197010E949F
:1080600043D9181624F4EC82FD820E831F83E0901E
:108070008203F09083030091840310918503688547
:1080800079858A859B85A80197010E9443D9181696
:1080900024F4E886F9860A871B87DF91CF911F9128
:1080A0000F91FF90EF9008958091F80708950F9336
:1080B0001F93CF93DF938130910569F46F5F7F4FFA
:1080C00009F059C08DE095E00E94C13789EF97E033
:1080D0000E94158F50C0892B09F04DC06F5F7F4FF4
:1080E00009F049C081E694E09093F7068093F60684
:1080F0008091FD06882321F08AEF96E00E942F826E
:1081000081E694E09093D8068093D7068091DE06AE
:10811000882321F08BED96E00E942F82C3E9D6E000
:1081200001E614E005C06F9785E0CD35D80751F022
:10813000198308838F818823B1F3CE0104960E94AE
:108140002F82F1CF81E694E0998388838F81882301
:1081500021F0CE0104960E942F8281E694E0909354
:108160003D0580933C0580914305882321F080E400
:1081700095E00E942F82DF91CF911F910F9108957A
:1081800080E090E06FEF7FEF0E945740089581E01C
:1081900090E06FEF7FEF0E94574008950E94CB99C7
:1081A0008091F807882309F03AC081E08093F807AE
:1081B0008091510A9091520AA091530AB091540AA9
:1081C0008093550A9093560AA093570AB093580A81
:1081D000EDE1F5E0949108C08091C00085FFFCCFEF
:1081E0009093C600319694919923B1F7EEE2F5E0B1
:1081F000949108C08091C00085FFFCCF9093C60089
:10820000319694919923B1F78091C00085FFFCCFFE
:108210008AE08093C60084E295E00E9425C108951B
:10822000F8940E94CB995E9A1092E8075E9A109299
:10823000E907159A1092EA075E9AEDE1F5E094914C
:1082400008C08091C00085FFFCCF9093C600319696
:1082500094919923B1F7EDEAF5E0949108C08091EB
:10826000C00085FFFCCF9093C6003196949199236E
:10827000B1F78091C00085FFFCCF8AE08093C600F3
:1082800084EA95E00E9434C1FFCF0E9469D06093D8
:10829000590A70935A0A80935B0A90935C0AE091A2
:1082A000820AF091830AEC57F54F80818823A9F464
:1082B000ECECF5E0949108C08091C00085FFFCCF04
:1082C0009093C600319694919923B1F78091C000A4
:1082D00085FFFCCF8AE08093C6000895EF92FF925D
:1082E0000F931F930E9469D0E0905D0AF0905E0AA0
:1082F00000915F0A1091600A2091590A30915A0A40
:1083000040915B0A50915C0A621B730B840B950BC6
:10831000E616F7060807190738F4E114F104010519
:10832000110511F00E94104180919A0390919B03D6
:10833000A0919C03B0919D030097A105B10559F14F
:108340000E9469D02091590A30915A0A40915B0AE3
:1083500050915C0A621B730B840B950B20919A035E
:1083600030919B0340919C0350919D032617370742
:108370004807590780F49091BE148091BF14981754
:1083800051F45E9A1092E8075E9A1092E907159AE6
:108390001092EA075E9A0E94746F1F910F91FF90EE
:1083A000EF9008956F927F928F929F92AF92BF92BB
:1083B000CF92DF92EF92FF920F931F93F82E60916E
:1083C000610A7091620A8091630A9091640A209117
:1083D000650A3091660A4091670A5091680A0E94C6
:1083E00050D93B014C0100D000D000D00DB71EB7D2
:1083F0000F5F1F4F6091720370917303882777FDA1
:108400008095982F0E94D7D720919E0330919F038B
:108410004091A0035091A1030E9415DA20E030E0C2
:1084200040E752E40E943CD720E030E048EC52E4C0
:108430000E943CD75B016C01F801608271828282EC
:108440009382F4828091EB07858380EC97E06DE660
:108450007AE041E65AE020E001E032E0E32E0E94BB
:10846000606880916D0A90916E0AA0916F0AB09138
:10847000700A8093C0079093C107A093C207B0937E
:10848000C3078091710A9091720AA091730AB0910A
:10849000740A8093C4079093C507A093C607B0934E
:1084A000C7078091750A9091760AA091770AB091DA
:1084B000780A8093C8079093C907A093CA07B0931E
:1084C000CB078091790A90917A0AA0917B0AB091AA
:1084D0007C0A8093CC079093CD07A093CE07B093EE
:1084E000CF078DB79EB706960FB6F8949EBF0FBE06
:1084F0008DBF0E9469D06093590A70935A0A809385
:108500005B0A90935C0A1F910F91FF90EF90DF90B0
:10851000CF90BF90AF909F908F907F906F90089575
:10852000CF92DF92EF92FF920F931F938DE69AE026
:108530000E94C23F0E9469D06093590A70935A0A00
:1085400080935B0A90935C0A6091C0077091C107A9
:108550008091C2079091C30720916D0A30916E0AF5
:1085600040916F0A5091700A0E9435D7882309F014
:108570007AC06091C4077091C5078091C607909139
:10858000C7072091710A3091720A4091730A509185
:10859000740A0E9435D7882309F065C060919E0354
:1085A00070919F038091A0039091A10320E030E09F
:1085B00040E752E40E943CD77B018C018DE69AE0B3
:1085C00061E77AE045E75AE029E73AE0EBEECE2EA4
:1085D000E7E0DE2E0E945D7280916D0A90916E0A36
:1085E000A0916F0AB091700A8093C0079093C10761
:1085F000A093C207B093C3078091710A9091720A49
:10860000A091730AB091740A8093C4079093C50730
:10861000A093C607B093C7078091750A9091760A18
:10862000A091770AB091780A8093C8079093C90700
:10863000A093CA07B093CB078091790A90917A0AE8
:10864000A0917B0AB0917C0A8093CC079093CD07D0
:10865000A093CE07B093CF071F910F91FF90EF909B
:10866000DF90CF9008956091720370917303882713
:1086700077FD8095982F0E94D7D720919E03309147
:108680009F034091A0035091A1030E9415DA20E0BE
:1086900030E040E752E40E943CD720E030E048EC74
:1086A00052E488CF8CE095E00E94DB3DEFECF5E0F2
:1086B000949108C08091C00085FFFCCF9093C600C4
:1086C000319694919923B1F74091510A5091520AF1
:1086D0006091530A7091540A4F5F5F4F6F4F7F4F05
:1086E0008CE095E02AE030E00E94AF3E8091C0002F
:1086F00085FFFCCF8AE08093C6000E944541089523
:108700004091820A5091830A20E630E0B901469FE9
:108710009001479F300D569F300D1124682F772709
:1087200067FD7095C9018257954F0E94C5249C0131
:1087300090938D0A80938C0A80E0232B09F081E0CE
:108740000895FC01949108C08091C00085FFFCCF82
:108750009093C600319694919923B1F78CE095E0FF
:1087600022E030E00E94BF3F08952F923F924F9247
:108770005F926F927F928F929F92AF92BF92CF92B1
:10878000DF92EF92FF920F931F93DF93CF93CDB7BA
:10879000DEB728970FB6F894DEBF0FBECDBF9A8321
:1087A00089838330910508F091C1FC01EB51F84FAA
:1087B000D4908C01000F111F000F111FF801E0541D
:1087C000F84F80E090E0A0E0B0E080839183A28346
:1087D000B38380EC97E064EC77E048EC57E02CEC56
:1087E00037E00E944D6DE981FA81EE0FFF1FEA57D5
:1087F000FC4F0190F081E02DF7FD0EC0CF01880FF6
:10880000991F8E0F9F1F04571C4FD8016D917C91AB
:108810008750984F0E94DF8F69807A80660C771CA2
:10882000660C771CF301E851F84FE590F59005913F
:1088300014916D2D772767FD7095882777FD8095BA
:10884000982F0E94D7D71B012C01F301E359F54F54
:10885000F887EF83C801B70120E030E040EC5FE328
:108860000E9415DAA20191010E9415DAAF81B88544
:108870006D937D938D939C931397F301EE59FC4F69
:10888000FC83EB83608171818281938160939E037D
:1088900070939F038093A0039093A10320E030E0A6
:1088A00040E752E40E943CD77B018C018DE69AE0C0
:1088B00061E77AE045E75AE029E73AE0EBEECE2EB1
:1088C000E7E0DE2E0E945D720E94EB91930120543E
:1088D000384F3E832D8380E090E0A0E0B0E0F901C6
:1088E00080839183A283B38380EC97E064EC77E08C
:1088F00048EC57E02CEC37E00E944D6DF301EC5052
:10890000F84F85909590A590B490C501B40190580A
:10891000A20191010E9415DAAF81B8856D937D9314
:108920008D939C93139760919E0370919F03809108
:10893000A0039091A10320E030E040E752E40E94C0
:108940003CD77B018C018DE69AE061E77AE045E750
:108950005AE029E73AE00E945D720E94EB91C5015E
:10896000B401A50194010E945CD6A20191010E946C
:1089700015DAEF81F8856083718382839383AB81FD
:10898000BC816D917D918D919C9120E030E040E023
:108990005FE30E9415DA60939E0370939F038093B8
:1089A000A0039093A10320E030E040E752E40E944E
:1089B0003CD77B018C018DE69AE061E77AE045E7E0
:1089C0005AE029E73AE00E945D720E94EB91F301C0
:1089D000E050F84F6591759185919491F301E053C2
:1089E000F84FA080B180C280D380A60195010E947B
:1089F0005CD67B018C01CB01D801ED81FE818083A7
:108A00009183A283B383F301E45FF74F659175917E
:108A1000859194912CED822E27E0922E860C971C46
:108A2000A60195010E945CD6D4016D937D938D9330
:108A30009C931397F301E85EF74F659175918591CB
:108A40009491EAE7F3E06E0E7F1EA60195010E9465
:108A50005CD6D3016D937D938D939C931397C7013F
:108A6000D801EF81F88580839183A283B38380E06E
:108A700090E0A0E0B0E080939E0390939F03A093CA
:108A8000A003B093A1030E940991E981FA81E85102
:108A9000F84F81E08083A981BA81AA0FBB1FFD0135
:108AA000EA57FC4F0190F081E02DF7FD0FC0CF0198
:108AB000880F991F8E0F9F1FAA0FBB1FA257BC4F75
:108AC0006D917C918750984F0E94DF8F28960FB64A
:108AD000F894DEBF0FBECDBFCF91DF911F910F91F4
:108AE000FF90EF90DF90CF90BF90AF909F908F90CE
:108AF0007F906F905F904F903F902F9008950F93CD
:108B00001F93CF93DF93C6E8D3E00EE813E02881EC
:108B1000398137FD0CC0C901880F991F820F931F3F
:108B2000F801608171818750984F0E94DF8F2296F3
:108B30000C5F1F4FF3E0CC38DF0749F7DF91CF918F
:108B40001F910F91089580918C0A90918D0A019642
:108B500060E070E04AE050E00E9434230895809184
:108B60008C0A90918D0A019660E070E00E94D421F9
:108B70000895CF93DF93EC018091EB078093500A27
:108B800084E50E948043882309F46FC00E94AF45AA
:108B90000E94A9D7262F6093500A662309F465C066
:108BA000E7E1F5E0949108C08091C00085FFFCCF1B
:108BB0009093C600319694919923B1F7C936D105A7
:108BC00099F0CA36D10524F4C836D105F1F50FC0A5
:108BD000CD36D10531F0CA3DD105B9F5EEE3F1E06E
:108BE00031C0E5E5F1E023C0ECE6F1E015C0E3E8D3
:108BF000F1E007C08091C00085FFFCCF31969093D3
:108C0000C60090819923B1F720C08091C00085FFF4
:108C1000FCCF31969093C60090819923B1F715C08F
:108C20008091C00085FFFCCF31969093C600908163
:108C30009923B1F70AC08091C00085FFFCCF31961F
:108C40009093C60090819923B1F78CE095E0622F54
:108C500040E050E00E949D3E8091C00085FFFCCF27
:108C60008AE08093C60081E001C080E0DF91CF916F
:108C70000895AF92BF92CF92DF92EF92FF920F933F
:108C80001F93CF93DF9350ECE52E57E0F52ECDE602
:108C9000DAE000E010E0F801EF5DFB4F80810E9418
:108CA0008043882339F10E94AF455B016C01F801D4
:108CB000E654F84F8081882311F061E002C0609192
:108CC0007D0A70E0882777FD8095982F0E94D7D77E
:108CD000F70120813181428153810E9415DA9B0185
:108CE000AC01C601B5010E945CD6688379838A8392
:108CF0009B8309C0F70180819181A281B381888320
:108D00009983AA83BB830F5F1F4F84E090E0E80E36
:108D1000F91E24960430110509F0BDCF86E40E94A7
:108D200080438823E1F00E94AF457B018C01609372
:108D30007E0A70937F0A8093800A9093810A20E0D4
:108D400030E040E050E00E9443D9181644F4E0922D
:108D50009E03F0929F030093A0031093A103DF9161
:108D6000CF911F910F91FF90EF90DF90CF90BF9028
:108D7000AF9008950E94394689E40E948043882379
:108D800059F00E94AF456093610A7093620A809324
:108D9000630A9093640A0CC080E090E0A0E0B0E029
:108DA0008093610A9093620AA093630AB093640A65
:108DB0008AE40E948043882359F00E94AF45609363
:108DC000650A7093660A8093670A9093680A08950B
:108DD00080E090E0A0E0B0E08093650A9093660A9E
:108DE000A093670AB093680A0895EF92FF920F93D9
:108DF0001F9380911005882309F423C180910F05EA
:108E0000882309F41EC1E090C807F090C9070091BB
:108E1000CA071091CB07C801B70120E030E040E05D
:108E200050E00E9443D918160CF00BC16091120853
:108E3000709113088091140890911508A80197016A
:108E40000E9435D7882309F4FCC061E070E080E01F
:108E500090E020E031E040E050E00E943DD6609399
:108E6000FD0760934B0A8091C0079091C107A091C4
:108E7000C207B091C3078093FE079093FF07A093AA
:108E80000008B09301088091C4079091C507A09194
:108E9000C607B091C7078093020890930308A09378
:108EA0000408B09305082091C8073091C907409184
:108EB000CA075091CB0720930608309307084093C8
:108EC0000808509309088091CC079091CD07A09194
:108ED000CE07B091CF0780930A0890930B08A09318
:108EE0000C08B0930D082093120830931308409398
:108EF00014085093150880919E0390919F03A091B0
:108F0000A003B091A10380930E0890930F08A09343
:108F10001008B093110880915317909154179093B3
:108F200017088093160880915517909156179093C3
:108F300019088093180880915717909158179093AB
:108F40001B0880931A088091591790915A17909393
:108F50001D0880931C088091551790915617909387
:108F60001F0880931E088091820A9091830A909333
:108F70002108809320088091120C9091130C9093FB
:108F80002308809322088091180C9091190C9093DB
:108F9000250880932408A6E2B8E0EEE8FAE080E82D
:108FA00091E001900D920197E1F78091EE07909189
:108FB000EF07A091F007B091F1078093AA09909371
:108FC000AB09A093AC09B093AD098DE095E06EEAD2
:108FD00079E00E94172E8091AF079091B007A09181
:108FE000B107B091B2078093A6099093A709A09307
:108FF000A809B093A9098DE095E06BE37AE04AE512
:109000000E94172B8DE095E06DEF77E04FE452E082
:109010000E94F4318F5F9F4FA1F4EAE9F1E007C0AD
:109020008091C00085FFFCCF31969093C60090815F
:109030009923B1F78091C00085FFFCCF8AE080932F
:10904000C6001F910F91FF90EF900895FC0194913D
:1090500008C08091C00085FFFCCF9093C600319678
:1090600094919923B1F78CE095E02AE030E00E94DA
:109070007F3E0895CF93DF93FC0180818B3309F409
:109080006FC08091180C9091190C04970CF068C077
:109090008091120C9091130C20E630E0829FE00149
:1090A000839FD00D929FD00D1124C257D54FCE0172
:1090B000BF010E94D024E7E1F5E0949108C08091BF
:1090C000C00085FFFCCF9093C60031969491992300
:1090D000B1F7E8EBFAE0949108C08091C00085FFF9
:1090E000FCCF9093C600319694919923B1F7FE017D
:1090F00007C08091C00085FFFCCF31969093C600D9
:1091000090819923B1F7E6EBFAE0949108C0809141
:10911000C00085FFFCCF9093C600319694919923AF
:10912000B1F78091C00085FFFCCF8AE08093C60034
:109130008091120C9091130C019664E070E00E94F3
:109140001ADB9093130C8093120C8091180C909161
:10915000190C01969093190C8093180C81E001C0B2
:1091600080E0DF91CF910895EF92FF920F931F93CC
:10917000DF93CF93CDB7DEB76E970FB6F894DEBF0F
:109180000FBECDBF6091F6077091F70761157105AD
:1091900011F480E037C08E010F5F1F4FC8014DE111
:1091A00050E00E947B241E8EEE24FF24C801FC01A7
:1091B000EE0DFF1D1081112331F01A3021F00894BB
:1091C000E11CF11CF4CFCE010196FC01EE0DFF1D58
:1091D00010820E943A488823A1F0112371F008946C
:1091E000E11CF11C8091F6079091F7078E0D9F1DF1
:1091F0009093F7078093F60704C01092F707109238
:10920000F60781E06E960FB6F894DEBF0FBECDBFB5
:10921000CF91DF911F910F91FF90EF900895909360
:10922000F7078093F6070E94B448089580914C0A8E
:1092300090914D0A1816190614F080E00895809157
:109240001B0C90911C0C20E630E0AC01429FC00149
:10925000439F900D529F900D1124835E934F0E9467
:109260003A48882311F481E0089580911B0C909175
:109270001C0C019690931C0C80931B0C80914C0A43
:1092800090914D0A019790934D0A80934C0A81E08A
:1092900008952F923F924F925F926F927F928F929A
:1092A0009F92AF92BF92CF92DF92EF92FF920F9375
:1092B0001F93DF93CF93CDB7DEB76E970FB6F894B9
:1092C000DEBF0FBECDBF0E94B448882309F415C28B
:1092D000F5C32D3071F02A3321F480910F0C8823CF
:1092E00041F08091100C9091110C8F3591050CF488
:1092F000DFC1E091100CF091110C309709F417C305
:10930000A091120CB091130CAA9D7001AB9DF00CB2
:10931000BA9DF00C1124EE0DFF1DE257F54F10829F
:1093200080910F0C882309F0BEC110920F0CAC572E
:10933000B54F1C9287010257154FC8016EE470E0CB
:109340000E94C5249C01009709F4F7C090938D0AF0
:1093500080938C0A2F5F3F4F201B310B2E0D3F1D3A
:10936000C9018257954F60E070E04AE050E00E94EA
:1093700034236093140C7093150C8093160C909307
:10938000170CC090510AD090520AE090530AF09006
:10939000540AA70196012F5F3F4F4F4F5F4F62174F
:1093A00073078407950709F46AC38091120C9091A2
:1093B000130C9C012A9DC0012B9D900D3A9D900D90
:1093C00011248257954F64E779E00E948A24892B03
:1093D00009F055C3EDE1F5E0949108C08091C0001B
:1093E00085FFFCCF9093C600319694919923B1F7F5
:1093F000E1E4F9E0949108C08091C00085FFFCCFC2
:109400009093C600319694919923B1F78CE095E042
:10941000B701A6012AE030E00E94AF3E8091C00073
:1094200085FFFCCF73C0FE264F5FFC01E40FF11DEA
:10943000E257F54FE081EA32B1F730938D0A20937D
:109440008C0AC901019660E070E00E94D4210E945C
:10945000A4D72F2D30E02617370709F45DC0EDE1C2
:10946000F5E0949108C08091C00085FFFCCF9093F7
:10947000C600319694919923B1F7E2E2F9E0949114
:1094800008C08091C00085FFFCCF9093C600319644
:1094900094919923B1F74091510A5091520A6091E9
:1094A000530A7091540A8CE095E02AE030E00E9463
:1094B000AF3E8091C00085FFFCCF28C0EDE1F5E014
:1094C000949108C08091C00085FFFCCF9093C600A6
:1094D000319694919923B1F7E8EFF8E0949108C0A0
:1094E0008091C00085FFFCCF9093C6003196949187
:1094F0009923B1F78CE095E0B701A6012AE030E0AE
:109500000E94AF3E8091C00085FFFCCF8AE080932F
:10951000C6000E9452434AC08091140C9091150CD1
:10952000A091160CB091170C8093510A9093520A97
:10953000A093530AB093540A3EC0C8016AE270E097
:109540000E94C524009709F436C0EDE1F5E094913E
:1095500008C08091C00085FFFCCF9093C600319673
:1095600094919923B1F7EEECF8E0949108C08091C2
:10957000C00085FFFCCF9093C6003196949199234B
:10958000B1F74091510A5091520A6091530A70917B
:10959000540A8CE095E02AE030E00E94AF3E8091D2
:1095A000C00085FFFCCF8AE08093C6001092110CAA
:1095B0001092100C83C28091120C9091130C8A9D12
:1095C00070018B9DF00C9A9DF00C112487010257BD
:1095D000154FC80167E470E00E94C5249C01009704
:1095E00009F44BC090938D0A80938C0A2F5F3F4FF4
:1095F000201B310B2E0D3F1DC9018257954F60E096
:1096000070E00E94D4210E94A4D764307105A8F5AF
:109610008091F8078823C9F480910D05882369F5A6
:10962000992DEBECF8E008C08091C00085FFFCCFDD
:109630009093C600319694919923B1F78091C00020
:1096400085FFFCCF7092C60018C0982DE5E5F8E0C4
:1096500008C08091C00085FFFCCF9093C600319672
:1096600094919923B1F78091C00085FFFCCF70924F
:10967000C6008BE498E00E9425C18091120C909165
:10968000130C019664E070E00E941ADB9093130CB7
:109690008093120C8091180C9091190C0196909364
:1096A000190C8093180C1092110C1092100C32C0EF
:1096B0002B3311F460920F0C80910F0C882351F51D
:1096C0002091100C3091110C8091120C9091130C80
:1096D0008A9DF0018B9DF00D9A9DF00D1124E20FF3
:1096E000F31FE257F54F80910E0C80832F5F3F4FA1
:1096F0003093110C2093100C0DC0A0E6AA2EB12CB3
:10970000E5E5F8E08490FAE07F2EEBECF8E0949049
:1097100066246394809108059091090520910A05BB
:1097200030910B05821B930B8F779070892B09F476
:10973000C0C18091180C9091190C04970CF0B9C11C
:109740008CE095E00E94BD3D282F80930E0C8A305E
:1097500009F0BFCDCECD8091100C9091110C892BCA
:1097600009F0ACC10E941649882309F0A7C1809175
:10977000180C9091190C892B09F02FC110921A0C1A
:109780002CC14D3099F0433211F04A3321F48091CD
:109790000F0C882359F08091100C9091110C8F358B
:1097A000910524F42F5F3F4F09F0F2C02091AF07DD
:1097B0003091B0074091B1075091B2078091A7074F
:1097C0009091A807A091A907B091AA072817390777
:1097D0004A075B0708F49EC0932DE8E3F8E008C051
:1097E0008091C00085FFFCCF9093C6003196949184
:1097F0009923B1F78091C00085FFFCCF2092C6006D
:109800000E9469D06093F2077093F3078093F40786
:109810009093F5072091EE073091EF074091F00704
:109820005091F107621B730B840B950B28EE33E00C
:1098300040E050E00E942DDBF22EE32ED42EC52E08
:10984000EDB7FEB738970FB6F894FEBF0FBEEDBF69
:109850000DB71EB70F5F1F4FB282A182F80153826E
:109860004282622F732F842F952F20E13EE040E04B
:1098700050E00E942DDBF801358324836F2D7E2D6F
:109880008D2D9C2D2CE330E040E050E00E942DDB3C
:10989000CA01B9012CE330E040E050E00E942DDB2A
:1098A000F801778366830E94F424982DE7E1F5E0C0
:1098B0002DB73EB7285F3F4F0FB6F8943EBF0FBE9F
:1098C0002DBF08C08091C00085FFFCCF9093C600DB
:1098D000319694919923B1F7F50107C08091C000AA
:1098E00085FFFCCF31969093C60090819923B1F704
:1098F0008091C00085FFFCCF2092C600C5010E9468
:1099000048C18DE095E00E9413328DE095E061E062
:109910000E94A43380910E0C833211F490921A0CA1
:109920002091100C3091110C2115310519F4109271
:109930000F0CC4C08091120C9091130C869DF00105
:10994000879DF00D969DF00D1124E20FF31FE25755
:10995000F54F1082FC01EC57F54F90822091180CC6
:109960003091190C2F5F3F4F3093190C2093180C36
:10997000019664E070E00E941ADB9093130C8093D0
:10998000120C10920F0C1092110C1092100C3AC085
:109990004B3311F490920F0C80910F0C882391F5AA
:1099A0002091100C3091110C8091120C9091130C9D
:1099B000869DF001879DF00D969DF00D1124E20F1C
:1099C000F31FE257F54F80910E0C80832F5F3F4FBE
:1099D0003093110C2093100C15C0E0E66E2E712C04
:1099E00099249394E8E3F8E034907AE0272E5E011E
:1099F0000894A11CB11C64E2462E68E0562EE7E1F3
:109A0000F5E084902091AF073091B0074091B10705
:109A10005091B2078091A7079091A807A091A9073C
:109A2000B091AA07281739074A075B0708F046C014
:109A30008091180C9091190C04970CF03FC0809104
:109A40001A0C8823D9F58091E3069091E406A09141
:109A5000E506B091E6068093AF079093B007A09318
:109A6000B107B093B2078BED96E00E94DC849C01B5
:109A7000482F80930E0C8A3009F083CE97CE8091C8
:109A8000120C9091130C8A9D80018B9D100D9A9D54
:109A9000100D1124C8018257954F6AE270E00E94B0
:109AA000C5249C01009709F409CDFF2440E0C801BA
:109AB000BCCC80910F05882309F04DCE6E960FB671
:109AC000F894DEBF0FBECDBFCF91DF911F910F91F4
:109AD000FF90EF90DF90CF90BF90AF909F908F90CE
:109AE0007F906F905F904F903F902F900895AF922E
:109AF000BF92CF92DF92EF92FF920F931F93DF936B
:109B0000CF93CDB7DEB7C055D0400FB6F894DEBFC7
:109B10000FBECDBF8FE492E0EDEFF7E0DF019C01D7
:109B20001D9221503040E1F780E693E0EDE1FCE04A
:109B3000DF019C011D9221503040E1F7809110051A
:109B4000882321F48DE095E00E94C43280911005B5
:109B5000882309F459C3E7EBF1E007C08091C00006
:109B600085FFFCCF31969093C60090819923B1F781
:109B70008091C00085FFFCCF8AE08093C600E2EDB3
:109B8000F1E007C08091C00085FFFCCF3196909333
:109B9000C60090819923B1F78091C00085FFFCCF6A
:109BA0008AE08093C6008CE095E06FE472E04AE0C2
:109BB00050E00E948C3E8091C00085FFFCCF8AE07F
:109BC0008093C6008BE39AE062EB7AE04FE050E0CE
:109BD0000E947B248DE095E06BE37AE00E940C2BE1
:109BE000882309F411C38DE095E06BE37AE041E04E
:109BF0000E94172B8DE095E06DEF77E04FE452E087
:109C00000E94EF318DE095E00E94322AE9EDF1E00B
:109C100007C08091C00085FFFCCF31969093C600AD
:109C200090819923B1F78091C00085FFFCCF8AE035
:109C30008093C6004091FD0750E060E070E08CE04A
:109C400095E02AE030E00E947F3E8091C00085FFD1
:109C5000FCCF8AE08093C60040914B0A50E060E060
:109C600070E08CE095E02AE030E00E947F3E809139
:109C7000C00085FFFCCF8AE08093C6009091FD076D
:109C8000992309F4AFC280914B0A981709F0A2C238
:109C90001598E6EEF1E007C08091C00085FFFCCF8B
:109CA00031969093C60090819923B1F78091C000BE
:109CB00085FFFCCF8AE08093C6000EEF17E02AE014
:109CC000F22ED8014D915D916D917C918CE095E0E3
:109CD00022E030E00E94BF3F8091C00085FFFCCFB2
:109CE000F092C6000C5F1F4FB8E00E301B0749F71B
:109CF000F80140815181628173818CE095E022E01E
:109D000030E00E94BF3F8091C00085FFFCCF8AE019
:109D10008093C60006E118E09AE0F92ED8016D9113
:109D20007C918CE095E04AE050E00E94E43E809116
:109D3000C00085FFFCCFF092C6000E5F1F4FB8E059
:109D40000E311B0759F7F801608171818CE095E0B5
:109D50004AE050E00E94E43E8091C00085FFFCCFC5
:109D60008AE08093C600EDE0F2E007C08091C00079
:109D700085FFFCCF31969093C60090819923B1F76F
:109D80008091C00085FFFCCF8AE08093C60060917F
:109D90002008709121088CE095E04AE050E00E9494
:109DA000E43E8091C00085FFFCCF8AE08093C6002E
:109DB00060912208709123088CE095E04AE050E021
:109DC0000E94E43E8091C00085FFFCCF8AE0809332
:109DD000C60060912408709125088CE095E04AE067
:109DE00050E00E94E43E8091C00085FFFCCF8AE0F5
:109DF0008093C60020E030E040E650E06AE0249F17
:109E0000F001259FF00D349FF00D1124EA5DF74F0E
:109E100007C08091C00085FFFCCF31969093C600AB
:109E200090819923B1F78091C00085FFFCCF6093AA
:109E3000C6002F5F3F4F2430310509F781E2E82E3D
:109E4000F12CEC0EFD1E80E1D701E82F1D92EA9562
:109E5000E9F7D701E82F1D92EA95E9F7D701E82F36
:109E60001D92EA95E9F701E3C02ED12CCC0EDD1E40
:109E7000D601E82F1D92EA95E9F711E4A12EB12C45
:109E8000AC0EBD1ED5011D928A95E9F76091FE07C3
:109E90007091FF07809100089091010841E023E054
:109EA0008E010F5F1F4F0E94522160910208709136
:109EB0000308809104089091050841E023E08E0199
:109EC0000F5E1F4F0E945221609106087091070893
:109ED000809108089091090841E023E087010E94E1
:109EE00052216091060870910708809108089091AE
:109EF000090820E030E040EA50E40E945CD641E0EE
:109F000023E085010E94522160910A0870910B089C
:109F100080910C0890910D0841E023E086010E9499
:109F20005221EDB7FEB738970FB6F894FEBF0FBEBB
:109F3000EDBF31968DE19CE0ADB7BEB712969C9314
:109F40008E93119786EA9AE093838283F582E48266
:109F5000D782C6820E94F4240F900F90EDB7FEB70F
:109F600031968DE79CE0ADB7BEB712969C938E9369
:109F700011978FE99AE093838283B582A4820E942D
:109F8000F4240F900F908DED9CE0EDB7FEB7928317
:109F9000818385E99AE0948383830E94F42400D02E
:109FA000EDB7FEB731968DE39DE0ADB7BEB7129623
:109FB0009C938E9311978EE89AE093838283F58227
:109FC000E4820E94F4240F900F908DE99DE0EDB79C
:109FD000FEB7928381838DE79AE0948383830E9406
:109FE000F42485E090E090934D0A80934C0A05E0BC
:109FF00010E00F900F900F900F90B0E6EB2EF12C29
:10A0000039C00E9DC0010F9D900D1E9D900D112415
:10A010000F5F1F4F20912008309121082E9DB00125
:10A020002F9D700D3E9D700D11246A5D774F835EEC
:10A03000934F0E94D02480914C0A90914D0A019632
:10A0400090934D0A80934C0A8091240890912508A2
:10A05000019790932508809324088091200890917F
:10A060002108019664E070E00E941ADB90932108B9
:10A0700080932008809124089091250818161906CD
:10A080000CF4BFCF40914C0A50914D0A20E030E0D3
:10A0900060E670E0AAE01CC0269FF001279FF00D4B
:10A0A000369FF00D1124E35EF34F07C08091C0008E
:10A0B00085FFFCCF31969093C60090819923B1F72C
:10A0C0008091C00085FFFCCFA093C6002F5F3F4F5B
:10A0D000241735070CF3E2E2F2E007C08091C000DC
:10A0E00085FFFCCF31969093C60090819923B1F7FC
:10A0F0008091C00085FFFCCF8AE08093C60040912C
:10A10000AA095091AB096091AC097091AD098CE03E
:10A1100095E02AE030E00E947F3E8091C00085FFFC
:10A12000FCCF8AE08093C600EEEAF9E007C0809198
:10A13000C00085FFFCCF31969093C6009081992393
:10A14000B1F78091C00085FFFCCF8AE08093C60004
:10A150004091A6095091A7096091A8097091A90999
:10A160008CE095E02AE030E00E947F3E8091C000C4
:10A1700085FFFCCF8AE08093C6008091AA09909168
:10A18000AB09A091AC09B091AD098093EE07909313
:10A19000EF07A093F007B093F1078DE095E06EEA2A
:10A1A00079E041E021E00E94602E4091A6095091A3
:10A1B000A7096091A8097091A9094093AF0750932E
:10A1C000B0076093B1077093B2078BED96E00E94E1
:10A1D00017811AC08AE69AE09093F7078093F607F2
:10A1E0000E94B4488FE492E0EDEFF7E0DF019C01BC
:10A1F0001D9221503040E1F78BE39AE066E67AE069
:10A200004FE050E00E947B24C05BDF4F0FB6F89414
:10A21000DEBF0FBECDBFCF91DF911F910F91FF9099
:10A22000EF90DF90CF90BF90AF9008952F923F9224
:10A230004F925F926F927F928F929F92AF92BF9256
:10A24000CF92DF92EF92FF920F931F93DF93CF9302
:10A25000CDB7DEB7EE970FB6F894DEBF0FBECDBF19
:10A2600087E40E948043882309F42FC20E94AF45EF
:10A270000E94A4D76430710509F441C065307105AE
:10A2800054F46230710541F1633071056CF5772348
:10A29000CCF40C94F6656A35710509F4BBC16B35D5
:10A2A000710534F46C31710511F00C94F6656FC0D2
:10A2B0006B35710509F4B2C16C35710511F00C9460
:10A2C000F665B1C18091F807882331F40E943946C0
:10A2D0000E9490420C9404668091F807882321F430
:10A2E0000E94BA4681E007C08091F807882339F4BC
:10A2F0000E94BA4680E00E94D2410C9404668BED25
:10A3000097E00E9425C180E50E948043882321F4C4
:10A31000EE24FF24870106C00E94AF450E94A9D702
:10A320007B018C0183E50E948043882361F00E94B9
:10A33000AF4520E030E04AE754E40E9415DA0E947D
:10A34000A9D77B018C010E94EB910E9469D05B012F
:10A350006C01AE0CBF1CC01ED11E0E9469D0609360
:10A36000590A70935A0A80935B0A90935C0A06C05C
:10A370000E94D59D0E946E410E946AC10E9469D0D0
:10A380006A157B058C059D0598F30C94F665809104
:10A390009E0390919F03A091A003B091A10380938D
:10A3A000880A9093890AA0938A0AB0938B0A8091B5
:10A3B0007203909173039093BF078093BE0784E666
:10A3C00090E090937303809372030E9469D060932E
:10A3D000590A70935A0A80935B0A90935C0A81E051
:10A3E0000E9410918091C0079091C107A091C2076F
:10A3F000B091C30780936D0A90936E0AA0936F0A81
:10A40000B093700A8091C4079091C507A091C607C8
:10A41000B091C7078093710A9093720AA093730A50
:10A42000B093740A8091C8079091C907A091CA0798
:10A43000B091CB078093750A9093760AA093770A20
:10A44000B093780A8091CC079091CD07A091CE0768
:10A45000B091CF078093790A90937A0AA0937B0AF0
:10A46000B0937C0A80E090E0A0E0B0E080939E038F
:10A4700090939F03A093A003B093A10388E50E944B
:10A480008043882361F489E50E948043882339F45E
:10A490008AE50E948043882311F481E001C080E0B6
:10A4A0008093A203882329F488E50E9480438823AF
:10A4B00021F080E090E00E94B5438091A2038823C0
:10A4C00029F489E50E948043882321F081E090E00F
:10A4D0000E94B54388E50E9480438823D9F00E94FA
:10A4E000A3456115710581059105A1F00E94AF4555
:10A4F0002091D0073091D1074091D2075091D307D6
:10A500000E945CD66093C0077093C1078093C20716
:10A510009093C30789E50E9480438823D9F00E9465
:10A52000A3456115710581059105A1F00E94AF4514
:10A530002091D4073091D5074091D6075091D70785
:10A540000E945CD66093C4077093C5078093C607CA
:10A550009093C7078091A203882329F48AE50E947B
:10A560008043882321F082E090E00E94B5438AE591
:10A570000E9480438823D9F00E94A345611571058C
:10A5800081059105A1F00E94AF452091D807309137
:10A59000D9074091DA075091DB070E945CD660939F
:10A5A000C8077093C9078093CA079093CB0780ECC4
:10A5B00097E064EC77E048EC57E02CEC37E00E9441
:10A5C0004D6D80E00E9410918091880A9091890AD7
:10A5D000A0918A0AB0918B0A80939E0390939F0367
:10A5E000A093A003B093A1038091BE079091BF07F1
:10A5F00090937303809372030E9469D06093590A09
:10A6000070935A0A80935B0A90935C0A0E940991A6
:10A610000C94F66510927D0A0C94F66581E08093A7
:10A620007D0A0C94F66585E40E948043882311F42A
:10A630000E94EB9150ECE52E57E0F52E40EDC42E34
:10A6400047E0D42E00E010E0BB24B394F801EF5DA6
:10A65000FB4F80810E948043882351F1033061F4D5
:10A660000E94AF45F70160837183828393838CECF2
:10A6700097E00E942F6D1CC0023011F4B092EA07DF
:10A680000E94AF45F60120813181428153810E94B1
:10A690005CD6F701608371838283938380EC97E0BB
:10A6A00064EC77E048EC57E02CEC37E00E944D6D0D
:10A6B0000F5F1F4F24E030E0E20EF31EC20ED31EE8
:10A6C0000430110519F60C94F6658DE40E94804360
:10A6D000882311F40C9418650E94AF450E94A4D7FA
:10A6E0006237710511F40C94315D633771050CF01C
:10A6F0009BC06E31710509F492C26F3171050CF087
:10A7000042C06631710509F4ECC167317105E4F4AA
:10A710006131710509F4A3C16231710534F462300D
:10A72000710510F00C94F6653BC16431710509F4B4
:10A73000A0C1653171050CF0CCC16231710511F019
:10A740000C94F6650C941A5C6931710509F4FFC12B
:10A750006A31710554F46731710509F4C8C1683173
:10A76000710511F00C94F665DEC16B31710509F4C9
:10A7700013C26B3171050CF4F0C16C31710511F02D
:10A780000C94F6650FC26435710511F40C941A5CD3
:10A790006535710514F56A32710509F4E0C36B3251
:10A7A000710554F46F31710509F42AC360327105E3
:10A7B00011F00C94F66579C26235710511F40C94B0
:10A7C000115C6335710514F00C94155C61357105ED
:10A7D00011F00C94F6650C94F65B6936710509F47A
:10A7E00039C46A36710584F46C35710511F40C9422
:10A7F000845C6836710509F4FCC36535710511F098
:10A800000C94F6650C946D5C6B36710511F40C9428
:10A81000F05B6B36710514F40C94BF5B6D367105FB
:10A8200011F00C94F6653AC56C3D710511F40C9469
:10A830001B606D3D71050CF04FC06E3B710509F456
:10A840008BC66F3B71051CF56737710509F4A4C011
:10A850006837710564F46337710511F40C940A5D6F
:10A860006537710511F00C94F6650C941A5D693723
:10A87000710511F40C942B5E6937710514F40C9476
:10A88000265E6C38710511F00C94F665D2C36B3CF2
:10A89000710511F40C94615F6C3C710564F4683CC3
:10A8A000710511F40C94B75E693C710511F00C94BC
:10A8B000F6650C943F5F6D3C710511F40C949F5F3D
:10A8C0006D3C710514F40C947F5F6E3C710511F0C2
:10A8D0000C94F6650C94FD5F31E06F32730711F450
:10A8E0000C94896241E0603374073CF56A3F71055E
:10A8F00011F40C944E626B3F710564F46D3D71056B
:10A9000011F40C942A60623E710511F00C94F66506
:10A910000C94396051E06C32750711F40C943F616E
:10A9200081E06D32780711F40C94766168517140C2
:10A9300011F00C94F6650C949160E1E0673F7E079E
:10A9400011F40C94D462F1E0683F7F079CF421E09D
:10A95000653F720711F40C94CC6231E0663F7307D7
:10A9600014F00C94D1626059714011F00C94F665AA
:10A970000C94C96253E0603A750709F406C283E09B
:10A98000673E780711F40C9401656855724011F028
:10A990000C94F6650C94D762E9E4F2E00C94375E0F
:10A9A0008AEC97E00E9425C180E50E9480438823BD
:10A9B00021F4EE24FF24870106C00E94AF450E94C7
:10A9C000A9D77B018C0183E50E948043882361F035
:10A9D0000E94AF4520E030E04AE754E40E9415DAD7
:10A9E0000E94A9D77B018C010E94EB910E9469D043
:10A9F0006093590A70935A0A80935B0A90935C0A99
:10AA0000E114F1040105110501F10E9469D05B0117
:10AA10006C01AE0CBF1CC01ED11E0E9469D06A150D
:10AA20007B058C059D05A8F40E9430A4882389F439
:10AA30000E94D59D0E946E410E946AC1EECF0E9485
:10AA4000D59D0E946E410E946AC10E9430A4882355
:10AA5000B1F380EC97E00E9425C10C94F66587EB7A
:10AA600097E00E9425C15E985E9815985E980C94B8
:10AA7000F665E7EAF7E0949108C08091C00085FF91
:10AA8000FCCF9093C600319694919923B1F78091B1
:10AA9000C00085FFFCCF8AE08093C6008DE095E082
:10AAA0000E947337E9E9F7E0949108C08091C000F3
:10AAB00085FFFCCF9093C600319694919923B1F70E
:10AAC0008091C00085FFFCCF8AE08093C6000C9483
:10AAD000F6658DE095E00E94C4320E94774D0C949B
:10AAE000F6658DE095E00E94CF290C94F665809183
:10AAF0008C0A90918D0A04966AE270E00E94C52447
:10AB0000FC01009711F03197108260918C0A7091CE
:10AB10008D0A6C5F7F4F8DE095E041E021E00E945F
:10AB2000602E0C94F6658DE095E00E94E42D8DE09A
:10AB300095E00E94D3290E9469D06093EE0770933C
:10AB4000EF078093F0079093F1070C94F6658DE082
:10AB500095E00E94DA290C94F6658091100588230F
:10AB600011F40C94F66583E50E948043882311F468
:10AB70000C94F6650E94A345AB01BC014093AF075E
:10AB80005093B0078093B1077093B2078BED96E0B6
:10AB90000E9417810C94F6658DE095E00E94182CB8
:10ABA0000C94F66580918C0A90918D0A04966AE265
:10ABB00070E00E94C5248C01009719F12091820A4F
:10ABC0003091830A80E690E0FC012E9FC0012F9F08
:10ABD000900D3E9F900D11248257954F6EE470E0CA
:10ABE0000E94C52460E270E00E94C5249C012F5F92
:10ABF0003F4F30938D0A20938C0A01501040F8018A
:10AC0000108260918C0A70918D0A6C5F7F4F8DE08D
:10AC100095E040E021E00E94602E0C94F665809162
:10AC20001005882311F40C94F6658DE095E060E042
:10AC30000E94872B80918C0A90918D0A04966AE27B
:10AC400070E00E94C5248C01009719F12091820ABE
:10AC50003091830A80E690E0AC01249FC001259FDB
:10AC6000900D349F900D11248257954F6EE470E043
:10AC70000E94C52460E270E00E94C5249C012F5F01
:10AC80003F4F30938D0A20938C0A01501040F801F9
:10AC9000108260918C0A70918D0A6C5F7F4F8DE0FD
:10ACA00095E00E94722C0C94F66580910F05882324
:10ACB00011F00E94EB91E0908C0AF0908D0A24E054
:10ACC00030E0E20EF31EC7016AE270E00E94C52484
:10ACD0008C01C70161E270E00E94C524009721F059
:10ACE0007C010894E11CF11C0115110521F00150B3
:10ACF0001040F801108280E50E948043182F809157
:10AD00008C0A90918D0AE816F90608F410E08091FB
:10AD10001005882311F40C94F66521E021278DE0BD
:10AD200095E0B70141E00E94602E83E50E948043D8
:10AD30008823B9F080918C0A90918D0A8E159F0519
:10AD400080F40E94A345AB01BC014093AF07509330
:10AD5000B0078093B1077093B2078BED96E00E9425
:10AD600017818DE095E00E94D329112311F00C94F6
:10AD7000F6650E9469D06093EE077093EF078093A9
:10AD8000F0079093F1070C94F66580918C0A9091EE
:10AD90008D0A05966AE270E00E94C5248C01009736
:10ADA00019F12091820A3091830A80E690E0AC018B
:10ADB000249FC001259F900D349F900D1124825730
:10ADC000954F6EE470E00E94C52460E270E00E943E
:10ADD000C5249C012F5F3F4F30938D0A20938C0A2E
:10ADE00001501040F801108260918C0A70918D0A18
:10ADF0006B5F7F4F8DE095E00E94E6310C94F66525
:10AE00000E9469D06093F2077093F3078093F40770
:10AE10009093F5072091EE073091EF074091F007EE
:10AE20005091F107621B730B840B950B28EE33E0F6
:10AE300040E050E00E942DDBF22EE32ED42EC52EF2
:10AE40002DB73EB7285030400FB6F8943EBF0FBE26
:10AE50002DBF0DB71EB70F5F1F4FCE018196EDB707
:10AE6000FEB7928381838AE897E0F8019383828317
:10AE70006F2D7E2D842F952F2CE330E040E050E0A5
:10AE80000E942DDBF801358324836F2D7E2D8D2DBF
:10AE90009C2D2CE330E040E050E00E942DDBF801D7
:10AEA000778366830E94F424E7E1F5E094912DB75F
:10AEB0003EB7285F3F4F0FB6F8943EBF0FBE2DBF81
:10AEC00008C08091C00085FFFCCF9093C6003196EA
:10AED00094919923B1F7FE01B19607C08091C0000B
:10AEE00085FFFCCF31969093C60090819923B1F7EE
:10AEF0008091C00085FFFCCF8AE08093C600CE0120
:10AF000081960E9448C18091ED0F882311F40C9422
:10AF1000F6651092ED0F8091EB07082F10E0000FFF
:10AF2000111F0D5A184EF80160817181882777FD35
:10AF30008095982F0E94D7D72091A7033091A8031E
:10AF40004091A9035091AA030E9443D9181614F006
:10AF50000C94F665F801118210820C94F66583E575
:10AF60000E948043882311F40C94F6650E94AF453B
:10AF70000E94A4D77B018C016B0180E50E94804375
:10AF8000882369F0F7FC0BC0FFEFEF16F10409F01E
:10AF900034F40E94AF450E94A4D78B0102C00FEF8A
:10AFA0001FEFE5E2F4E0808191818017910711F4B1
:10AFB0000C94F665329624E0E539F207A1F70430E7
:10AFC000110529F4D092ED07C092EC0704C017FFD9
:10AFD00002C00C94F665802F61E00E9496D1802F0C
:10AFE0006C2D0E9413D2802FB6010E9418D10C94B0
:10AFF000F66588E690E00E94B945882311F00C942C
:10B00000F66583E50E948043882379F00E94AF456E
:10B010002091500A022F10E0000F111F0D5A184EF8
:10B020000E94A4D7F801718360830E94CA990C948E
:10B03000F66583E50E948043882311F40C94F6653D
:10B040000E94AF450E94A4D770935617609355177E
:10B050000C94F66589E690E00E94B945882311F0CA
:10B060000C94F665E4E8F7E0949108C08091C00084
:10B0700085FFFCCF9093C600319694919923B1F748
:10B08000E091500AF0E0EE0FFF1FEE0FFF1FE75AAE
:10B09000F84E40815181628173818CE095E021E01E
:10B0A00030E00E94BF3FE1E8F7E0949108C0809152
:10B0B000C00085FFFCCF9093C600319694919923F0
:10B0C000B1F7E091500AF0E0EE0FFF1FED5AF84E95
:10B0D00060817181882777FD8095982F0E94D7D74E
:10B0E000AB01BC018CE095E021E030E00E94BF3F65
:10B0F000EDE7F7E0949108C08091C00085FFFCCF98
:10B100009093C600319694919923B1F740915F17BF
:10B110005091601760916117709162178CE095E013
:10B1200021E030E00E94BF3FEAE7F7E0949108C0D9
:10B130008091C00085FFFCCF9093C600319694911A
:10B140009923B1F76091551770915617882777FDAD
:10B150008095982F0E94D7D7AB01BC018CE095E079
:10B1600021E030E00E94BF3FE7E7F7E0949108C09C
:10B170008091C00085FFFCCF9093C60031969491DA
:10B180009923B1F78CE095E060E070E04AE050E090
:10B190000E94E43EE5E7F7E0949108C08091C0008A
:10B1A00085FFFCCF9093C600319694919923B1F717
:10B1B0004091591750915A1760915B1770915C1725
:10B1C0008CE095E021E030E00E94BF3FE2E7F7E04D
:10B1D000949108C08091C00085FFFCCF9093C60079
:10B1E000319694919923B1F7609153177091541748
:10B1F000882777FD8095982F0E94D7D7AB01BC0197
:10B200008CE095E021E030E00E94BF3FEEE6F7E001
:10B21000949108C08091C00085FFFCCF9093C60038
:10B22000319694919923B1F78091500A0E940F9919
:10B23000BC018CE095E04AE050E00E94E43EE9E683
:10B24000F7E0949108C08091C00085FFFCCF9093F7
:10B25000C600319694919923B1F78FEF9FEF0E942A
:10B260000F99BC018CE095E04AE050E00E94E43E7A
:10B27000E2E6F2E007C08091C00085FFFCCF319686
:10B280009093C60090819923B1F78091C00085FF0B
:10B29000FCCF8AE08093C6000C9404668DE690E0B3
:10B2A0000E94B945882311F00C94F6658EE597E06D
:10B2B0000E9425C11092ED0F83E50E9480438823F0
:10B2C00099F00E94AF452091500A022F10E0000F24
:10B2D000111F0D5A184E0E94A4D7F8017183608384
:10B2E00081E08093990316C082E50E948043882301
:10B2F00089F00E94AF452091500A022F10E0000F04
:10B30000111F0D5A184E0E94A4D7F8017183608353
:10B310001092990383E50E948043882351F00E9494
:10B32000AF456093A7037093A8038093A9039093FC
:10B33000AA0382E40E948043882351F00E94AF4513
:10B340006093A3037093A4038093A5039093A60333
:10B3500086E40E948043882369F00E94AF45609391
:10B36000AB037093AC038093AD039093AE0381E085
:10B370008093ED0F0E94CA990E9469D06B017C01F5
:10B380002091500A022F10E01092FC07000F111FAD
:10B39000F801ED5AF84E60817181882777FD80951C
:10B3A000982F0E94D7D7000F111F075A184EF80187
:10B3B00020813181428153810E9443D918160CF0BB
:10B3C00066C081E08093FC0762C00E9469D06C195E
:10B3D0007D098E099F09695E73408040904008F4A2
:10B3E0004FC09A2DEBE5F7E008C08091C00085FFC3
:10B3F000FCCF9093C600319694919923B1F7E091D8
:10B40000500AF0E0EE0FFF1FEE0FFF1FE75AF84E55
:10B4100040815181628173818CE095E021E030E0D0
:10B420000E94BF3F9B2DE7E5F7E008C08091C00078
:10B4300085FFFCCF9093C600319694919923B1F784
:10B440006091500A8CE095E070E04AE050E00E9484
:10B45000E43EE2E6F2E007C08091C00085FFFCCF49
:10B4600031969093C60090819923B1F78091C000E6
:10B4700085FFFCCF9092C6000E9469D06B017C01D1
:10B480000E94D59D0E946E410E946AC108C0EBE5F2
:10B49000F7E0A490E7E5F7E0B4906AE0962E80919B
:10B4A000FC070091500A8823E9F010E0000F111FFB
:10B4B000F801ED5AF84E60817181882777FD8095FB
:10B4C000982F0E94D7D7000F111F075A184EF80166
:10B4D00020813181428153810E9443D918160CF496
:10B4E00074CF20C010E0000F111FF801ED5AF84E84
:10B4F00060817181882777FD8095982F0E94D7D72A
:10B50000000F111F075A184EF80120813181428126
:10B5100053810E9435D788232CF480919903882386
:10B5200009F453CF89E497E00E9425C10E9469D0B5
:10B530006093EE077093EF078093F0079093F10705
:10B540000E9469D06093590A70935A0A80935B0AEB
:10B5500090935C0A0C94F6658CE397E00E9425C1F9
:10B5600083E50E948043882361F00E94AF450E94DA
:10B57000A4D7709356176093551781E08093990371
:10B580000FC082E50E948043882351F00E94AF459E
:10B590000E94A4D770935617609355171092990381
:10B5A0000E9469D07B018C011092FC0760915517B5
:10B5B00070915617882777FD8095982F0E94D7D7CE
:10B5C00020915F1730916017409161175091621779
:10B5D0000E9443D918160CF082C081E08093FC07CA
:10B5E0007EC00E9469D06E197F09800B910B695E45
:10B5F00073408040904008F46BC0E091EB07F0E0AE
:10B60000EE0FFF1FEE0FFF1FE75AF84E40815181EA
:10B61000628173819B2DE9E3F7E008C08091C0004F
:10B6200085FFFCCF9093C600319694919923B1F792
:10B630008CE095E022E030E00E94BF3F9C2DE5E3E6
:10B64000F7E008C08091C00085FFFCCF9093C60052
:10B65000319694919923B1F76091EB078CE095E0D6
:10B6600070E04AE050E00E94E43E9D2DE1E3F7E007
:10B6700008C08091C00085FFFCCF9093C600319632
:10B6800094919923B1F740915F17509160176091A1
:10B690006117709162178CE095E021E030E00E9424
:10B6A000BF3FE2E6F2E007C08091C00085FFFCCF1B
:10B6B00031969093C60090819923B1F78091C00094
:10B6C00085FFFCCFA092C6000E9469D07B018C014F
:10B6D0000E94D59D0E946E410E946AC10BC0E9E3A1
:10B6E000F7E0B490E5E3F7E0C490E1E3F7E0D4904D
:10B6F000AAE0AA2E8091FC07209155173091561789
:10B700008823A9F0B901882777FD8095982F0E949A
:10B71000D7D720915F1730916017409161175091F2
:10B7200062170E9443D918160CF45BCF18C0B901F8
:10B73000882777FD8095982F0E94D7D720915F1793
:10B740003091601740916117509162170E9435D770
:10B7500088232CF480919903882309F442CF87E24F
:10B7600097E00E9425C10E9469D06093590A7093A6
:10B770005A0A80935B0A90935C0A0C94F66583E501
:10B780000E948043882321F10E94AF4520E030E0F1
:10B7900040E050E00E9435D788231CF460E070E060
:10B7A00011C00E94AF4520E030E04FE753E40E9413
:10B7B00043D918161CF46FEF70E004C00E94AF4527
:10B7C0000E94A4D77093ED076093EC070C94F66584
:10B7D0008FEF90E09093ED078093EC070C94F66563
:10B7E0001092ED071092EC070C94F6650E94CB992D
:10B7F0000E94EB915E9A0E94F9911092ED071092CF
:10B80000EC0768EE73E080E090E00E9477D0109241
:10B81000980384E197E00E9425C10E946AC10C94BC
:10B82000F6651092BD070C94F66581E08093BD0724
:10B830000C94F66583E50E9480438823A1F00E9462
:10B84000AF4520E030E04AE754E40E9415DA0E9458
:10B85000A9D760939A0370939B0380939C03909362
:10B860009D030C94F66588E50E948043882311F0BF
:10B870000C94F96589E50E948043882311F00C94AB
:10B88000F9658AE50E948043882311F00C94F965DC
:10B8900085E40E948043882311F00C94F9650E948E
:10B8A000EB915E9A0E94F9910C94F6655E9A109263
:10B8B000E80789E50E948043882319F05E9A109278
:10B8C000E9078AE50E948043882311F40C94F66509
:10B8D000159A1092EA070C94F66583E50E9480435E
:10B8E0000E94AF4520E030E04AE754E40E9415DAB8
:10B8F0000E94A9D760935D0A70935E0A80935F0AE5
:10B900009093600A0C94F665F1E96F2EFFE07F2EAC
:10B91000E1E82E2EEFE03E2E7DEC472E7FE0572E05
:10B9200088249924F401EF5DFB4F80810E948043BD
:10B93000882309F45DC023E0821609F052C00E94FA
:10B94000AF455B016C0120E030E040EA51E40E9429
:10B9500035D788230CF03FC0F3016081718182816B
:10B960009381A60195010E943CD77B018C016091D7
:10B97000C50F7091C60F8091C70F9091C80FA80195
:10B9800097010E9415DA6093C50F7093C60F8093DC
:10B99000C70F9093C80FF1016081718182819381FB
:10B9A000A80197010E9415DAF101608371838283F7
:10B9B0009383F20160817181828193810E94D5D746
:10B9C000A80197010E9415DA0E94A9D7F2016083AD
:10B9D000718382839383F301A082B182C282D38276
:10B9E00007C00E94AF45F301608371838283938314
:10B9F0000894811C911C24E030E0620E731E220E1C
:10BA0000331E420E531E34E08316910409F08ACF90
:10BA10000C94F665E7E4F6E0949108C08091C000CC
:10BA200085FFFCCF9093C600319694919923B1F78E
:10BA30000C94F66580918C0A90918D0A05966AE2C5
:10BA400070E00E94C524FC01009711F0319710822C
:10BA500080918C0A90918D0A05960E9448C10C94A1
:10BA6000F665E4E4F6E0949108C08091C00085FF9B
:10BA7000FCCF9093C600319694919923B1F74091F1
:10BA8000C0075091C1076091C2077091C3078CE055
:10BA900095E022E030E00E94BF3FE1E4F6E09491BF
:10BAA00008C08091C00085FFFCCF9093C6003196FE
:10BAB00094919923B1F74091C4075091C5076091C3
:10BAC000C6077091C7078CE095E022E030E00E9445
:10BAD000BF3FEEE3F6E0949108C08091C00085FF7F
:10BAE000FCCF9093C600319694919923B1F7409181
:10BAF000C8075091C9076091CA077091CB078CE0C5
:10BB000095E022E030E00E94BF3FEBE3F6E0949145
:10BB100008C08091C00085FFFCCF9093C60031968D
:10BB200094919923B1F74091CC075091CD07609142
:10BB3000CE077091CF078CE095E022E030E00E94C4
:10BB4000BF3FE0E3F6E0949108C08091C00085FF1C
:10BB5000FCCF9093C600319694919923B1F780E081
:10BB60000E94B6910E94D7D72091910F3091920FE9
:10BB70004091930F5091940F0E943CD7AB01BC01B0
:10BB80008CE095E022E030E00E94BF3FEDE2F6E07D
:10BB9000949108C08091C00085FFFCCF9093C600AF
:10BBA000319694919923B1F781E00E94B6910E9459
:10BBB000D7D72091950F3091960F4091970F5091C4
:10BBC000980F0E943CD7AB01BC018CE095E022E0CD
:10BBD00030E00E94BF3FEAE2F6E0949108C0809115
:10BBE000C00085FFFCCF9093C600319694919923B5
:10BBF000B1F782E00E94B6910E94D7D72091990FA9
:10BC000030919A0F40919B0F50919C0F0E943CD70E
:10BC1000AB01BC018CE095E022E030E00E94BF3F28
:10BC2000E2E6F2E007C08091C00085FFFCCF3196CC
:10BC30009093C60090819923B1F78091C00085FF51
:10BC4000FCCF8AE08093C6000C94F66580E00E94E9
:10BC500010910C94F66581E00E9410910C94F665A9
:10BC60008091C00085FFFCCF31969093C6009081F3
:10BC70009923B1F78091C00085FFFCCF8AE08093C3
:10BC8000C600E2E2F6E0949108C08091C00085FF12
:10BC9000FCCF9093C600319694919923B1F73299D5
:10BCA00003C0E3E6F2E00AC0E8E6F2E007C08091F4
:10BCB000C00085FFFCCF31969093C60090819923F8
:10BCC000B1F78091C00085FFFCCF8AE08093C60069
:10BCD000EAE1F6E0949108C08091C00085FFFCCFB6
:10BCE0009093C600319694919923B1F7339903C08C
:10BCF000E3E6F2E00AC0E8E6F2E007C08091C000A7
:10BD000085FFFCCF31969093C60090819923B1F7BF
:10BD10008091C00085FFFCCF8AE08093C600E2E1FD
:10BD2000F6E0949108C08091C00085FFFCCF90930D
:10BD3000C600319694919923B1F7349903C0E3E694
:10BD4000F2E00AC0E8E6F2E007C08091C00085FF9B
:10BD5000FCCF31969093C60090819923B1F78091E2
:10BD6000C00085FFFCCF8AE08093C6003FC784E413
:10BD70000E948043882309F439C70E94AF4520E020
:10BD800030E040E05FE30E9415DA7B018C0120E0A7
:10BD900030E040E050E00E9435D7882359F40F2E60
:10BDA000F0E0CF2EF0E0DF2EF0E8EF2EFFE3FF2EE5
:10BDB000F02D11C0C801B701A80197010E9415DA42
:10BDC0009B01AC01CA012BED3FE049E450E40E9425
:10BDD00015DA6B017C018091EB078093500A84E5B2
:10BDE0000E948043882399F10E94AF450E94A9D701
:10BDF000262F6093500A6623D9F0E7E1F5E094918D
:10BE000008C08091C00085FFFCCF9093C60031969A
:10BE100094919923B1F7E2E7F2E007C08091C00066
:10BE200085FFFCCF31969093C60090819923B1F79E
:10BE30008CE095E0622F40E050E00E949D3E8091B2
:10BE4000C00085FFFCCF8AE08093C600CFC68091FA
:10BE5000500A082F10E0000F111F000F111F0A5881
:10BE60001C4F60E070E080E89FE3A70196010E940C
:10BE70003CD7F8016083718382839383B7C601E264
:10BE800014E051EAE52E5FE0F52EF80180810E9472
:10BE90008043882349F00E94AF450E94A9D7F7014B
:10BEA00060837183828393830F5F1F4F24E030E0B0
:10BEB000E20EF31E34E00532130739F70E94046DD9
:10BEC00095C601E214E041E8E42E4FE0F42EF801BB
:10BED00080810E948043882339F00E94AF45F7019A
:10BEE00060837183828393830F5F1F4F24E030E070
:10BEF000E20EF31E34E00532130749F777C683E5F7
:10BF00000E948043882351F00E94AF456093B50F93
:10BF10007093B60F8093B70F9093B80F84E50E948B
:10BF20008043882309F462C60E94AF456093B90F2D
:10BF30007093BA0F8093BB0F9093BC0F57C683E5E5
:10BF40000E948043882351F00E94AF456093B10F57
:10BF50007093B20F8093B30F9093B40F84E50E9457
:10BF60008043882351F00E94AF456093C90F7093BE
:10BF7000CA0F8093CB0F9093CC0F82E40E94804332
:10BF8000882361F00E94AF450E94A9D760937D0F7E
:10BF900070937E0F80937F0F9093800F88E50E94AF
:10BFA0008043882351F00E94AF456093BD0F70938A
:10BFB000BE0F8093BF0F9093C00F8AE50E9480430D
:10BFC000882351F00E94AF456093C10F7093C20F58
:10BFD0008093C30F9093C40F85E40E94804388230D
:10BFE00009F404C60E94AF456093C50F7093C60F55
:10BFF0008093C70F9093C80FF9C501E214E030EDAC
:10C00000E32E37E0F32EF80180810E9480438823DD
:10C0100039F00E94AF45F701608371838283938377
:10C020000F5F1F4F24E030E0E20EF31E34E00432D5
:10C03000130749F7DBC583E50E948043882309F491
:10C04000D5C50E94AF450E94A4D770937303609337
:10C050007203CCC583E50E948043882309F4C6C5DA
:10C060000E94AF450E94A4D7709375036093740338
:10C07000BDC580E50E948043882309F4B7C50E94AE
:10C08000AF450E94A4D77B0183E50E9480438823AB
:10C0900019F40FEF1FEF05C00E94AF450E94A4D70F
:10C0A0008B01C8010196039708F0A0C5E5E2F4E012
:10C0B000808191818E159F0509F498C5329644E0E0
:10C0C000E539F407A9F7F7FC91C50E94EB91DE2C46
:10C0D0008E2D60E00E9496D10115110541F00130CE
:10C0E000110579F05FEF0F3F1507A1F403C000E0E1
:10C0F00010E010C08E2D0E9446D200E010E0892B87
:10C1000049F401E010E006C00E94D59D0E946E41F6
:10C110000E946AC18D2D0E9446D280179107A1F717
:10C1200065C580E50E948043882319F40FEF1FEF57
:10C1300005C00E94AF450E94A4D78B0183E50E94F1
:10C140008043882309F446C00E94AF4501151105BC
:10C1500051F40E94A4D79B01AC0189EF97E0B9018B
:10C160000E94DF8F43C5E7E1F5E0949108C080911C
:10C17000C00085FFFCCF9093C6003196949199231F
:10C18000B1F7E9E8F2E007C08091C00085FFFCCF7D
:10C1900031969093C60090819923B1F78CE095E099
:10C1A000B8014AE050E00E94E43EE0E9F2E007C056
:10C1B0008091C00085FFFCCF31969093C60090819E
:10C1C0009923B1F78091C00085FFFCCF8AE080936E
:10C1D000C6000CC517FD0AC5EEE9F2E007C0809164
:10C1E000C00085FFFCCF31969093C60090819923C3
:10C1F000B1F7E1EAF2E007C08091C00085FFFCCF13
:10C2000031969093C60090819923B1F78CE095E028
:10C21000B8014AE050E00E94E43EE9EAF2E007C0DB
:10C220008091C00085FFFCCF31969093C60090812D
:10C230009923B1F7C801880F991F800F911F87506C
:10C24000984F0E948A8FBC018CE095E04AE050E054
:10C250000E94E43EE2E6F2E007C08091C00085FF64
:10C26000FCCF31969093C60090819923B1F78091CD
:10C27000C00085FFFCCF8AE08093C600B7C483E589
:10C280000E948043882321F4BEE6CB2ED12C05C02A
:10C290000E94AF450E94A4D76B0180E50E948043B5
:10C2A000882319F468EE73E004C00E94AF450E9431
:10C2B000A4D77B010027F7FC0095102F1C141D0448
:10C2C00084F48BE1B60120E030E040E050E00E94D1
:10C2D0006BD3C801B7010E9477D08BE10E94F4D2E2
:10C2E00085C4C801B7010E9477D080C480E50E9450
:10C2F0008043882351F00E94AF456093B40370934C
:10C30000B5038093B6039093B70389E40E948043FA
:10C31000882361F00E94AF450E94DA996093B803C8
:10C320007093B9038093BA039093BB0384E40E9493
:10C330008043882361F00E94AF450E94E899609392
:10C34000BC037093BD038093BE039093BF0383E44B
:10C350000E948043882351F00E94AF456093C00340
:10C360007093C1038093C2039093C3030E94F89813
:10C37000EEE9F2E007C08091C00085FFFCCF319666
:10C380009093C60090819923B1F7ECEAF2E007C0E0
:10C390008091C00085FFFCCF31969093C6009081BC
:10C3A0009923B1F74091B4035091B5036091B6035E
:10C3B0007091B7038CE095E022E030E00E94BF3F2F
:10C3C000E0EBF2E007C08091C00085FFFCCF319622
:10C3D0009093C60090819923B1F76091B803709152
:10C3E000B9038091BA039091BB030E94E199AB011C
:10C3F000BC018CE095E022E030E00E94BF3FE4EB1E
:10C40000F2E007C08091C00085FFFCCF3196909389
:10C41000C60090819923B1F76091BC037091BD0370
:10C420008091BE039091BF030E94EF99AB01BC01C4
:10C430008CE095E022E030E00E94BF3FE8EBF2E0C4
:10C4400007C08091C00085FFFCCF31969093C60055
:10C4500090819923B1F74091C0035091C10360913D
:10C46000C2037091C3038CE095E022E030E00E94AB
:10C47000BF3FE2E6F2E007C08091C00085FFFCCF3D
:10C4800031969093C60090819923B1F78091C000B6
:10C4900085FFFCCF8AE08093C600A8C383E40E9496
:10C4A0008043882349F00E94AF450E94A4D7DC0155
:10C4B000CB018F730E9418C1EDEFF5E0949108C095
:10C4C0008091C00085FFFCCF9093C6003196949177
:10C4D0009923B1F76091B2197091B3198CE095E08E
:10C4E0004AE050E00E94E43EE2E6F2E007C08091BC
:10C4F000C00085FFFCCF31969093C60090819923B0
:10C50000B1F78091C00085FFFCCF8AE08093C60020
:10C510006DC385E40E948043882319F4CC24DD2474
:10C5200012C00E94AF450E94A4D76B0177FF0BC0D9
:10C530000F2EF0E0EF2EF0E0FF2EFCE80F2FF2E4DC
:10C540001F2FF02D0AC00F2EF0E0EF2EF0E0FF2E8F
:10C55000F6E10F2FF3E41F2FF02D83E50E948043B7
:10C56000882321F00E94AF457B018C0183E40E9467
:10C570008043882319F425E030E005C00E94AF45D0
:10C580000E94A4D79B01C801B701A6010E94AA9FDF
:10C590002DC30E94EB912AC30E946D380E941A3A63
:10C5A00025C30E946D3822C30E941A3A1FC3A0906F
:10C5B000C007B090C107C090C207D090C307A9823E
:10C5C000BA82CB82DC82E090C407F090C50700916C
:10C5D000C6071091C707ED82FE820F83188720914E
:10C5E000C8073091C9074091CA075091CB072987E6
:10C5F0003A874B875C878091CC079091CD07A091BB
:10C60000CE07B091CF078D879E87AF87B88BA98A59
:10C61000BA8ACB8ADC8AED8AFE8A0F8B188F298F23
:10C620003A8F4B8F5C8F8D8F9E8FAF8FB8A385E431
:10C630000E948043882369F0ED84FE840F85188969
:10C640000E94AF459B01AC01C801B7010E945CD6B6
:10C650000AC06D857E858F85988920E030E040E0B6
:10C6600050E40E945BD66D877E878F87988B6091A0
:10C670009E0370919F038091A0039091A10320E0FD
:10C6800030E040E752E40E943CD77B018C01CE01B0
:10C690000196BE016B5F7F4FAE01475F5F4F9E010A
:10C6A000235F3F4FABEECA2EA7E0DA2E0E945D72E9
:10C6B0008AE50E948043882359F0E984FA840B8537
:10C6C0001C850E94AF459B01AC01C801B70108C0A1
:10C6D00069857A858B859C8520E030E040E251E4D5
:10C6E0000E945CD669877A878B879C8760919E03BE
:10C6F00070919F038091A0039091A10320E030E00E
:10C7000040E752E40E943CD77B018C01CE010196A8
:10C71000BE016B5F7F4FAE01475F5F4F9E01235F9E
:10C720003F4FFBEECF2EF7E0DF2E0E945D7288E5D3
:10C730000E948043882389F0E980FA800B811C8164
:10C740000E94AF459B01AC01C801B7010E945CD6B5
:10C7500069837A838B839C8308C080E090E0A0E4A7
:10C76000B0E489839A83AB83BC8389E50E948043CC
:10C77000882339F00E94AF456D837E838F8398872D
:10C7800008C080E090E0A0E4B0E48D839E83AF8396
:10C79000B88760919E0370919F038091A003909150
:10C7A000A10320E030E040E752E40E943CD77B0147
:10C7B0008C01CE010196BE016B5F7F4FAE01475FDA
:10C7C0005F4F9E01235F3F4FEBEECE2EE7E0DE2E64
:10C7D0000E945D728CE40E948043882369F0ED849E
:10C7E000FE840F8518890E94AF459B01AC01C801EA
:10C7F000B7010E945CD60AC06D857E858F859889B9
:10C8000020E030E048EC52E40E945BD66D877E87E2
:10C810008F87988B60919E0370919F038091A003F6
:10C820009091A10320E030E040E752E40E943CD721
:10C830007B018C01CE010196BE016B5F7F4FAE0183
:10C84000475F5F4F9E01235F3F4FBBEECB2EB7E0AC
:10C85000DB2E0E945D720E94EB915E9A64E670E0AE
:10C8600080E090E00E9477D08DEE95E00E9434C188
:10C8700010E018C01F5F0E94D59D0E946E410E946B
:10C880006AC1112379F40C9A149A63E070E080E095
:10C8900090E00E9477D0149863E070E080E090E030
:10C8A0000E9477D00E9430A4882321F38CE40E9458
:10C8B0008043882369F0ED84FE840F8518890E94E7
:10C8C000AF459B01AC01C801B7010E945BD60AC00D
:10C8D0006D857E858F85988920E030E048EC52E4B4
:10C8E0000E945CD66D877E878F87988B8D859E850D
:10C8F000AF85B8898093CC079093CD07A093CE07DE
:10C90000B093CF078CEC97E00E942F6DA9E04A2EE0
:10C91000512C4C0E5D1EFDE06F2E712C6C0E7D1E99
:10C9200060919E0370919F038091A0039091A10359
:10C9300020E030E040E752E40E943CD77B018C01CC
:10C94000CE010196BE016B5F7F4FA2019301EBEE1A
:10C95000CE2EE7E0DE2E0E945D7251E1A52EB12CB5
:10C96000AC0EBD1E45E1842E912C8C0E9D1E609157
:10C970009E0370919F038091A0039091A10320E0FA
:10C9800030E040E752E40E943CD77B018C01C501B6
:10C99000B401A20193010E945D7239E1432E512C32
:10C9A0004C0E5D1E60919E0370919F038091A003C9
:10C9B0009091A10320E030E040E752E40E943CD790
:10C9C0007B018C01C501B401A20193010E945D723B
:10C9D00060919E0370919F038091A0039091A103A9
:10C9E00020E030E040E752E40E943CD77B018C011C
:10C9F000C501B401A2019E01235E3F4F0E945D72FA
:10CA0000F5C01092F8070E942DA48091550A9091CC
:10CA1000560AA091570AB091580A8093510A9093F0
:10CA2000520AA093530AB093540A0E945243DEC0A4
:10CA300084E50E948043882309F48DC00E94AF459D
:10CA40000E94A9D7262F6093500A6623B9F1E7E127
:10CA5000F5E0949108C08091C00085FFFCCF9093D1
:10CA6000C600319694919923B1F7ECEBF2E007C040
:10CA70008091C00085FFFCCF31969093C6009081D5
:10CA80009923B1F78CE095E0622F40E050E00E94DE
:10CA90009D3EEEEBF2E007C08091C00085FFFCCF29
:10CAA00031969093C60090819923B1F78091C00090
:10CAB00085FFFCCF8AE08093C60098C086E40E9480
:10CAC00080438823E1F00E94AF457B018C01609395
:10CAD0007E0A70937F0A8093800A9093810A20E0F7
:10CAE00030E040E050E00E9443D9181644F4E09250
:10CAF0009E03F0929F030093A0031093A103E7E12C
:10CB0000F5E0949108C08091C00085FFFCCF909320
:10CB1000C600319694919923B1F7EFECF2E007C08B
:10CB20008091C00085FFFCCF31969093C600908124
:10CB30009923B1F76091EB078CE095E070E04AE053
:10CB400050E00E94E43E8091C00085FFFCCF8AE067
:10CB50008093C6004BC0E7E1F5E0949108C0809156
:10CB6000C00085FFFCCF9093C60031969491992325
:10CB7000B1F7EAEDF5E0949108C08091C00085FF1F
:10CB8000FCCF9093C600319694919923B1F72091F0
:10CB9000820A3091830A80E690E0289FF001299F65
:10CBA000F00D389FF00D1124E257F54F07C080912A
:10CBB000C00085FFFCCF31969093C60090819923E9
:10CBC000B1F7E8EDF5E0949108C08091C00085FFD1
:10CBD000FCCF9093C600319694919923B1F7809140
:10CBE000C00085FFFCCF8AE08093C6000E944541CB
:10CBF0000BC00E94EB9188E50E948043882311F0CE
:10CC00000C94565C0C94595CEE960FB6F894DEBF0B
:10CC10000FBECDBFCF91DF911F910F91FF90EF908D
:10CC2000DF90CF90BF90AF909F908F907F906F904C
:10CC30005F904F903F902F900895CF93DF93809116
:10CC4000180C9091190C039714F40E9449498DE037
:10CC500095E060E00E94A4338091180C9091190C2B
:10CC6000892B09F46FC080910D05882309F450C009
:10CC70002091820A3091830A80E690E0289FE001AB
:10CC8000299FD00D389FD00D1124C257D54FCE010A
:10CC90006EE879E00E948A24892BF9F48DE095E012
:10CCA000BE010E94A02B80910E05882319F00E94DE
:10CCB000165132C0EBE8F9E0949108C08091C000B1
:10CCC00085FFFCCF9093C600319694919923B1F7DC
:10CCD0008091C00085FFFCCF17C08DE095E060E03B
:10CCE0000E94872BE9E7F9E0949108C08091C00089
:10CCF00085FFFCCF9093C600319694919923B1F7AC
:10CD00008091C00085FFFCCF8AE08093C60004C0FC
:10CD10000E9416510E94F5468091180C9091190CB2
:10CD200001979093190C8093180C8091820A90912E
:10CD3000830A019664E070E00E941ADB9093830AF4
:10CD40008093820A0E94D59D0E946E410E944E9857
:10CD50000E946AC1DF91CF910895DF93CF9300D0F5
:10CD6000CDB7DEB78CE095E040E052EC61E070E0DA
:10CD70000E94853DE0E6FAE0949108C08091C000F1
:10CD800085FFFCCF9093C600319694919923B1F71B
:10CD90008091C00085FFFCCF8AE08093C60047E108
:10CDA00055E0FA01949108C08091C00085FFFCCF46
:10CDB0009093C600319694919923B1F784B7282FA8
:10CDC00080FF15C0E8E5FAE0949108C08091C000AA
:10CDD00085FFFCCF9093C600319694919923B1F7CB
:10CDE0008091C00085FFFCCF8AE08093C60021FFC0
:10CDF00015C0E8E4FAE0949108C08091C00085FF76
:10CE0000FCCF9093C600319694919923B1F780910D
:10CE1000C00085FFFCCF8AE08093C60022FF15C0CA
:10CE2000E7E3FAE0949108C08091C00085FFFCCF51
:10CE30009093C600319694919923B1F78091C000E8
:10CE400085FFFCCF8AE08093C60023FF15C0E7E290
:10CE5000FAE0949108C08091C00085FFFCCF9093C8
:10CE6000C600319694919923B1F78091C00085FF57
:10CE7000FCCF8AE08093C60025FF15C0E7E1FAE009
:10CE8000949108C08091C00085FFFCCF9093C600AC
:10CE9000319694919923B1F78091C00085FFFCCF22
:10CEA0008AE08093C60014BEEFE0FAE0949108C0D7
:10CEB0008091C00085FFFCCF9093C600319694917D
:10CEC0009923B1F7E9E0FAE0949108C08091C0009D
:10CED00085FFFCCF9093C600319694919923B1F7CA
:10CEE0008091C00085FFFCCF8AE08093C600FA01E4
:10CEF0009491E7E1F5E008C08091C00085FFFCCF88
:10CF00009093C600319694919923B1F7E9EFF9E037
:10CF1000949108C08091C00085FFFCCF9093C6001B
:10CF2000319694919923B1F7E4EEF9E0949108C019
:10CF30008091C00085FFFCCF9093C60031969491FC
:10CF40009923B1F7E8EDF9E0949108C08091C00011
:10CF500085FFFCCF9093C600319694919923B1F749
:10CF6000EFECF9E0949108C08091C00085FFFCCF00
:10CF70009093C600319694919923B1F78091C000A7
:10CF800085FFFCCF8AE08093C600E4ECF9E0949141
:10CF900008C08091C00085FFFCCF9093C6003196F9
:10CFA00094919923B1F7E8EBF9E0949108C080914E
:10CFB000C00085FFFCCF9093C600319694919923D1
:10CFC000B1F78091C00085FFFCCF8AE08093C60056
:10CFD000FA019491E7E1F5E008C08091C00085FF77
:10CFE000FCCF9093C600319694919923B1F7E9EA6A
:10CFF000F9E0949108C08091C00085FFFCCF909328
:10D00000C600319694919923B1F720910F1B30916E
:10D01000101BCE0101962115310519F485519B4154
:10D0200002C0821B930B9A83898369817A818CE089
:10D0300095E04AE050E00E94E43EE2E9F9E0949194
:10D0400008C08091C00085FFFCCF9093C600319648
:10D0500094919923B1F78CE095E060ED74E04AE09B
:10D0600050E00E94E43E8091C00085FFFCCF8AE042
:10D070008093C6001092840A1092850A1092860A44
:10D080001092870A0E946D380E941A3A0E94149DDD
:10D090000E949A6F0E9419910E947F450E9451C27E
:10D0A00080E197E220E931E0F9013197F1F701974A
:10D0B000D9F70E94774D0F900F90CF91DF9108958F
:10D0C0002F923F924F925F926F927F928F929F9298
:10D0D000AF92BF92CF92DF92EF92FF920F931F9386
:10D0E000DF93CF93CDB7DEB7CD55D0400FB6F894D0
:10D0F000DEBF0FBECDBF2F969FAF8EAF2F9761962D
:10D100007FAF6EAF61972A0162962FAF62976396E9
:10D110000FAF63976496EFAE64976896ACAEBDAE02
:10D12000CEAEDFAE6897E22EFF24EE0CFF1CEE0CB5
:10D13000FF1C9A012E0D3F1D2D963FAF2EAF2D9750
:10D14000D9016D907D908D909C90FC01EE0DFF1D9E
:10D15000C401B30120813181428153810E945CD698
:10D1600069AF7AAF8BAF9CAF10E0000F111F000FBB
:10D17000111FF201E00FF11F2B96FFAFEEAF2B97BF
:10D18000A080B180C280D3802F96EEADFFAD2F97E7
:10D19000E00FF11FC601B501208131814281538129
:10D1A0000E945CD66DAB7EAB8FAB98AF64962FAD13
:10D1B0006497E22FF0E0EE0FFF1FEE0FFF1F2F9698
:10D1C000AEADBFAD2F97AE0FBF1F4D915D916D916D
:10D1D0007C9129964CAF5DAF6EAF7FAF299761967A
:10D1E0006EAD7FAD6197E60FF71F6081718182811F
:10D1F000938129962CAD3DAD4EAD5FAD29970E9430
:10D200005BD669AB7AAB8BAB9CAB6196AEADBFAD79
:10D2100061971C968D919D910D90BC91A02D2596A6
:10D220008CAF9DAFAEAFBFAF25972F96AEADBFAD64
:10D230002F971C962D913D914D915C911F972196B2
:10D240002CAF3DAF4EAF5FAF2197A4019301505873
:10D250002DA73EA74FA758ABB601A501705849A707
:10D260005AA76BA77CA761966EAD7FAD6197E60E5E
:10D27000F71ED7016D917D918D919C9129AD3AADAD
:10D280004BAD5CAD0E945BD63B014C016196EEADAF
:10D29000FFAD61970E0F1F1FD8016D917D918D918C
:10D2A0009C912DA93EA94FA958AD0E945BD65B0168
:10D2B0006C016DA57EA58FA598A9A60195010E9478
:10D2C00015DA7B018C0169A57AA58BA59CA5A40123
:10D2D00093010E9415DA9B01AC01C801B7010E94BD
:10D2E0005BD61B012C016DA57EA58FA598A9A40175
:10D2F00093010E9415DA7B018C0169A57AA58BA5A3
:10D300009CA5A60195010E9415DA9B01AC01C801FC
:10D31000B7010E945CD69B01AC01C201B1010E9421
:10D32000CFD65B016C0120E030E040E050E00E948D
:10D3300035D7882354F4C601B5012BED3FE049EC05
:10D3400050E40E945CD65B016C01E7968FADE797D5
:10D35000882351F0C601B5012BED3FE049EC50E4C4
:10D360000E945BD65B016C01C601B501E6962CAD4F
:10D370003DAD4EAD5FADE6970E9415DA29A93AA9F9
:10D380004BA95CA95F770E9450D97B018C012FE6E5
:10D3900032E143E85AE30E9435D787FDF6C1C80160
:10D3A000B7010E9412D80E94A9D778A76FA3672B54
:10D3B00021F4E1E0F0E0F8A7EFA32FA138A5B9012F
:10D3C00080E090E00E94D5D77B018C01C601B501B9
:10D3D000A80197010E943CD76BA37CA38DA39EA3B9
:10D3E00069A97AA98BA99CA9A80197010E943CD799
:10D3F0006F8F78A389A39AA325966CAD7DAD8EAD72
:10D400009FAD259721962CAD3DAD4EAD5FAD2197DB
:10D410000E945BD6A80197010E943CD76B8F7C8F3E
:10D420008D8F9E8F6BA17CA18DA19EA120E030E00D
:10D4300040E05FEB0E9415DA2BA13CA14DA15EA15B
:10D440000E9415DA20E030E040E85FE30E945CD6FD
:10D450006F8B788F898F9A8F64963FAD6497E32F97
:10D46000F0E0EE0FFF1FEE0FFF1F9E012F5F3F4FFB
:10D47000E20FF31F29964CAD5DAD6EAD7FAD2997E0
:10D4800040835183628373832F96AEADBFAD2F97D8
:10D490001C964D915D916D917C911F974D875E8794
:10D4A0006F87788B41E050E05A8B498B66246296F7
:10D4B0007FAD6297672F70E0660F771F660F771F4B
:10D4C000C901860F971F6A969FAF8EAF6A976396C2
:10D4D000BFAD6397AB2FB0E0AA0FBB1FAA0FBB1F56
:10D4E00021E030E02C0F3D1F2A0F3B1F6C963FAF11
:10D4F0002EAF6C976E96FFAFEEAF6E971AC138E104
:10D5000036150CF446C06DA57EA58FA598A92BA154
:10D510003CA14DA15EA10E9415DA7B018C0169A599
:10D520007AA58BA59CA52F89388D498D5A8D0E948F
:10D5300015DA9B01AC01C801B7010E945CD67B01E2
:10D540008C016DA57EA58FA598A92F89388D498D51
:10D550005A8D0E9415DA5B016C0169A57AA58BA52D
:10D560009CA52BA13CA14DA15EA10E9415DA9B01B7
:10D57000AC01C601B5010E945BD66DA77EA78FA73F
:10D5800098AB6394C701D80189A79AA7ABA7BCA79A
:10D5900065C049895A89BA0180E090E00E94D5D7D8
:10D5A0002BA13CA14DA15EA10E9415DA7B018C014B
:10D5B000C8010E9439D76B8B7C8B8D8B9E8BB701FA
:10D5C000C8010E9478DA3B014C012D96AEADBFAD8B
:10D5D0002D97ED90FD900D911C9117FB109517F96B
:10D5E00010952B96EEADFFAD2B97208031804280B9
:10D5F0005380C801B7012B893C894D895E890E94FF
:10D6000015DA5B016C01C201B101A40193010E9412
:10D6100015DA9B01AC01C601B5010E945CD66DA76D
:10D620007EA78FA798ABC801B701A40193010E9400
:10D6300015DA7B018C01C201B1012B893C894D892E
:10D640005E890E9415DA9B01AC01C801B7010E94F6
:10D650005BD669A77AA78BA79CA7662469AD7AAD2C
:10D660008BAD9CAD2DA53EA54FA558A90E945CD6BB
:10D670006A96AEADBFAD6A976D937D938D939C9383
:10D6800013976DA97EA98FA998AD29A53AA54BA599
:10D690005CA50E945CD66C96EEADFFAD6C97608386
:10D6A0007183828393836E96AEADBFAD6E976D919D
:10D6B0007D918D919C912F8D38A149A15AA10E94F5
:10D6C0005CD66E96EEADFFAD6E97608371838283FC
:10D6D00093836D857E858F8598892B8D3C8D4D8DAF
:10D6E0005E8D0E945CD66D877E878F87988BCE017A
:10D6F00001960E94C23FCE010196BE016B5F7F4F33
:10D70000AE01475F5F4F9E01235F3F4F6896ECACD1
:10D71000FDAC0EAD1FAD6897F7E7CF2ED12CCC0E28
:10D72000DD1E0E945D7229893A892F5F3F4F3A8B37
:10D73000298B49895A896FA178A54617570708F49C
:10D74000DECE61964EAD5FAD6197485F5F4F6196EB
:10D750002EAD3FAD6197245F3F4F61968EAD9FAD7B
:10D760006197DC0114966196BFAFAEAF6197BD01C2
:10D770006896ECACFDAC0EAD1FAD6897E7E7CE2E1A
:10D78000D12CCC0EDD1E0E945D72C35ADF4F0FB646
:10D79000F894DEBF0FBECDBFCF91DF911F910F91E7
:10D7A000FF90EF90DF90CF90BF90AF909F908F90C1
:10D7B0007F906F905F904F903F902F9008953F9291
:10D7C0004F925F926F927F928F929F92AF92BF9291
:10D7D000CF92DF92EF92FF920F931F93CF93DF933D
:10D7E0008091ED0F882309F4F6C08090A7039090F4
:10D7F000A803A090A903B090AA0360915317709159
:10D800005417882777FD8095982F0E94D7D720E05E
:10D8100030E040E050E40E945CD6A50194010E94F3
:10D8200035D787FDD8C03090BF140F2EF0E04F2EB3
:10D83000F0E05F2EF0E06F2EF0E07F2EF02DCDE4D3
:10D84000D0E058C0232D30E02C9FF0012D9FF00D2B
:10D850003C9FF00D1124E251F04F80819181A28113
:10D86000B3810097A105B10581F484819581A681DA
:10D87000B7810097A105B10541F480859185A28506
:10D88000B3850097A105B10591F12C9F60012D9FF3
:10D89000D00C3C9FD00C11248EEE9FE0C80ED91EF8
:10D8A000F60164857585868597850E94D7D77B01AB
:10D8B0008C01F60160897189828993890E94D5D78C
:10D8C0009B01AC01C801B7010E943CD7F60122A11F
:10D8D00033A144A155A10E9415DA7B018C01A3015B
:10D8E00092010E9443D9181614F427013801339489
:10D8F000FFE03F228091BE14381609F0A3CFC30188
:10D90000B2012091AB033091AC034091AD03509133
:10D91000AE030E9415DA9B01AC01C501B4010E945F
:10D920005CD67B018C01A50194010E9435D787FD4F
:10D9300002C0470158011091A3030091A403F09085
:10D94000A503E090A603C501B401212F302F4F2D70
:10D950005E2D0E9443D9181634F4812F902FAF2DDD
:10D96000BE2D4C015D014090D4145090D5146090B0
:10D97000D6147090D714C301B201A50194010E947E
:10D9800043D91816C4F4C501B40120E037ED43EAC9
:10D990005CE30E9415DA7B018C01C301B20128E42B
:10D9A00031EE4AE75FE30E9415DAA80197010E9471
:10D9B0005CD64B015C018092D4149092D514A09255
:10D9C000D614B092D714C501B4010E94A4D77093A5
:10D9D000541760935317DF91CF911F910F91FF90D0
:10D9E000EF90DF90CF90BF90AF909F908F907F90FF
:10D9F0006F905F904F903F9008958091BE149091EA
:10DA0000BF14891B8F7008950F931F93CF93DF93DB
:10DA1000C0E0D0E08E010353104FFE01EF55F04FF0
:10DA200060817181828193810E94D5D7FE01EF567A
:10DA3000F04F20813181428153810E9415DA0E948A
:10DA4000A9D7F80160837183828393832496C031C0
:10DA5000D10501F7DF91CF911F910F910895FC013E
:10DA6000608171818281938120919D0F30919E0F01
:10DA700040919F0F5091A00F0E9415DA0E94E5D9A6
:10DA80006093E90F7093EA0F8093EB0F9093EC0F84
:10DA900089EE9FE00E94A59108958F929F92AF9288
:10DAA000BF92CF92DF92EF92FF920F931F93FC01F0
:10DAB0008B015A014901608171818281938120919A
:10DAC000910F3091920F4091930F5091940F0E94BB
:10DAD00015DA0E94E5D93DEDC32E3FE0D32E6093C9
:10DAE000DD0F7093DE0F8093DF0F9093E00FF8014E
:10DAF00060817181828193812091950F3091960F81
:10DB00004091970F5091980F0E9415DA0E94E5D925
:10DB100024E0E22EF12CEC0CFD1C6093E10FF701E8
:10DB2000718382839383F501608171818281938106
:10DB30002091990F30919A0F40919B0F50919C0F1B
:10DB40000E9415DA0E94E5D98601085F1F4F609395
:10DB5000E50FF801718382839383F4016081718101
:10DB60008281938120919D0F30919E0F40919F0F54
:10DB70005091A00F0E9415DA0E94E5D9F6013C965B
:10DB80006093E90F718382839383C601B701A80173
:10DB90009F010E946B9180E090E0A0E0B0E0809354
:10DBA000C0149093C114A093C214B093C314809373
:10DBB000C4149093C514A093C614B093C714809353
:10DBC000C8149093C914A093CA14B093CB14809333
:10DBD000CC149093CD14A093CE14B093CF14809313
:10DBE000D0149093D114A093D214B093D3141F9156
:10DBF0000F91FF90EF90DF90CF90BF90AF909F90EC
:10DC00008F9008958F929F92AF92BF92CF92DF92A2
:10DC1000EF92FF920F931F93CF93DF93EC016B0171
:10DC2000009709F45CC08FA9882309F058C0EEA0C2
:10DC3000FFA008A519A5FB01B6A0A7A090A481A4E8
:10DC4000C801B7012B2D3A2D492D582D0E9435D7EB
:10DC500088230CF044C0C801B701A80197010E94B5
:10DC600015DA7B018C016AA97BA98CA99DA9905822
:10DC700020E030E040E050EC0E9415DA2EA53FA5F0
:10DC800048A959A90E9415DA9B01AC01C801B70146
:10DC90000E945CD60E9482DA7B018C016B2D7A2D6A
:10DCA000892D982D9701A8010E9435D7882324F447
:10DCB000EB2CFA2C092D182D6B2D7A2D892D982DF2
:10DCC0009701A8010E9435D7882349F0C701D801E0
:10DCD000F60186A397A3A0A7B1A781E086ABDF9149
:10DCE000CF911F910F91FF90EF90DF90CF90BF9059
:10DCF000AF909F908F900895EF92FF920F931F9394
:10DD0000CF93DF93F090BF1400E010E020E030E00C
:10DD10004DE4E42E12C0FE9CE0011124C251D04F0C
:10DD2000C901B801AE010E94026E8F2D8F5F803154
:10DD300009F480E0F82E98018E018091BE14F81647
:10DD400051F7C901B80140E050E00E94026EDF9136
:10DD5000CF911F910F91FF90EF900895AF92BF92D6
:10DD6000CF92DF92EF92FF920F931F93CF93DF93A7
:10DD7000EB018A016115710509F466C04115510571
:10DD800009F462C0DAA4CBA4BCA4ADA46EA17FA1A7
:10DD900088A599A52D2D3C2D4B2D5A2D0E9435D7A8
:10DDA000882309F451C08FA9882309F043C0F801E2
:10DDB000E6A0F7A000A511A56D2D7C2D8B2D9A2D29
:10DDC000A80197010E9443D91816A4F5C801B7010C
:10DDD000A80197010E9415DA7B018C016AA97BA931
:10DDE0008CA99DA9905820E030E040E050EC0E94C2
:10DDF00015DA2EA53FA548A959A90E9415DA9B015D
:10DE0000AC01C801B7010E945CD60E9482DA7B0196
:10DE10008C016D2D7C2D8B2D9A2D9701A8010E94D0
:10DE200035D7882324F4ED2CFC2C0B2D1A2DC7019B
:10DE3000D80104C08D2D9C2DAB2DBA2D8EA39FA390
:10DE4000A8A7B9A781E08EABDF91CF911F910F9169
:10DE5000FF90EF90DF90CF90BF90AF900895CF925A
:10DE6000DF92EF92FF920F93DF93CF9300D0CDB765
:10DE7000DEB78091BE148FB7F894F090BF148FBFB7
:10DE80008091BE1490E040968F1991098F70907028
:10DE9000049704F10091BE1403500F70CC24DD24CC
:10DEA00040E050E06DE4E62E13C0802F002309F41B
:10DEB00080E1082F01500E9DC00111248251904F26
:10DEC0009A838983B6010E94AE6EA601C980DA806A
:10DED0000F1559F70F900F90CF91DF910F91FF9091
:10DEE000EF90DF90CF9008956091EC079091BF1470
:10DEF0008091BE149817B9F04091BF14242F30E0E0
:10DF00008DE490E0289FF001299FF00D389FF00DDF
:10DF10001124EA5CFF4E608102C04F5F4F70809118
:10DF2000BE144817D1F784E070E00E9418D10E9417
:10DF3000DF6B08951092BE141092BF1480E1EDEDD6
:10DF4000FFE0DF011D928A95E9F780E090E0A0E014
:10DF5000B0E08093C4149093C514A093C614B093FA
:10DF6000C7148093C8149093C914A093CA14B09393
:10DF7000CB148093CC149093CD14A093CE14B09373
:10DF8000CF148093D0149093D114A093D214B09353
:10DF9000D3148093C0149093C114A093C214B0936F
:10DFA000C31408952F923F924F925F926F927F9287
:10DFB0008F929F92AF92BF92CF92DF92EF92FF9299
:10DFC0000F931F93DF93CF93CDB7DEB766970FB64E
:10DFD000F894DEBF0FBECDBF9E8B8D8B6A017B0197
:10DFE00048015901DC01D8966D917D918D919C91EC
:10DFF000DB970E94D5D7698B7A8B8B8B9C8BA70183
:10E0000096010E9415DA0E9422D70E94A9D76D833B
:10E010007E838F83988769897A898B899C89A501FA
:10E0200094010E9415DA0E9422D70E94A9D7698321
:10E030007A838B839C832D813E814F81588528373D
:10E0400031054105510540F448E750E060E070E0DB
:10E050004D835E836F83788769817A818B819C8110
:10E06000683771058105910540F488E790E0A0E0EC
:10E07000B0E089839A83AB83BC83AD89BE89AC5BF6
:10E08000BF4FAD90BD90CD90DC901397A454B0409D
:10E09000BE8BAD8B6D817E818F8198850E94D5D797
:10E0A0006D877E878F87988BC601B5010E94D7D771
:10E0B0001B012C0120E030E040E050E00E9435D709
:10E0C000882321F4E0E070E060E028C069897A8963
:10E0D0008B899C899B01AC010E9415DA7B018C0124
:10E0E0006D857E858F8598899B01AC010E9415DA2C
:10E0F0009B01AC01C801B7010E945BD67B018C017A
:10E10000C201B101A20191010E945CD69B01AC0148
:10E11000C801B7010E943CD7E62F692F2E2F372F59
:10E12000482F562FB901CA010E9422D70E94A4D7B6
:10E130003B014C0169817A818B819C810E94D5D7FA
:10E1400069877A878B879C8766277727CB016A192F
:10E150007B098C099D090E94D7D75B016C0120E0E7
:10E1600030E040E050E00E9435D7882321F4E0E021
:10E1700070E060E028C069857A858B859C859B016D
:10E18000AC010E9415DA7B018C0169897A898B893F
:10E190009C899B01AC010E9415DA9B01AC01C8016E
:10E1A000B7010E945BD67B018C01C601B501A601B7
:10E1B00095010E945CD69B01AC01C801B7010E9489
:10E1C0003CD7E62F692F2E2F372F482F562FB90116
:10E1D000CA010E9412D8ED89FE89A088B188C28840
:10E1E000D38886017501E618F708080919090E9405
:10E1F000A4D7A8019701261B370B480B590B57FFD3
:10E2000071C0C201B10120E030E040E050E00E9466
:10E2100035D7882321F4E0E070E060E044C0C2011B
:10E22000B101A20191010E945CD67B018C01C60163
:10E23000B5010E94D5D79B01AC01C801B7010E946E
:10E2400015DA7B018C016D857E858F8598899B0110
:10E25000AC010E9415DA9B01AC01C801B7010E9414
:10E260005BD67B018C0169857A858B859C859B01BA
:10E27000AC010E9415DA9B01AC01C801B7010E94F4
:10E280005CD67B018C01C201B10120E030E040E8A6
:10E2900050E40E9415DA9B01AC01C801B7010E944D
:10E2A0003CD7E62F692F2E2F372F482F562FB90135
:10E2B000CA010E9422D70E94A4D7AC01CB01DA0187
:10E2C0003C014D0197FE03C06624772443016A1484
:10E2D0007B048C049D0410F03501460120E030E001
:10E2E00040E050E09FB7F8946D897E89645B7F4F72
:10E2F000DB018C91AC54B040BE8BAD8B882321F5F3
:10E30000FD01648A758A868A978A260D371D481D05
:10E31000591D58962D933D934D935C935B972D819A
:10E320003E814F815885DC962D933D934D935C93B0
:10E33000DF97A05CBF4F29813A814B815C812D938F
:10E340003D934D935C9313979FBF66960FB6F894D9
:10E35000DEBF0FBECDBFCF91DF911F910F91FF9018
:10E36000EF90DF90CF90BF90AF909F908F907F9075
:10E370006F905F904F903F902F9008954F925F92D3
:10E380007F928F929F92AF92BF92CF92DF92EF9245
:10E39000FF920F931F93CF93DF937090BF14C0E051
:10E3A000D0E07DE4472E512C46C02097B1F18EA9D4
:10E3B000882361F4849CF001859CF00D949CF00D01
:10E3C0001124E251F04F86A9882339F1EAA0FBA07D
:10E3D0000CA11DA16EA17FA188A599A5A8019701F7
:10E3E0000E943CD75B016C01849CF001859CF00D80
:10E3F000949CF00D1124E251F04F66A177A180A505
:10E4000091A5A80197010E943CD78B019C01CE01E8
:10E41000B601A5010E94D26F1EAA739480E17816FE
:10E4200009F47724849CE001859CD00D949CD00D48
:10E430001124C251D04F872C992487FC909480914D
:10E44000BE1490E08816990609F0AFCF2097F1F03E
:10E45000EAA0FBA00CA11DA16EA17FA188A599A592
:10E46000A80197010E943CD75B016C016DEC7CEC2C
:10E470008CE49DE3A80197010E943CD78B019C018D
:10E48000CE01B601A5010E94D26F1EAADF91CF91E5
:10E490001F910F91FF90EF90DF90CF90BF90AF90C2
:10E4A0009F908F907F905F904F9008950E942F6F64
:10E4B0000E947C6E0E94BE7108952F923F924F92EF
:10E4C0005F926F927F928F929F92AF92BF92CF9204
:10E4D000DF92EF92FF920F931F93DF93CF93CDB70D
:10E4E000DEB7CC59D0400FB6F894DEBF0FBECDBF1B
:10E4F0005C014B013A012901C756DF4FE882C95937
:10E50000D040C656DF4FF882CA59D040C556DF4FBB
:10E510000883CB59D040C456DF4F1883CC59D04024
:10E52000E796DFAECEAEE7978091BE148F5F803165
:10E5300009F480E0282F332727FD309538A72FA333
:10E5400006C00E94D59D0E946E410E946AC18091C2
:10E55000BF1490E04FA158A58417950791F36091DF
:10E56000910F7091920F8091930F9091940FE59677
:10E570006CAF7DAF8EAF9FAFE597D5012D913D91EB
:10E580004D915C910E9415DA0E94E5D9CD57DF4F7D
:10E590006883C358D040CC57DF4F7883C458D040ED
:10E5A000CB57DF4F8883C558D040CA57DF4F988379
:10E5B000C658D0402091950F3091960F4091970FFB
:10E5C0005091980FE1962CAF3DAF4EAF5FAFE19702
:10E5D000CA01B901D4012D913D914D915C910E94E8
:10E5E00015DA0E94E5D9C957DF4F6883C758D04074
:10E5F000C857DF4F7883C858D040C757DF4F88834C
:10E60000C958D040C657DF4F9883CA58D040209190
:10E61000990F30919A0F40919B0F50919C0FAD969E
:10E620002CAF3DAF4EAF5FAFAD97CA01B901D3017B
:10E630002D913D914D915C910E9415DA0E94E5D992
:10E64000C557DF4F6883CB58D040C457DF4F78831E
:10E65000CC58D040C357DF4F8883CD58D040C257E5
:10E66000DF4F9883CE58D04020919D0F30919E0F60
:10E6700040919F0F5091A00FA9962CAF3DAF4EAF88
:10E680005FAFA997CA01B901D2012D913D914D917A
:10E690005C910E9415DA0E94E5D9C157DF4F68836B
:10E6A000CF58D040C057DF4F7883C059D040CF56A5
:10E6B000DF4F8883C159D040CE56DF4F9883C2596F
:10E6C000D0408091BE14E82FF0E0A596FFAFEEAFEA
:10E6D000A5978DE490E09F01289FF001299FF00D00
:10E6E000389FF00D1124E251F04FE45BFF4F108290
:10E6F000EC54F0404091DD0F5091DE0F6091DF0F40
:10E700007091E00FA3964CAF5DAF6EAF7FAFA39754
:10E71000CD57DF4F88819981AA81BB81C358D040F2
:10E72000841B950BA60BB70B6F968CAF9DAFAEAF4E
:10E73000BFAF6F9780839183A283B383B7FF0BC072
:10E74000B095A095909581959F4FAF4FBF4F808317
:10E750009183A283B3832091E10F3091E20F409126
:10E76000E30F5091E40F6B962CAF3DAF4EAF5FAF10
:10E770006B97C957DF4F688179818A819B81C75820
:10E78000D040621B730B840B950B67966CAF7DAF0B
:10E790008EAF9FAF67978DE490E0A596AEADBFAD0D
:10E7A000A597A89FF001A99FF00DB89FF00D112427
:10E7B000E251F04F67962CAD3DAD4EAD5FAD679722
:10E7C000248335834683578357FF0DC0DA01C9017F
:10E7D000B095A095909581959F4FAF4FBF4F848383
:10E7E0009583A683B7834091E50F5091E60F609122
:10E7F000E70F7091E80F63964CAF5DAF6EAF7FAFE0
:10E800006397C557DF4F88819981AA81BB81CB5817
:10E81000D040841B950BA60BB70B2F968CAF9DAFEA
:10E82000AEAFBFAF2F978DE490E0A596AEADBFAD74
:10E83000A597A89FF001A99FF00DB89FF00D112496
:10E84000E251F04F2F962CAD3DAD4EAD5FAD2F9701
:10E85000208731874287538757FF0DC0DA01C901EE
:10E86000B095A095909581959F4FAF4FBF4F8087F2
:10E870009187A287B3872090E90F3090EA0F4090EC
:10E88000EB0F5090EC0FC157DF4F488159816A81DF
:10E890007B81CF58D04042195309640975092B96E2
:10E8A0004CAF5DAF6EAF7FAF2B97E091EB07F0E021
:10E8B000EE0FFF1FEE0FFF1FEA58FC4F60817181C2
:10E8C0008281938127966CAF7DAF8EAF9FAF2797E4
:10E8D000809174039091750323969FAF8EAF239719
:10E8E0002B966CAD7DAD8EAD9FAD2B9797FF07C07E
:10E8F00090958095709561957F4F8F4F9F4F0E94A7
:10E90000D7D727962CAD3DAD4EAD5FAD27970E9472
:10E9100015DA0E94A4D72396AEADBFAD23979D0113
:10E92000442737FD4095542F0E94E7DA24E630E073
:10E9300040E050E00E944FDB8DE490E0A5966EAD84
:10E940007FADA597689FF001699FF00D789FF00D4E
:10E950001124E251F04FDF011C96248711963C935D
:10E96000119712964C93129713965C93E080F18066
:10E97000028113816480758086809780A084B18431
:10E98000C284D384C901DA018A159B05AC05BD0593
:10E9900014F4D601C50186159705A805B90514F428
:10E9A000D401C3019C01AD018E159F05A007B107DD
:10E9B00014F4A80197018DE490E0A596AEADBFAD2B
:10E9C000A597A89FB001A99F700DB89F700D112445
:10E9D0006251704FFB01208B318B428B538B263061
:10E9E00031054105510510F40C94F77DE85BFF4FAC
:10E9F0008091EC079091ED07AA2797FDA095BA2F7B
:10EA000080839183A283B383DB0190961C92CD57C0
:10EA1000DF4F288139814A815B81C358D040A3965A
:10EA20008CAD9DADAEADBFADA397281739074A0792
:10EA30005B0724F481E0DB0190968C93C957DF4F8C
:10EA4000288139814A815B81C758D0406B966CAD73
:10EA50007DAD8EAD9FAD6B972617370748075907D9
:10EA600094F48DE490E0A596AEADBFADA597A89FB8
:10EA7000F001A99FF00DB89FF00D1124E251F04F65
:10EA800080A1826080A3C557DF4F288139814A81E8
:10EA90005B81CB58D04063966CAD7DAD8EAD9FADA4
:10EAA0006397261737074807590794F48DE490E0D9
:10EAB000A596AEADBFADA597A89FF001A99FF00D9B
:10EAC000B89FF00D1124E251F04F80A1846080A323
:10EAD000C157DF4F288139814A815B81CF58D040AF
:10EAE000221533054405550594F48DE490E0A59670
:10EAF0004EAD5FADA597489FF001499FF00D589F1F
:10EB0000F00D1124E251F04F80A1886080A38DE4C4
:10EB100090E0A5966EAD7FADA597689FF001699FC7
:10EB2000F00D789FF00D1124E251F04FE796AEAD55
:10EB3000BFADE7978C9181A32081318142815381C0
:10EB400021962CAF3DAF4EAF5FAF21972115310518
:10EB50004105510509F05E988DE490E0A5964EAD13
:10EB60005FADA597489FF001499FF00D589FF00DAC
:10EB70001124E251F04F6480758086809780611483
:10EB800071048104910409F05E988DE490E0A596EB
:10EB90006EAD7FADA597689FF001699FF00D789FDE
:10EBA000F00D1124E251F04FA084B184C284D384CB
:10EBB000A114B104C104D10409F015988DE490E0CA
:10EBC000A596AEADBFADA597A89FF001A99FF00D8A
:10EBD000B89FF00D1124E251F04F84859585A685EC
:10EBE000B7850097A105B10551F05E982090B10F4F
:10EBF0003090B20F4090B30F5090B40F08C02090E7
:10EC0000C90F3090CA0F4090CB0F5090CC0FC75611
:10EC1000DF4F6881C959D040C656DF4F7881CA5945
:10EC2000D040C556DF4F8881CB59D040C456DF4F06
:10EC30009881CC59D040A20191010E9435D787FD1F
:10EC400016C0C756DF4F8881C959D040C656DF4F1E
:10EC50009881CA59D040C556DF4FA881CB59D040C2
:10EC6000C456DF4FB881CC59D0401C012D016F969E
:10EC70006CAD7DAD8EAD9FAD6F970E94D7D7E596F9
:10EC80002CAD3DAD4EAD5FADE5970E943CD7C15870
:10EC9000DF4F6883CF57D040C058DF4F7883C058CC
:10ECA000D040CF57DF4F8883C158D040CE57DF4F79
:10ECB0009883C258D040AC01CB01DA0189839A8392
:10ECC000AB83BC8367966CAD7DAD8EAD9FAD679712
:10ECD0000E94D7D7E1962CAD3DAD4EAD5FADE1972B
:10ECE0000E943CD7EC966FAFEC97ED967FAFED9717
:10ECF000EE968FAFEE97EF969FAFEF97AC01CB01FB
:10ED0000DA018D839E83AF83B8872F966CAD7DAD7E
:10ED10008EAD9FAD2F970E94D7D7AD962CAD3DAD50
:10ED20004EAD5FADAD970E943CD7E8966FAFE897C8
:10ED3000E9967FAFE997EA968FAFEA97EB969FAF98
:10ED4000EB97AC01CB01DA0189879A87AB87BC8747
:10ED50002B966CAD7DAD8EAD9FAD2B970E94D7D716
:10ED6000A9962CAD3DAD4EAD5FADA9970E943CD7A5
:10ED700027962CAD3DAD4EAD5FAD27970E9415DABD
:10ED80007B018C012396EEADFFAD2397BF01882751
:10ED900077FD8095982F0E94D7D79B01AC01C801C1
:10EDA000B7010E9415DA20E030E048EC52E40E94FE
:10EDB0003CD79B01AC016D877E878F87988B21960E
:10EDC0006CAD7DAD8EAD9FAD21976630710581052F
:10EDD00091051CF576E06716710481049104ECF44A
:10EDE00086E0A816B104C104D104BCF48DE490E01F
:10EDF000A596AEADBFADA597A89FF001A99FF00D58
:10EE0000B89FF00D1124E251F04FDA01C901BF772C
:10EE100086A797A7A0ABB1AB5DC0C158DF4F2881D3
:10EE2000CF57D040C058DF4F3881C058D040CF575F
:10EE3000DF4F4881C158D040CE57DF4F5881C2586C
:10EE4000D040B901CA010E94CCDA3B014C01EC96DA
:10EE50002FADEC97ED963FADED97EE964FADEE975B
:10EE6000EF965FADEF97B901CA010E94CCDA5B0162
:10EE70006C01E8962FADE897E9963FADE997EA96E1
:10EE80004FADEA97EB965FADEB97B901CA010E94CF
:10EE9000CCDA7B018C01C401B301A60195010E946B
:10EEA0005CD6A80197010E945CD60E9482DA2DE40C
:10EEB00030E0A5964EAD5FADA597429FF001439F10
:10EEC000F00D529FF00D1124E251F04F66A777A785
:10EED00080AB91AB8DE490E0A5966EAD7FADA5972C
:10EEE000689FF001699FF00D789FF00D1124E251A9
:10EEF000F04F86A597A5A0A9B1A989AF9AAFABAFEE
:10EF0000BCAF60E070E080E89FE329AD3AAD4BAD67
:10EF10005CAD0E943CD79B01AC01C201B1010E94D3
:10EF200015DA2B013C018091BE149091BF14A82FDB
:10EF3000B0E05096A91BB109AF70B070BEA3ADA3ED
:10EF4000A230B1050CF451C05D01CC24B7FCC094D3
:10EF5000DC2CC601B5010E94D7D720E030E040E0AC
:10EF600051E40E9435D788230CF03FC060E074E282
:10EF700084E799E4A30192010E943CD70E94E5D95D
:10EF80007B018C0160917D0F70917E0F80917F0FCE
:10EF90009091800FE616F7060807190730F56E19ED
:10EFA0007F09800B910B660F771F881F991FA601A1
:10EFB00095010E942DDBCA01B9010E94D5D70E949C
:10EFC000E5D99B01AC012E0D3F1D401F511FCA0109
:10EFD000B9010E94D5D79B01AC0160E074E284E7DF
:10EFE00099E40E943CD72B013C018DE490E0A5966A
:10EFF000EEADFFADA597E89F8001E99F100DF89F4A
:10F00000100D11240251104F69AD7AAD8BAD9CAD3E
:10F01000A30192010E9415DAD80192966D937D9317
:10F020008D939C93959750966D917D918D919C9128
:10F0300053970E94D5D7A30192010E9415DA0E942E
:10F0400022D70E94A9D7F80160AF71AF82AF93AF0A
:10F05000CD56DF4F1882C359D040CC56DF4F1882AF
:10F06000C459D04020E8222E9FE3392E88249924C9
:10F07000E1E0F0E0EC0FFD1FE80DF91DC301B20166
:10F0800020813181428153810E9415DAE1E1F0E073
:10F09000EC0FFD1FE80DF91D60837183828393835C
:10F0A0005B016C01E894D7F8F401EF57F04FE08072
:10F0B000F18002811381C601B501A80197010E9468
:10F0C00043D91816CCF4C801B701A60195010E94D6
:10F0D0003CD76B017C01CD56DF4F6881C359D040CE
:10F0E000CC56DF4F7881C459D040C101A7019601A9
:10F0F0000E9435D788236CF4CD56DF4F8881C359E1
:10F10000D040CC56DF4F9881C459D040D1016C011A
:10F110007D0124E030E0820E931E30E183169104DD
:10F1200071F0D701C601CD56DF4FC882C359D04018
:10F13000CC56DF4F9883C459D0401D0199CFC701E9
:10F14000B60120E030E040E85FE30E9435D7882335
:10F150000CF04CC08E010F5E1F4F81E2A82EB12C27
:10F16000AC0EBD1ED8016D917D918D919C91A70132
:10F1700096010E9415DAF80161937193819391933E
:10F180008F01EA15FB0571F78DE490E0A5962EAD91
:10F190003FADA597289F8001299F100D389F100D26
:10F1A00011240251104FD80192966D917D918D914D
:10F1B0009C919597A70196010E9415DAF80162A328
:10F1C00073A384A395A360AD71AD82AD93AD0E948E
:10F1D000D5D7A70196010E9415DA0E94A9D7D801B8
:10F1E000D8966D937D938D939C93DB978DE490E0FF
:10F1F000A596EEADFFADA597E89F8001E99F100DA4
:10F20000F89F100D11240251104FD80150966D91A6
:10F210007D918D919C9153970E94D5D7F80126A599
:10F2200037A540A951A90E943CD71B012C01F80128
:10F2300080819181A281B3810097A105B10549F533
:10F2400084819581A681B7810097A105B10509F553
:10F2500080859185A285B3850097A105B105C9F484
:10F26000C201B1012091B90F3091BA0F4091BB0F8B
:10F270005091BC0F0E9415DA0E9422D70C5B1F4FE1
:10F280000E94A9D7D8016D937D938D939C9313977A
:10F2900071C1C201B1012091B50F3091B60F4091FB
:10F2A000B70F5091B80F0E9415DA0E9422D70E9422
:10F2B000A9D72DE430E0A596EEADFFADA597E29F6E
:10F2C0006001E39FD00CF29FD00C11242EEE3FE0A2
:10F2D000C20ED31EB4E46B2E712C6C0C7D1CD301BA
:10F2E0006D937D938D939C9313978090CD0F909009
:10F2F000CE0FA090CF0FB090D00F0E94D5D77B013A
:10F300008C01F60160817181828193810E94D7D73F
:10F310009B01AC01C801B7010E9415DA7B018C0189
:10F32000D60150966D917D918D919C9153970E943D
:10F33000D5D79B01AC01C801B7010E943CD77B0126
:10F340008C01C501B4010E94D5D79B01AC01C80155
:10F35000B7010E9443D918162CF4F30180829182E0
:10F36000A282B3828090D10F9090D20FA090D30F41
:10F37000B090D40F8DE490E0A5962EAD3FADA5974B
:10F38000289F6001299FD00C389FD00C11244EEE8D
:10F390005FE0C40ED51EA4E46A2E712C6C0C7D1C9B
:10F3A000D3016D917D918D919C910E94D5D77B0168
:10F3B0008C01F60164817581868197810E94D7D77F
:10F3C0009B01AC01C801B7010E9415DA7B018C01D9
:10F3D000D60150966D917D918D919C9153970E948D
:10F3E000D5D79B01AC01C801B7010E943CD77B0176
:10F3F0008C01C501B4010E94D5D79B01AC01C801A5
:10F40000B7010E9443D918162CF4F301808291822F
:10F41000A282B3828090D90F9090DA0FA090DB0F78
:10F42000B090DC0F8DE490E0A5962EAD3FADA59792
:10F43000289F6001299FD00C389FD00C11244EEEDC
:10F440005FE0C40ED51EF4E46F2E712C6C0C7D1C95
:10F45000D3016D917D918D919C910E94D5D77B01B7
:10F460008C01F60164857585868597850E94D7D7BE
:10F470009B01AC01C801B7010E9415DA7B018C0128
:10F48000D60150966D917D918D919C9153970E94DC
:10F49000D5D79B01AC01C801B7010E943CD77B01C5
:10F4A0008C01C501B4010E94D5D79B01AC01C801F4
:10F4B000B7010E9443D918162CF4F301808291827F
:10F4C000A282B3828090D50F9090D60FA090D70FD4
:10F4D000B090D80F8DE490E0A5962EAD3FADA597E6
:10F4E000289F6001299FD00C389FD00C11244EEE2C
:10F4F0005FE0C40ED51EE4E46E2E712C6C0C7D1CF6
:10F50000D3016D917D918D919C910E94D5D77B0106
:10F510008C01F60160857185828593850E94D7D71D
:10F520009B01AC01C801B7010E9415DA7B018C0177
:10F53000D60150966D917D918D919C9153970E942B
:10F54000D5D79B01AC01C801B7010E943CD77B0114
:10F550008C01C501B4010E94D5D79B01AC01C80143
:10F56000B7010E9443D918162CF4F30180829182CE
:10F57000A282B3828DE490E0A5962EAD3FADA59713
:10F58000289F6001299FD00C389FD00C11244EEE8B
:10F590005FE0C40ED51EF601EC5BFF4F6081718108
:10F5A000828193810E94D5D77B018C01A2019101B8
:10F5B0000E943CD7D601D2966D937D938D939C93F8
:10F5C000D597C801B7012DEB37E346E051E40E941F
:10F5D00015DA0E94A4D7F601648F758F868F978FF6
:10F5E0006090BD0F7090BE0F8090BF0F9090C00FC5
:10F5F000C401B30120E030E040E05FE30E9415DA8F
:10F600005B016C01298D3A8D4B8D5C8D2DAB3EAB32
:10F610004FAB58AF4091C10F5091C20F6091C30FD3
:10F620007091C40F49AB5AAB6BAB7CABCB01BA0149
:10F6300020E030E040E05FE30E9415DA7B018C01BE
:10F640006DA97EA98FA998AD9F77A80197010E9407
:10F6500043D9181644F4C601B501A80197010E94C8
:10F6600035D7882314F4860175016D8D7E8D8F8DBD
:10F6700098A16DA77EA78FA798AB8091C50F909199
:10F68000C60FA091C70FB091C80F89A79AA7ABA7C3
:10F69000BCA7BC01CD0120E030E040E05FE30E9468
:10F6A00015DA1B012C016DA57EA58FA598A99F7762
:10F6B000A20191010E9443D9181644F4C801B70170
:10F6C000A20191010E9435D7882314F41701280163
:10F6D0008DE490E0A596AEADBFADA597A89FF001D3
:10F6E000A99FF00DB89FF00D1124E251F04F22A117
:10F6F00033A144A155A129A33AA34BA35CA3C20102
:10F70000B1010E9435D787FD04C029A03AA04BA0C3
:10F710005CA04DA15EA1423051050CF405C1509191
:10F72000C014CB56DF4F5883C559D0406091C114E7
:10F73000CA56DF4F6883C659D0407091C214C9566B
:10F74000DF4F7883C759D0408091C314C856DF4F2C
:10F750008883C859D040652FCA56DF4F7881C65973
:10F76000D040C956DF4F8881C759D040C856DF4FB7
:10F770009881C859D04027E137EB41ED58E30E940A
:10F7800043D918160CF0D0C069897A898B899C8975
:10F790002091C4143091C5144091C6145091C714DF
:10F7A0000E945BD69B01AC010E9415DA7B018C01A3
:10F7B0006D897E898F89988D2091C8143091C914E4
:10F7C0004091CA145091CB140E945BD69B01AC01AE
:10F7D0000E9415DA9B01AC01C801B7010E945CD6FA
:10F7E0000E9482DA7B018C01A40193010E9443D91B
:10F7F00018165CF00F2EF0E06F2EF0E07F2EF0E890
:10F800008F2EFFE39F2EF02D08C0C401B301A80185
:10F8100097010E943CD73B014C016DA97EA98FA99D
:10F8200098AD2091CC143091CD144091CE145091CC
:10F83000CF140E945BD67B018C01E89417F9C801B4
:10F84000B70129A93AA94BA95CA90E9443D9181666
:10F8500094F469A97AA98BA99CA9A80197010E948F
:10F860003CD75B016C01C401B301A60195010E9464
:10F8700035D7882314F4640153016DA57EA58FA5A7
:10F8800098A92091D0143091D1144091D214509164
:10F89000D3140E945BD67B018C01E89417F9C80150
:10F8A000B70129A53AA54BA55CA50E9443D9181616
:10F8B00094F469A57AA58BA59CA5A80197010E943F
:10F8C0003CD77B018C01C601B501A80197010E94BC
:10F8D00035D7882314F48601750169A17AA18BA11B
:10F8E0009CA1A80197010E9415DA7B018C01CB56DF
:10F8F000DF4F6881C559D040CA56DF4F7881C6595D
:10F90000D040C956DF4F8881C759D040C856DF4F15
:10F910009881C859D040A80197010E9435D787FD2A
:10F9200019C0D801C70102C0D201C101CB56DF4FB7
:10F930008883C559D040CA56DF4F9883C659D040F6
:10F94000C956DF4FA883C759D040C856DF4FB88388
:10F95000C859D0408DE490E0A596AEADBFADA59757
:10F96000A89F8001A99F100DB89F100D112402516E
:10F97000104FCB56DF4F8881C559D040CA56DF4F54
:10F980009881C659D040C956DF4FA881C759D04089
:10F99000C856DF4FB881C859D040F80182A793A755
:10F9A000A4A7B5A762A973A984A995A9905820E036
:10F9B00030E040E050EC0E9415DAD8019E962D917F
:10F9C0003D914D915C91D1970E9415DA2BE037ED76
:10F9D00043E25BE30E945CD60E9482DAF62EE72EB9
:10F9E000D82EC92ECB56DF4F6881C559D040CA5694
:10F9F000DF4F7881C659D040C956DF4F8881C7593B
:10FA0000D040C856DF4F9881C859D0402F2D3E2D89
:10FA10004D2D5C2D0E9435D787FD14C0CB56DF4F8E
:10FA2000F882C559D040CA56DF4FE882C659D04047
:10FA3000C956DF4FD882C759D040C856DF4FC88259
:10FA4000C859D0408DE490E0A596EEADFFADA597E6
:10FA5000E89F8001E99F100DF89F100D11240251BD
:10FA6000104FCB56DF4F8881C559D040CA56DF4F63
:10FA70009881C659D040C956DF4FA881C759D04098
:10FA8000C856DF4FB881C859D040F80186A397A364
:10FA9000A0A7B1A762A173A184A195A12F2D3E2D8E
:10FAA0004D2D5C2D0E9435D718162CF081E0D80121
:10FAB000D7968C9302C0F80117AA8DE490E0A59622
:10FAC0002EAD3FADA597289FF001299FF00D389FDF
:10FAD000F00D1124E251F04F81E086ABA4ECB4E1CB
:10FAE000FE01719680E101900D928150E1F78DE465
:10FAF00090E0A5964EAD5FADA597489F6001499FE8
:10FB0000D00C589FD00C11246EEE7FE0C60ED71E8D
:10FB1000D6019296ED90FD900D911C919597E092F3
:10FB2000C014F092C1140093C2141093C31496969B
:10FB30006D917D918D919C919997A80197010E945B
:10FB40003CD74B015C01C201B101A80197010E94A1
:10FB50003CD78B019C01C601B501A4010E94D26F64
:10FB6000BFA1B093BE14C157DF4F288139814A81AC
:10FB70005B81CF58D0402093E90F3093EA0F409338
:10FB8000EB0F5093EC0FC557DF4F488159816A81C5
:10FB90007B81CB58D0404093E50F5093E60F6093A4
:10FBA000E70F7093E80FC957DF4F688179818A8129
:10FBB0009B81C758D0406093E10F7093E20F809310
:10FBC000E30F9093E40FCD57DF4F88819981AA818D
:10FBD000BB81C358D0408093DD0F9093DE0FA0937C
:10FBE000DF0FB093E00F0E9456720E941391C4562B
:10FBF000DF4F0FB6F894DEBF0FBECDBFCF91DF91C0
:10FC00001F910F91FF90EF90DF90CF90BF90AF903A
:10FC10009F908F907F906F905F904F903F902F902C
:10FC20000895FF920F931F93CF93DF938B010E9450
:10FC300069D0EB01FF24FA9409C00E9469D06C1BC3
:10FC40007D0B6017710710F080E008C0FEBC0DB49A
:10FC500007FEFDCF8EB58F3F81F781E0DF91CF9119
:10FC60001F910F91FF900895FC014281242F30E0F5
:10FC7000C9019595879580658CBD40FF02C080E0E5
:10FC800004C080E0463009F081E08DBD808160E0F5
:10FC90000E9413D20895DF92EF92FF920F931F9369
:10FCA000CF93DF93EC01D62E79018A010E94347E36
:10FCB000CE016CE271E00E94117E8D2D80648EBDBC
:10FCC0000DB407FEFDCF28E130E0D801C701022EB8
:10FCD00004C0B695A795979587950A94D2F78EBDDF
:10FCE0000DB407FEFDCF285030408FEF283F380776
:10FCF00061F7DD2011F485E906C088E0D81611F41B
:10FD000087E801C08FEF8EBD0DB407FEFDCF8CE0FC
:10FD1000D81631F48FEF8EBD0DB407FEFDCF8EB532
:10FD20009FEF2FEF2EBD0DB407FEFDCF8EB587FFE1
:10FD300004C0992311F09150F5CF8B83DF91CF91BF
:10FD40001F910F91FF90EF90DF900895FC0180814B
:10FD500061E00E9413D20895DC016EBDFA0120E03B
:10FD600030E00DB407FEFDCF80818EBD0DB407FEDF
:10FD7000FDCF81818EBD2E5F3F4F329682E02030D5
:10FD8000380779F70DB407FEFDCF8FEF8EBD0DB4A8
:10FD900007FEFDCF8FEF8EBD0DB407FEFDCF8FEFB9
:10FDA0008EBD0DB407FEFDCF8EB513968C931397C1
:10FDB0008F71853011F481E0089583E111968C9361
:10FDC0001197CD010E94A67E80E00895CF92DF9228
:10FDD000EF92FF920F931F93CF93DF93EC017A0181
:10FDE0008B0169018C81833039F059E0EE0CFF1CE6
:10FDF000001F111F5A95D1F7CE0168E1A8019701A4
:10FE00000E944B7E882311F086E023C0CE016EEF66
:10FE1000A6010E94AC7E8823E9F0CE0168E572E07D
:10FE20000E94117E882311F487E113C0CE016DE09A
:10FE300020E030E040E050E00E944B7E882341F417
:10FE40008FEF8EBD0DB407FEFDCF8EB5882379F000
:10FE500086E18983CE010E94A67E80E0DF91CF916A
:10FE60001F910F91FF90EF90DF90CF900895CE01FA
:10FE70000E94A67E81E0F2CFBF92CF92DF92EF92F6
:10FE8000FF920F931F93CF93DF93EC016B017A01E5
:10FE90000E9469D08B01BB24BA9409C00E9469D02A
:10FEA000601B710B6D52714010F081E10BC0BEBC44
:10FEB0000DB407FEFDCF8EB58B838F3F79F38E3F58
:10FEC00039F08FE08983CE010E94A67E80E02FC0AA
:10FED000D7011197EF28D9F08FEF8EBD20E030E0E9
:10FEE0009FEF0BC00DB407FEFDCF8EB5F601E20FFC
:10FEF000F31F80839EBD2F5F3F4F2A173B0790F370
:10FF00000DB407FEFDCF8EB5AC0DBD1D8C938FEFEC
:10FF10008EBD0DB407FEFDCF8EB58FEF8EBD0DB437
:10FF200007FEFDCF8EB5CE010E94A67E81E0DF9157
:10FF3000CF911F910F91FF90EF90DF90CF90BF90E6
:10FF40000895CF92DF92EF92FF920F931F93CF937A
:10FF5000DF93EC017A018B0169018C81833039F0E8
:10FF6000A9E0EE0CFF1C001F111FAA95D1F7CE01CE
:10FF700061E1A80197010E944B7E882339F084E05B
:10FF80008983CE010E94A67E80E006C0CE01B60124
:10FF900040E052E00E943C7FDF91CF911F910F9192
:10FFA000FF90EF90DF90CF900895BF92CF92DF92B5
:10FFB000EF92FF920F931F93CF93DF93EC01B62E36
:10FFC0001C82198248830E9469D06B01888161E09C
:10FFD0000E9496D1CE010E94A67E86E060E00E943B
:10FFE00096D185E061E00E9496D187E061E00E94B1
:10FFF00096D184E061E00E9496D184E061E00E94A5
:020000021000EC
:1000000013D285E08A8382E58CBD1DBC80E09FEF22
:100010009EBD0DB407FEFDCF8F5F8A30C9F709C0C2
:100020000E9469D06C197D09615D774010F081E014
:100030005EC0CE0160E020E030E040E050E00E9491
:100040004B7E182F8B83813059F7CE0168E02AEA66
:1000500031E040E050E00E944B7E82FF02C01C83F2
:1000600011C080E02FEF2EBD0DB407FEFDCF9EB571
:100070008F5F8430C1F79B839A3A11F082E037C0DA
:1000800082E08C838C81823021F0EE24FF24870172
:100090000FC0E12CF12C012D00E4102F09C00E94AB
:1000A00069D06C197D09615D774010F08AE01FC04E
:1000B000CE0167E320E030E040E050E00E944B7E5C
:1000C000CE0169E2A80197010E944B7E8B838823B1
:1000D00031F78C81823029F5CE016AE320E030E0EF
:1000E00040E050E00E944B7E882331F088E0898315
:1000F000CE010E94A67E21C08FEF8EBD0DB407FEFB
:10010000FDCF8EB5807C803C11F483E08C8380E051
:100110009FEF9EBD0DB407FEFDCF2EB58F5F8330E0
:10012000C1F7CE010E94A67E86E08B1518F488E107
:10013000898303C0BA8281E001C080E0DF91CF9162
:100140001F910F91FF90EF90DF90CF90BF90089597
:10015000CF93DF93EB01DC0190E020E03EE28C9155
:10016000803269F0283029F4FE01E90FF11D308357
:100170009F5FFE01E90FF11D8C9180839F5F2F5FD0
:1001800011962B3061F7C90FD11D1882DF91CF91E5
:1001900008950F931F93CF93DF93DC01EB018A0146
:1001A00080E090E020E2FE01E80FF91F2083019635
:1001B0008B309105C1F757E040E024C0622F2E320A
:1001C00019F083EC9AE007C05A3051F15AE048E048
:1001D00018C0321729F1FC01019634913323C9F775
:1001E0005417F0F02132E0F02F37D0F4822F8156EF
:1001F0008A3110F4622F6052FE01E40FF11D60831A
:100200004F5F11962C91222311F02F32B9F6F8018D
:10021000B183A08390E08881803219F091E001C021
:1002200090E0892FDF91CF911F910F9108956F92E8
:100230007F928F929F92AF92BF92CF92DF92EF9276
:10024000FF920F931F93CF93DF93EC017A018B0101
:100250002B81222309F480C089899A89AB89BC89C2
:1002600084179507A607B70708F476C085C0E11480
:10027000F1040105110551F41C821D821E821F82AA
:10028000188619861A861B8681E067C028853985FD
:100290004A855B85E98DFA8D858590E00996215028
:1002A00030404040504039014A01082E04C0969425
:1002B0008794779467940A94D2F72F5F3F4F4F4FFC
:1002C0005F4F0894E108F10801091109570168011D
:1002D00004C0D694C794B794A7948A95D2F708948B
:1002E000E11CF11C011D111DA614B704C804D9049A
:1002F00028F0211531054105510549F48D899E8964
:10030000AF89B88D8C839D83AE83BF8316C0A6183A
:10031000B708C808D90811C04C815D816E817F8102
:10032000898D9A8D94010E94C68C0894A108B10809
:10033000C108D108882331F40FC084E0882E912CA5
:100340008C0E9D1EA114B104C104D10429F7E886C6
:10035000F9860A871B8798CF80E0DF91CF911F91A4
:100360000F91FF90EF90DF90CF90BF90AF909F9054
:100370008F907F906F900895223009F078CFE7CF6B
:10038000CF93DF93EC018C859D85AE85BF8540E0E2
:10039000611141E0BC01CD010E949C8A882319F4BF
:1003A00020E030E00AC08889282F30E095E0220F55
:1003B000331F9A95E1F722523B4EC901DF91CF914D
:1003C00008950F931F93CF93DF938C01FC018381DA
:1003D0008823E1F1818187FF36C0C80161E00E9476
:1003E000C081EC01009791F18881853E79F1F80197
:1003F0008381823040F481899289A389B4898C8F6A
:100400009D8FAE8FBF8FF80185899689A789B08DA2
:100410009B8F8A8FCD01AA27BB279D8B8C8BE09168
:10042000D814F091D914309751F0BE016A5E7F4F15
:10043000CE0148960995888D998D9B8B8A8BF80102
:1004400081818F7781830E94618A04C081E0F801F5
:10045000808380E0DF91CF911F910F9108950F93DA
:100460001F938C010E94E181F80113821F910F916B
:100470000895FC018381882319F0CF010E942F8207
:100480000895CF93DF93FC01EB018381882391F0E2
:100490008250823020F48FE28883198209C0CF0114
:1004A00060E00E94C081009729F0BE010E94A880F0
:1004B00081E001C080E0DF91CF9108956F927F923B
:1004C0008F929F92AF92BF92CF92DF92EF92FF9264
:1004D0000F931F93DF93CF9300D000D0CDB7DEB73B
:1004E0007C015A016B01DC0113968C9113978130CA
:1004F00009F091C011968C9181FF8DC0A0C000972A
:10050000A105B10511F481E087C0F7016084718411
:1005100082849384C701B601A5010E9417818823B4
:1005200009F479C0D70159968D919C915A97A114DD
:10053000B104C104D10489F455964D915D916D913A
:100540007C9158970E943C8D882309F464C0F70180
:10055000158A168A178A108E44C0D70114964D91B9
:100560005D916D917C9117979E012F5F3F4F0E9487
:10057000C68C882309F44FC0D7015996ED91FC91A0
:100580005A9749815A816B817C818789803149F4EE
:10059000483FBFEF5B07B0E06B07B0E07B0748F078
:1005A00020C0483F8FEF58078FEF68078FE078072C
:1005B000C0F4CF010E943C8D882369F1D7011496C5
:1005C0004D915D916D917C91179759968D919C916C
:1005D0005A970FEF1FEF2FEF3FE00E943F8C8823C9
:1005E000D1F0F701A18AB28AC38AD48A8181806856
:1005F0008183C7010E94E181882369F0B601A501CA
:100600006A147B048C049D0410F4B401A301C70197
:100610000E94178101C080E00F900F900F900F9003
:10062000CF91DF911F910F91FF90EF90DF90CF90CE
:10063000BF90AF909F908F907F906F900895F7013B
:1006400081899289A389B48984179507A607B7077A
:1006500008F055CFE0CFCF93DF93EC0140E050E0BE
:1006600060E070E00E945E82882369F0CE0161E064
:100670000E94C081FC01009731F085EE80831B82CF
:100680000E94618A01C080E0DF91CF9108952F928E
:100690003F924F925F926F927F928F929F92AF9212
:1006A000BF92CF92DF92EF92FF920F931F93CF935F
:1006B000DF93EC012A018B81882309F4B6C089817C
:1006C00080FFB3C0C8C025014E185F083B0174E02D
:1006D000272E312C2C0E3D1E4201A1C028853985C4
:1006E0004A855B856FEFA62E61E0B62EA222B3226B
:1006F0008B8179018A0199E016950795F794E79423
:100700009A95D1F7E98DFA8D823049F4428D538D57
:10071000648D758D4E0D5F1D601F711F3FC0D480AD
:10072000DA94DE20A114B104D9F4DD20C9F4211536
:1007300031054105510549F48D899E89AF89B88DF0
:100740008C839D83AE83BF830BC04C815D816E81A2
:100750007F81CF0191010E94C68C882309F465C076
:10076000E98DFA8D4C815D816E817F8142505040D0
:1007700060407040058404C0440F551F661F771FFA
:100780000A94D2F786859785A089B189480F591FA9
:100790006A1F7B1F4D0D511D611D711D80E092E090
:1007A0008A199B0984018815990508F48C0182E057
:1007B0000030180709F067C08091DA149091DB14BB
:1007C000A091DC14B091DD14481759076A077B0724
:1007D00009F459C08091DE169091DF1693010E94B2
:1007E000A17F882349F421C0950122523B4EC301C9
:1007F000B901A8010E94B124600E711E980140E069
:1008000050E088859985AA85BB85820F931FA41F18
:10081000B51F88879987AA87BB87801A910A811498
:10082000910409F05BCFA20102C04FEF5FEFCA0154
:10083000DF91CF911F910F91FF90EF90DF90CF90BC
:10084000BF90AF909F908F907F906F905F904F90F0
:100850003F902F900895A988BA88CB88DC88E884D7
:10086000F9840A851B859A0140E050E0D601C50154
:100870008E199F09A00BB10B281739074A075B0790
:1008800008F021CF23CFCB01BA0140E00E949C8A1F
:10089000882309F0A9CFC9CFCF92DF92EF92FF92C0
:1008A0000F931F93CF93DF937C01EB018A01FC012F
:1008B0008381823008F46FC080859185A285B385DD
:1008C0008F719070A070B0700097A105B10509F00C
:1008D00062C06DC0F8011082EDE0CE2ED12CC701B0
:1008E000BE0140E250E00E9447839C0180329105A6
:1008F00021F0009709F04FC050C04881442309F40B
:100900004CC0453E61F34E3251F38B858F738F306F
:10091000E9F501151105D1F18A8D9B8D892BB1F572
:10092000842F90E08F719070009781F18330910552
:100930006CF58C9D90018D9D300D9C9D300D11248A
:100940002D503040F801E20FF31F898180838B81A5
:1009500081838D8182838F818383898584838E8542
:100960008583888986838A8987838C8980878E8915
:100970008187888D82878C8D83878E8D84878881FF
:1009800086FF04C0F801E20FF31F15868B8583FDF7
:10099000A6CF822F03C08FEF01C080E0DF91CF91FF
:1009A0001F910F91FF90EF90DF90CF900895411528
:1009B000510509F08FCF90CFDF93CF930F92CDB732
:1009C000DEB7BE016F5F7F4F41E050E00E9447837A
:1009D000019719F02FEF3FEF03C08981282F30E0F6
:1009E000C9010F90CF91DF910895EF92FF920F937D
:1009F0001F93CF93DF93EC018B81823038F1E88431
:100A0000F9840A851B85CE010E94DC8497FD1EC0F7
:100A100088859985AA85BB854F96A11DB11D8887BC
:100A20009987AA87BB87A5E016950795F794E79461
:100A3000AA95D1F72E2D30E02F703070F5E0220FFF
:100A4000331FFA95E1F722523B4E02C020E030E01E
:100A5000C901DF91CF911F910F91FF90EF90089501
:100A60000F931F93CF93DF93EC018B018B8188232E
:100A700009F040C0FB018789803109F041C082E064
:100A80008B831D8A1E8A1F8A188E808D918DA0E00F
:100A9000B0E045E0880F991FAA1FBB1F4A95D1F708
:100AA000898B9A8BAB8BBC8B13C083E08B83F80153
:100AB000428D538D648D758D4D8B5E8B6F8B788FD2
:100AC0009E012F5E3F4FC8010E949A8D882391F0AE
:100AD0001A8F098F81E089831C821D821E821F82EA
:100AE000188619861A861B861C861D861E861F86FA
:100AF000188A01C080E0DF91CF911F910F91089576
:100B00008032C1F7D2CF1F93CF93DF93EC01142F24
:100B1000262F30E0F90175E0EE0FFF1F7A95E1F71F
:100B2000E252FB4E8385817121F0842F827109F09E
:100B300069C08091DA149091DB14A091DC14B0911B
:100B4000DD148C879D87AE87BF87688BF90165E0D0
:100B5000EE0FFF1F6A95E1F7E252FB4E84899589FB
:100B6000A0E0B0E0DC01992788278D8B9E8BAF8BAE
:100B7000B88F228D338DA90160E070E0482B592B8E
:100B80006A2B7B2B4D8B5E8B6F8B788F838590E0F0
:100B900088719070009751F4848D958DA68DB78DD6
:100BA000898B9A8BAB8BBC8B81E00CC0409751F545
:100BB0009E012F5E3F4F898D9A8D0E949A8D8823CA
:100BC00009F184E08B83812F8F7089831C821D82C1
:100BD0001E821F82188619861A861B8614FF18C06B
:100BE000CE0140E050E060E070E00E945E82882329
:100BF00079F40AC049895A896B897C89CE010E949F
:100C0000178102C01B8280E0DF91CF911F91089570
:100C100015FDF0CF81E0F8CFCF93DF93EC019C017D
:100C20002C5F3F4F898D9A8D41E050E060E070E08D
:100C30000E94068E8823A1F08D899E89AF89B88D88
:100C40000097A105B10559F48C819D81AE81BF81CA
:100C50008D8B9E8BAF8BB88F89818068898381E073
:100C6000DF91CF9108952F923F924F925F927F92A2
:100C70008F929F92AF92BF92CF92DF92EF92FF92AC
:100C80000F931F93DF93CF9300D000D000D0CDB748
:100C9000DEB76C01162F072F5E834D83DC011396A0
:100CA0008C911397813009F06FC111968C9181FF5F
:100CB0006BC188C1F6014189528963897489808535
:100CC0009185A285B38584179507A607B70731F0EC
:100CD000C6010E941781882309F456C1812F902FE5
:100CE0009C0119014D805E8013C1D6015996ED918A
:100CF000FC915A97DA01C90149E0B695A7959795F5
:100D000087954A95D1F774807A9478228FEF882E50
:100D100081E0982E82229322772009F053C081141B
:100D2000910409F04FC0D60114964D915D916D91DB
:100D30007C911797411551056105710581F4559610
:100D40008D919D910D90BC91A02D0097A105B105AD
:100D500061F1F60184839583A683B78333C0CF0105
:100D60009E012F5F3F4F0E94C68C882309F40CC15F
:100D700029813A814B815C81D6015996ED91FC9194
:100D80005A978789803149F4283FBFEF3B07B0E08D
:100D90004B07B0E05B0778F008C0283FEFEF3E0755
:100DA000EFEF4E07EFE05E0730F0C6010E940C86C1
:100DB000882341F4E9C0D60114962D933D934D93B9
:100DC0005C93179780E092E0881999095201841585
:100DD000950508F45C01D6015996ED91FC915A975E
:100DE0001496ED90FD900D911C9117978EEF9FEF4B
:100DF000AFEFBFEFE80EF91E0A1F1B1F058404C0EA
:100E0000EE0CFF1C001F111F0A94D2F786859785F0
:100E1000A089B189E80EF91E0A1F1B1FE70CF11CFF
:100E2000011D111D90E0A91692E0B90639F58091D7
:100E3000DA149091DB14A091DC14B091DD148E15BE
:100E40009F05A007B10771F41092E0168FEF9FEF96
:100E5000AFEFBFEF8093DA149093DB14A093DC1410
:100E6000B093DD148091DE169091DF16B801A701D2
:100E700091010E94E67E8823B9F586C08114910411
:100E800019F5D60118962D913D914D915C911B97C6
:100E900051968D919D910D90BC91A02D28173907E9
:100EA0004A075B0788F00E94618A882309F46CC0B6
:100EB00081E08093E016E092DA14F092DB14009364
:100EC000DC141093DD1408C0C801B70141E00E9492
:100ED0009C8A882309F458C0940122523B4EC901D0
:100EE000B101A5010E94B124950140E050E0F60156
:100EF00080859185A285B385820F931FA41FB51F9E
:100F000080879187A287B3872A0C3B1C4A185B080D
:100F1000D60118962D913D914D915C911B974114EE
:100F2000510409F0E2CE51968D919D910D90BC91A6
:100F3000A02D82179307A407B50748F4F601218B6B
:100F4000328B438B548B81818068818311C0809167
:100F5000D8149091D914892B59F08D819E81892BB9
:100F600039F0D60111968C911197806811968C9367
:100F7000F601818183FF05C0C6010E94E1818823BB
:100F800019F04D815E8105C081E0D6018C934FEF51
:100F90005FEFCA0126960FB6F894DEBF0FBECDBF35
:100FA000CF91DF911F910F91FF90EF90DF90CF9045
:100FB000BF90AF909F908F907F905F904F903F90A9
:100FC0002F90089582FD76CE89CEDF92EF92FF9228
:100FD0000F931F93CF93DF93EC0189899A89AB8993
:100FE000BC89805E9F4FAF41B04008F071C0CE0118
:100FF0000E940C86882309F46BC00E94618A8823B2
:1010000009F466C0E98DFA8DEC80FD800E811F81A8
:101010008EEF9FEFAFEFBFEFE80EF91E0A1F1B1F09
:10102000058404C0EE0CFF1C001F111F0A94D2F7A8
:1010300086859785A089B189E80EF91E0A1F1B1FB6
:1010400081E08093E016E092DA14F092DB140093D2
:10105000DC141093DD1480E092E0EEEDF4E1DF01AA
:101060009C011D9221503040E1F7DD24D39411C042
:10107000B801A7014D0D511D611D711D8091DE1636
:101080009091DF162EED34E10E94E67E882301F177
:10109000D394E98DFA8D8481D81650F320E032E0A4
:1010A00040E050E0058404C0220F331F441F551F49
:1010B0000A94D2F789899A89AB89BC89820F931FD8
:1010C000A41FB51F898B9A8BAB8BBC8B81E001C0B1
:1010D00080E0DF91CF911F910F91FF90EF90DF9013
:1010E00008958F929F92AF92BF92CF92DF92EF922C
:1010F000FF920F931F93CF93DF936C01EB01942E1C
:10110000852EA22E898D9A8DD6015A969C938E9308
:101110005997CB0140E050E060E070E00E941781F9
:10112000BB2438C0CE010E94F584FC01009709F46D
:1011300093C055E016950795F794E7945A95D1F723
:101140001E2D1F708081882311F0853EC9F4BB20BD
:1011500099F42091DA143091DB144091DC14509111
:10116000DD14D6011C962D933D934D935C931F97F0
:1011700050961C93BB24B3948081882359F418C0E3
:10118000892D982DBF014BE050E00E94A4240097C8
:1011900009F470C0E884F9840A851B8589899A89D5
:1011A000AB89BC89E816F9060A071B0708F4BACF11
:1011B000A6FE52C0A1FE50C0BB2051F0F60110891E
:1011C000C60161E00E94C081EC01009769F444C04F
:1011D0008B81823009F440C0CE010E94E5878823CC
:1011E000D9F110E0CEEDD4E180E2DE011D928A95C6
:1011F000E9F7DE01292D382DC901FC018BE00190B2
:101200000D928150E1F7E091D814F091D914309704
:1012100039F0BE01625F7F4FCE014096099508C04C
:1012200081E298E2998B888B80E098E09F878E8797
:10123000888999899B8B8A8B998F888F8E859F85CA
:101240009F8B8E8B0E94618A882331F0C601612FAB
:101250004A2D0E94838501C080E0DF91CF911F91CC
:101260000F91FF90EF90DF90CF90BF90AF909F9045
:101270008F900895A7FEEACFEFCF2F923F924F9223
:101280005F926F927F928F929F92AF92BF92CF9216
:10129000DF92EF92FF920F931F93DF93CF93CDB71F
:1012A000DEB7C654D0400FB6F894DEBF0FBECDBF38
:1012B0003C016B01DE01AE5BBF4F11965C934E9318
:1012C00025962FAF25971C861F861FA21AA661158B
:1012D000710509F480C0FC018381882309F07BC07B
:1012E000FA0180818F32F1F08601ECE0EE2EF12CD4
:1012F000EC0EFD1E72E4A72EB12CAC0EBD1E4E01ED
:101300000894811C911C2796FFAEEEAE279767E2EA
:10131000262E312C2C0E3D1E270124C01196B183A0
:10132000A08301C0FD01A081B1818C918F32B1F306
:10133000D60113968C91139782508230A8F28E01B9
:10134000095D1F4F59966D917C915A97C8010E9473
:101350003085882351F63FC0342D252D8701832FFA
:10136000922F7C01F50180819181B401A5010E9439
:10137000C980882329F42FC03196D501ED93FC93C1
:10138000D501ED91FC9180818F32B1F38823C9F0B2
:10139000C701B801A40121E00E9471888823D9F017
:1013A0000C151D0519F0C8010E942F822796EEAD7D
:1013B000FFAD2797EE16FF0679F6C101322D292FD2
:1013C000CDCFC301B801A40125962FAD25970E946A
:1013D0007188182F01C010E0CE0187960E943982D3
:1013E000CE010C960E943982812FCA5BDF4F0FB667
:1013F000F894DEBF0FBECDBFCF91DF911F910F914B
:10140000FF90EF90DF90CF90BF90AF909F908F9024
:101410007F906F905F904F903F902F9008950F9323
:101420001F93DF93CF93CDB7DEB76B970FB6F894CA
:10143000DEBF0FBECDBF9C01AB0119821C828E01A5
:101440000F5F1F4FC801B90122E00E943D89882328
:1014500011F410E004C0C8010E942B83182FCE01A4
:1014600001960E943982812F6B960FB6F894DEBFE9
:101470000FBECDBFCF91DF911F910F910895DB017A
:101480000D900020E9F71197A61BB70B0496AD014C
:101490000E9433860895DF93CF930F92CDB7DEB7C6
:1014A00069830496BE016F5F7F4F41E050E00E9468
:1014B00033860F90CF91DF91089504960E94338672
:1014C00008958091E016882399F14091DA145091A3
:1014D000DB146091DC147091DD148091DE16909124
:1014E000DF162EED34E10E94E67E882319F140914B
:1014F000E1165091E2166091E3167091E4164115E1
:1015000051056105710591F08091DE169091DF160D
:101510002EED34E10E94E67E882361F01092E11600
:101520001092E2161092E3161092E4161092E01652
:1015300081E0089580E00895DF92EF92FF920F938B
:101540001F937B018C01D42E8091DA149091DB14CF
:10155000A091DC14B091DD148E159F05A007B10792
:10156000C1F00E94618A8823E1F08091DE1690919B
:10157000DF16B801A7012EED34E10E94A17F882378
:1015800081F0E092DA14F092DB140093DC141093F3
:10159000DD14DD2011F481E005C081E08093E016C8
:1015A00001C080E01F910F91FF90EF90DF900895B0
:1015B0008F929F92AF92BF92CF92DF92EF92FF9263
:1015C0000F931F93CF93DF936C01142F7093DF164B
:1015D0006093DE16FC01178A82E090E0A0E0B0E0A4
:1015E00080839183A283B3831092E0161092E11658
:1015F0001092E2161092E3161092E4168FEF9FEF0E
:10160000AFEFBFEF8093DA149093DB14A093DC1458
:10161000B093DD14442321F488249924540140C05C
:10162000453008F01EC160E070E080E090E040E0EE
:101630000E949C8A882309F414C1C12FD0E021970D
:10164000FE0174E0EE0FFF1F7A95E1F7E252FB4EC8
:10165000E254FE4F8081EE5BF14090E08F77907016
:10166000892B09F0FEC0E653FE4F80819181A28153
:10167000B38184369105A105B10508F4F2C064E098
:10168000CC0FDD1F6A95E1F7CC55D94E8880998043
:10169000AA80BB8081149104A104B10409F4E1C0C3
:1016A000C501B40140E00E949C8A882309F4D9C096
:1016B0008091E9149091EA148050924009F0D1C0D1
:1016C0002091EE14222309F4CCC08091EC14909167
:1016D000ED14892B09F4C5C08091EB14882309F41B
:1016E000C0C0F601228B8091EB148483158661E0E3
:1016F00070E007C04F5FF60145874150483008F061
:10170000B0C0F6014585848190E09B01042E02C0A3
:10171000220F331F0A94E2F78217930759F720919B
:10172000F4143091F5142115310519F040E050E022
:1017300008C0209102153091031540910415509175
:101740000515F6012583368347835087E090EC1416
:10175000F090ED1400E010E0E80CF91C0A1D1B1DD0
:10176000E38AF48A058B168B8091EF149091F01424
:10177000918F808F6091EE1470E080E090E00E9485
:10178000E7DA6E0D7F1D801F911FF601628F738F48
:10179000848F958F2091EF143091F01455E0220F33
:1017A000331F5A95E1F721503E4F232F33272695BB
:1017B00040E050E0260F371F481F591F2687378704
:1017C000408B518B8091F1149091F214009719F095
:1017D000A0E0B0E008C08091FE149091FF14A091A9
:1017E0000015B091011585017401E21AF30A040B8A
:1017F000150BA8019701280F391F4A1F5B1FF6011F
:10180000058404C056954795379527950A94D2F7D5
:101810002187328743875487253FFFE03F07F0E069
:101820004F07F0E05F0720F48CE0F601878B19C0CA
:10183000255F3F4F4040504018F480E1F6010EC054
:1018400080910A1590910B15A0910C15B0910D1572
:10185000F601828F938FA48FB58F80E2878B81E012
:1018600001C080E0DF91CF911F910F91FF90EF9029
:10187000DF90CF90BF90AF909F908F9008956F9220
:101880007F928F929F92AF92BF92CF92DF92EF9210
:10189000FF920F931F93CF93DF93EC015A016B01DB
:1018A00038014901423051056105710508F45EC0F7
:1018B00089859A85AB85BC850196A11DB11D8417CC
:1018C0009507A607B70708F451C08F89803129F41E
:1018D000E52EF62E072F11270CC0803209F046C0E6
:1018E0007A018B0187E016950795F794E7948A951E
:1018F000D1F78B899C89AD89BE89E80EF91E0A1F34
:101900001B1FC801B70141E00E949C8A882371F126
:101910008F89803149F4F501F070EE0FFF1FE2521C
:10192000FB4E718260820DC0F501EF77F070EE0F13
:10193000FF1FEE0FFF1FE252FB4E60827182828218
:1019400093828A89823080F08D819E81AF81B885B3
:10195000E80EF91E0A1F1B1FE092E116F092E21634
:101960000093E3161093E41681E001C080E0DF915C
:10197000CF911F910F91FF90EF90DF90CF90BF908C
:10198000AF909F908F907F906F900895CF92DF924D
:10199000EF92FF920F931F93CF93DF93EC017A01A5
:1019A0008B01690189859A85AB85BC850196A11D4E
:1019B000B11D84179507A607B70708F453C08F8990
:1019C000803129F45527412F302F2F2D0CC0803224
:1019D00009F048C09A01AB0167E0569547953795E5
:1019E00027956A95D1F78B899C89AD89BE89280F87
:1019F000391F4A1F5B1F8091DA149091DB14A0916C
:101A0000DC14B091DD14281739074A075B0739F059
:101A1000CA01B90140E00E949C8A882319F18F898C
:101A2000803159F4F701F070EE0FFF1FE252FB4EC8
:101A300080819181A0E0B0E00EC0F701EF77F070F7
:101A4000EE0FFF1FEE0FFF1FE252FB4E80819181D0
:101A5000A281B381BF70F60180839183A283B38397
:101A600081E001C080E0DF91CF911F910F91FF9045
:101A7000EF90DF90CF900895AF92BF92CF92DF9218
:101A8000EF92FF920F931F93DF93CF9300D000D07C
:101A9000CDB7DEB76C017A018B0182E090E0A0E067
:101AA000B0E0F60180839183A283B3835E01089442
:101AB000A11CB11CC601B801A70195010E94C68CEA
:101AC000882341F1C601B801A70100E010E020E041
:101AD00030E00E943F8C8823E9F0E980FA800B8196
:101AE0001C81F6018789803151F4F8EFEF16FFEF82
:101AF000FF06F0E00F07F0E01F07E0F209C088EFF3
:101B0000E8168FEFF8068FEF08078FE0180790F2BE
:101B100081E001C080E00F900F900F900F90CF9167
:101B2000DF911F910F91FF90EF90DF90CF90BF90CA
:101B3000AF9008954F925F926F927F928F929F9293
:101B4000AF92BF92CF92DF92EF92FF920F931F93CB
:101B5000DF93CF9300D000D0CDB7DEB76C014983BF
:101B60005A836B837C833901EE24FF2487012E0185
:101B70000894411C511C812CE2E09E2EA12CB12C1A
:101B800049815A816B817C81C60192010E94C68C79
:101B9000882339F1D501C401F601058404C0880FFA
:101BA000991FAA1FBB1F0A94D2F7E80EF91E0A1F3D
:101BB0001B1F29813A814B815C818789803131F4F7
:101BC000285F3F4F40405040D8F205C0285F3F4F4C
:101BD0004F4F5F40A8F2F301E082F182028313834A
:101BE00081E00F900F900F900F90CF91DF911F9198
:101BF0000F91FF90EF90DF90CF90BF90AF909F90AC
:101C00008F907F906F905F904F9008952F923F92AA
